:100000000C948A1A0C94C8860C949D860C94728663
:100010000C9447860C941C860C94F1850C94C68530
:100020000C949B850C94123D0C94033D0C94F43C71
:100030000C94BB1A0C94BB1A0C94BB1A0C94BB1AEC
:100040000C94BB1A0C94E3440C94BB1A0C94BB1A8A
:100050000C94BB1A0C94BB1A0C9498CD0C9451853B
:100060000C94BB1A0C94E1430C94BB1A0C94BB1A6D
:100070000C94BB1A0C94BB1A0C94BB1A0C94BB1AAC
:100080000C94BB1A0C94BB1A0C94BB1A0C94BB1A9C
:100090000C94BB1A0C94BB1A0C94BB1A0C94BB1A8C
:1000A0000C94BB1A0C94BB1A0C94BB1A0C94BB1A7C
:1000B0000C94BB1A0C94BB1A0C94BB1A0C94BB1A6C
:1000C0000C94BB1A0C94BB1A0C94BB1A0C94BB1A5C
:1000D0000C94BB1A0C94BB1A0C94BB1A0C94BB1A4C
:1000E0000C94BB1ABE5EC75ED15EDA5EE35EFE5E56
:1000F0000B5F145FEC5EF55EEE82F182E082E482DB
:10010000EA822883F582F982FF82038307830D83C5
:100110001183158328831B831F8323836D8472843B
:10012000778481848B84048595849D84A584AF84A1
:10013000B984C384D284DC840485E684F084FA84A0
:10014000084AD73B3BCE016E84BCBFFDC12F3D6C3E
:1001500074319ABD56833DDA3D00C77F11BED9E4A4
:10016000BB4C3E916BAAAABE000000803F05A84C84
:10017000CDB2D44EB93836A9020C50B99186880850
:100180003CA6AAAA2ABE000000803F004E414E496C
:100190004E495459494E46CDCCCC3D0AD7233C1745
:1001A000B7D13877CC2B329595E6241FB14F0A0092
:1001B0000020410000C84200401C4620BCBE4CCA82
:1001C0001B0E5AAEC59D74434F4D4D554E4943418C
:1001D00054494F4E0044525952554E004552524FC9
:1001E000525300494E464F004543484F0020746F1C
:1001F0006F206C6F6E6720657874727573696F6EAF
:100200002070726576656E7465640A0020636F6C99
:100210006420657874727573696F6E20707265768C
:10022000656E7465640A0047322F4733206261644B
:1002300020706172616D65746572730A00536C653C
:1002400065702E2E2E00536E6170707933207265AA
:100250006164792E00526573756D696E67207072E6
:10026000696E7400436C69636B20746F20726573F0
:10027000756D652E2E2E004E6F206D6F76652E00EB
:10028000456E642066696C65206C6973740A00426F
:100290006567696E2066696C65206C6973740A0015
:1002A0004D313235005344207072696E74696E6747
:1002B000206279746520004E6F7420534420707260
:1002C000696E74696E670A0046696C652064656CC6
:1002D000657465643A0044656C6574696F6E206688
:1002E00061696C65642C2046696C653A20006F700A
:1002F000656E206661696C65642C2046696C653AA0
:1003000020002569730025696D2025697300256922
:10031000682025696D202569730025696420256999
:10032000682025696D202569730025697920256974
:1003300064202569682025696D2025697300507245
:10034000696E742074696D653A20000001363726A5
:1003500003FF3C3D380EFF2E303E1213FF0C080900
:10036000FFFFFF1A1C18FFFF08440AFF4324221E48
:10037000FFFFFFFFFFFF50726F74656374656420B9
:1003800050696E0A0045256920257300536E61701F
:100390007079332072656164792E00E801E301DC35
:1003A00001D501C7016F66660044454255473A00D2
:1003B0004B494C4C45442E20004D313133205300E5
:1003C0006F6B0048656174696E6720646F6E652E9F
:1003D0000020573A0045256920257300536E61704F
:1003E0007079332072656164792E00536E6170708C
:1003F0007933204F66662E004361703A454D455271
:1004000047454E43595F5041525345523A300A00D6
:100410004361703A434153455F4C494748545F42FA
:1004200052494748544E4553533A300A004361708D
:100430003A544F47474C455F4C49474854533A302C
:100440000A004361703A534F4654574152455F503A
:100450004F5745523A300A004361703A4C45564571
:100460004C494E475F444154413A300A0043617061
:100470003A5A5F50524F42453A300A004361703A4F
:100480004155544F4C4556454C3A300A0043617033
:100490003A5052494E545F4A4F423A310A00436142
:1004A000703A50524F47524553533A300A00436115
:1004B000703A4155544F5245504F52545F54454D38
:1004C000503A310A004361703A454550524F4D3A17
:1004D000310A004649524D574152455F4E414D4504
:1004E0003A4D61726C696E20312E312E36202847CC
:1004F00069746875622920534F555243455F434FD5
:1005000044455F55524C3A68747470733A2F2F67A4
:1005100069746875622E636F6D2F4D61726C696EC0
:100520004669726D776172652F4D61726C696E20DC
:1005300050524F544F434F4C5F56455253494F4EC4
:100540003A312E30204D414348494E455F54595071
:10055000453A536E61707079332045585452554472
:1005600045525F434F554E543A3120555549443A10
:1005700063656465326132662D343161322D343702
:1005800034382D396231322D633535633632663376
:10059000363766660A002F2F20007A325F6D696E4B
:1005A0003A20007A5F6D696E3A2000795F6D696E5E
:1005B0003A2000785F6D696E3A20005265706F7264
:1005C00074696E6720656E6473746F7020737461F4
:1005D0007475730A004D31343520533C696E64657F
:1005E000783E206F7574206F662072616E6765209B
:1005F00028302D31290A0053657474696E672054C0
:10060000726176656C20416363656C6572617469C3
:100610006F6E3A200053657474696E67205265747A
:100620007261637420416363656C65726174696FA4
:100630006E3A200053657474696E67205072696E5B
:100640007420416363656C65726174696F6E3A20F2
:100650000053657474696E67205072696E7420610E
:100660006E642054726176656C20416363656C65CD
:10067000726174696F6E3A20005A20456E6473741B
:100680006F702041646A7573746D656E7420736554
:100690007420746F20286D6D293A004F666673656B
:1006A0007473206170706C696564004572723A20E1
:1006B000546F6F206661722100546F6F2066617203
:1006C0002066726F6D207265666572656E63652067
:1006D000706F696E740A004E6F2063617365206CE1
:1006E000696768740A0041637469766520457874A7
:1006F00072756465723A2000556E6B6E6F776E206E
:10070000636F6D6D616E643A2022004E6F204C69FC
:100710006E65204E756D626572207769746820631E
:100720006865636B73756D2C204C617374204C6924
:100730006E653A20004B494C4C45442E20005354E2
:100740004F505045442E20005072696E74657220DF
:1007500073746F707065642064756520746F2065B4
:1007600072726F72732E20466978207468652065F6
:1007700072726F7220616E6420757365204D393915
:100780003920746F20726573746172742E2028543E
:10079000656D70657261747572652069732072652C
:1007A0007365742E205365742069742061667465C6
:1007B000722072657374617274696E67290A004EE3
:1007C0006F20436865636B73756D2077697468206B
:1007D0006C696E65206E756D6265722C204C61735C
:1007E00074204C696E653A2000636865636B7375AD
:1007F0006D206D69736D617463682C204C61737436
:10080000204C696E653A20004C696E65204E756D0E
:10081000626572206973206E6F74204C617374205E
:100820004C696E65204E756D6265722B312C204CC3
:10083000617374204C696E653A20004D313130008F
:100840004D3331004D383420582059205A2045006E
:1008500053442072656164206572726F720A0044AD
:100860006F6E65207072696E74696E672066696C60
:10087000650A0020496E76616C696420657874723F
:100880007564657220000000000000000000000098
:100890000000000046430000464300005C43202F58
:1008A0000020403A00205A3A0020593A0020436F75
:1008B000756E7420583A0020453A00205A3A0020BC
:1008C000593A00583A004B494C4C45442E200020E0
:1008D0002D20496E76616C69642065787472756448
:1008E0006572206E756D62657220210A00202050AD
:1008F0006C616E6E6572427566666572427974658A
:10090000733A20002046726565204D656D6F7279DF
:100910003A2000436F6D70696C65643A20466562E9
:1009200020203120323031380A00207C204175747B
:10093000686F723A202852657661724261742C2089
:10094000536E6170707920636F6E666967290A0063
:10095000323031372D31302D31302031323A303094
:1009600000204C61737420557064617465643A2092
:1009700000312E312E360A004D61726C696E0020F6
:10098000536F6674776172652052657365740A00EF
:10099000205761746368646F672052657365740AD9
:1009A000002042726F776E206F75742052657365F8
:1009B000740A002045787465726E616C205265730C
:1009C00065740A00506F77657255700A0073746120
:1009D00072740A006572726F722077726974696E40
:1009E0006720746F2066696C650A00456E647374D5
:1009F0006F70732025632025632025632025630005
:100A0000205A3A0020593A0020583A00656E647323
:100A1000746F7073206869743A2000446F6E6520AB
:100A2000736176696E672066696C652E0A004D32C7
:100A3000390024F4D43050C38E20C2A24017828BD8
:100A40007011127A910D816CD90AA861E108C7581A
:100A50006607615143061E4B5D05C145A7041A4157
:100A60001104093D9803713931034036DB026533C7
:100A70009102D4305402802E1D02632CEE01752A9F
:100A8000C501B028A001102781018F2564012B2406
:100A90004B01E0223401AC211F018D200D01801F8C
:100AA000FC00841EED00971DDF00B81CD200E61B81
:100AB000C600201BBC00641AB200B219A8000A19B3
:100AC000A0006A189900D117910040178B00B51645
:100AD000840031167E00B31579003A157300C714EF
:100AE0006F0058146A00EE13660088136300251324
:100AF0005E00C7125B006C12570015125400C11142
:100B0000510070114F0021114B00D61049008D107B
:100B100047004610440002104200C00F4000800F02
:100B20003E00420F3C00060F3B00CB0E3800930EF8
:100B300037005C0E3500270E3400F30D3200C10D76
:100B40003100900D3000600D2E00320D2D00050D8E
:100B50002C00D90C2B00AE0C2900850C29005C0C54
:100B60002700350C27000E0C2600E80B2400C40BD0
:100B70002400A00B23007D0B23005A0B2100390B0E
:100B80002100180B2000F80A1F00D90A1E00BB0A1A
:100B90001E009D0A1D00800A1D00630A1C00470AF2
:100BA0001B002C0A1B00110A1A00F7091A00DD09A4
:100BB0001900C4091900AB091900920917007B0933
:100BC0001800630917004C091600360916002009A1
:100BD00016000A091500F5081500E0081400CC08F5
:100BE0001400B8081400A4081400900813007D082D
:100BF00012006B081300580812004608120034084F
:100C00001100230811001208110001081100F0075B
:100C10001000E0071000D0071000C0071000B00758
:100C20000F00A107100091070E0083070F00740743
:100C30000F0065070E0057070E0049070E003B071F
:100C40000D002E070E0020070D0013070D000607EC
:100C50000D00F9060C00ED060D00E0060C00D406B0
:100C60000C00C8060C00BC060C00B0060C00A40664
:100C70000B0099060C008D060B0082060B00770610
:100C80000B006C060B0061060A0057060B004C06B1
:100C90000A0042060A0038060A002E060A00240648
:100CA0000A001A060A001006090007060A00FD05D8
:100CB0000900F4050900EB050900E2050900D90562
:100CC0000900D0050900C7050900BE050900B505E2
:100CD0000800AD050800A50509009C05080094055D
:100CE00008008C050800840508007C0508007405D0
:100CF00008006C050700650508005D05070056053E
:100D000008004E05070047050700400508003805A4
:100D10000700310507002A050700230507001C0509
:100D20000600160507000F05070008050600020566
:100D30000700FB040600F5040700EE040600E804C3
:100D40000600E2040700DB040600D5040600CF0419
:100D50000600C9040600C3040600BD040600B7046B
:100D60000600B1040500AC040600A6040600A004B9
:100D700005009B04060095040500900406008A0403
:100D8000050085040500800406007A04050075044A
:100D90000500700405006B0405006604050061048D
:100DA00005005C04050057040500520405004D04CD
:100DB000050048040500430405003E0404003A040D
:100DC000050035040500300404002C040500270448
:100DD0000400230405001E0404001A040400160481
:100DE0000500110404000D040400090405000404B6
:100DF000040000040400FC030400F8030400F403EE
:100E00000400F0030400EC030400E8030400E4031E
:100E10000400E0030400DC030400D8030400D4034E
:100E20000400D0030400CC030400C8030300C5037E
:100E3000030024F404D9201BC40C5C0E9804C409DC
:100E40005F0265077101F405F900FB04B300480473
:100E50008700C10369005803550003034500BE0223
:100E60003A008402310053022A00290225000402BC
:100E70002000E4011C00C8011900AF01170098010F
:100E80001400840113007101100061011000510170
:100E90000E0043010D0036010B002B010B00200159
:100EA0000B00150109000C01090003010800FB00FB
:100EB0000800F3000800EB000700E4000600DE0075
:100EC0000600D8000600D2000600CC000500C700CE
:100ED0000500C2000500BD000400B9000400B50013
:100EE0000400B1000400AD000400A9000400A50046
:100EF0000300A20003009F0004009B000300980071
:100F000003009500020093000300900003008D0091
:100F100002008B00030088000200860002008400AB
:100F20000300810002007F0002007D0002007B00C0
:100F300002007900020077000100760002007400D0
:100F4000020072000100710002006F0002006D00DB
:100F500001006C0002006A000100690002006700E5
:100F600001006600010065000100640002006200EB
:100F7000010061000100600001005F0002005D00EF
:100F800001005C0001005B0001005A0001005900F3
:100F900001005800010057000100560001005500F3
:100FA00001005400010053000000530001005200F2
:100FB000010051000100500001004F0001004E00EF
:100FC00000004E0001004D0001004C0001004B00EC
:100FD00000004B0001004A000100490001004800E8
:100FE00000004800010047000100460000004600E4
:100FF00001004500000045000100440001004300DD
:1010000000004300010042000000420001004100D6
:10101000000041000100400001003F0000003F00CF
:1010200001003E0000003E0001003D0000003D00C8
:1010300001003C0000003C0000003C0001003B00BF
:1010400000003B0001003A0000003A0001003900B6
:1010500000003900010038000000380000003800AE
:1010600001003700000037000100360000003600A4
:10107000000036000100350000003500000035009A
:10108000010034000000340000003400010033008F
:101090000000330000003300010032000000320085
:1010A000000032000100310000003100000031007A
:1010B00001003000000030000000300001002F006F
:1010C00000002F0000002F0000002F0001002E0064
:1010D00000002E0000002E0001002D0000002D0059
:1010E00000002D0000002D0001002C0000002C004D
:1010F00000002C0000002C0001002B0000002B0041
:1011000000002B0000002B0001002A0000002A0034
:1011100000002A0000002A00010029000000290028
:10112000000029000000290000002900010028001B
:10113000000028000000280000002800000028000F
:101140000100270000002700000027000000270002
:1011500000002700010026000000260000002600F5
:1011600000002600000026000100250000002500E8
:1011700000002500000025000000250000002500DB
:1011800001002400000024000000240000002400CE
:1011900000002400010023000000230000002300C1
:1011A00000002300000023000000230000002300B3
:1011B00001002200000022000000220000002200A6
:1011C0000000220000002200010021000000210098
:1011D000000021000000210000002100000021008B
:1011E000000021000100200000002000000020007D
:1011F000000020000000200000002000000020006F
:101200000000200001001F0000001F0000001F0060
:1012100000001F0000001F0000001F0000001F0052
:1012200001001E0000001E0000001E0000001E0045
:1012300000004D383420582059205A20450062655E
:10124000640A002C2073797374656D2073746F7059
:1012500070656421204865617465725F49443A2075
:101260000048617264636F646564204465666175FB
:101270006C742053657474696E6773204C6F61647D
:1012800065640A00E8030000E80300000A000000AB
:101290001027000000001643000016430000A04085
:1012A0000000C84100002042000020420000C84366
:1012B0000000C04220440020490020204D3330313E
:1012C0002050005049442073657474696E67733A06
:1012D0000A0020460020420020480020204D3134E2
:1012E000352053004D6174657269616C20686561D9
:1012F00074757020706172616D65746572733A0AFD
:101300000020204D363636205A005A3220456E6471
:1013100073746F702061646A7573746D656E743A6E
:101320000A00205A0020590020204D323036205823
:1013300000486F6D65206F66667365743A0A002019
:101340004500205A00205900205800204200205417
:101350000020204D323035205300416476616E63A9
:1013600065643A20533C6D696E5F666565647261C1
:1013700074653E20543C6D696E5F74726176656C75
:101380005F66656564726174653E20423C6D696E9E
:101390005F7365676D656E745F74696D655F6D73AE
:1013A0003E20583C6D61785F78795F6A65726B3E6C
:1013B000205A3C6D61785F7A5F6A65726B3E2045AA
:1013C0003C6D61785F655F6A65726B3E0A00205410
:1013D0000020520020204D32303420500041636301
:1013E000656C65726174696F6E2028756E697473BF
:1013F0002F7332293A20503C7072696E745F6163BA
:1014000063656C3E20523C726574726163745F6107
:101410006363656C3E20543C74726176656C5F61F9
:101420006363656C3E0A00204500205A0020590085
:1014300020204D3230312058004D6178696D756D36
:1014400020416363656C65726174696F6E202875F5
:101450006E6974732F7332293A0A00204500205AAE
:101460000020590020204D3230332058004D617843
:10147000696D756D20666565647261746573202899
:10148000756E6974732F73293A0A00204500205A3B
:101490000020590020204D393220580053746570C7
:1014A000732070657220756E69743A0A0020204DB1
:1014B0003230302044300A0020204D323030204479
:1014C000002044697361626C65640A0046696C615E
:1014D0006D656E742073657474696E67733A00206D
:1014E000204D3134392043203B20556E69747320E0
:1014F000696E2043656C736975730A00202047325A
:1015000031202020203B20556E69747320696E20A5
:101510006D6D0A0020204E6F7A7A6C653A20006368
:1015200068616E6765006F66207468652066696C27
:10153000616D656E74005761697420666F72207307
:1015400074617274005052494E54205041555345B5
:10155000440020204E6F7A7A6C653A2000200066A5
:10156000696C616D656E7420756E6C6F6164005797
:1015700061697420666F72005052494E5420504188
:10158000555345440020204E6F7A7A6C653A20000E
:101590002000506C6561736520776169742E2E2E72
:1015A0000048656174696E67206E6F7A7A6C6500B9
:1015B0005052494E54205041555345440020204E2E
:1015C0006F7A7A6C653A2000200068656174206E3D
:1015D0006F7A7A6C652E0050726573732062757431
:1015E000746F6E20746F005052494E542050415514
:1015F0005345440020204E6F7A7A6C653A2000747F
:101600006F20636F6E74696E75652E2E2E00616E8D
:101610006420707265737320627574746F6E004914
:101620006E736572742066696C616D656E740050CE
:1016300052494E54205041555345440020204E6F8E
:101640007A7A6C653A2000200066696C616D656E7F
:1016500074206C6F6164005761697420666F72005A
:101660005052494E54205041555345440020204E7D
:101670006F7A7A6C653A2000200066696C616D654E
:101680006E742065787472756465005761697420A2
:10169000666F72005052494E542050415553454494
:1016A00000746F20726573756D65005761697420F1
:1016B000666F72207072696E74005052494E5420E9
:1016C00050415553454400496E697469616C697AAB
:1016D0006520454550524F4D00436F6E74726F6CDC
:1016E00000526573746F7265206661696C73616620
:1016F00065004C6F61642073657474696E67730074
:10170000496E697469616C697A6520454550524F2C
:101710004D0053746F72652073657474696E6773DE
:101720000046696C616D656E74004D6F74696F6E13
:101730000054656D7065726174757265004D616904
:101740006E004D3330332055312045256920532517
:101750006900507265686561742041425320636F6F
:101760006E66005072656865617420504C4120635C
:101770006F6E6600504944204175746F74756E65D4
:1017800000504944204175746F74756E650050496E
:10179000442D44005049442D44005049442D4900F3
:1017A0005049442D49005049442D50005049442D82
:1017B00050002008204661637400200820466163C1
:1017C00074002008204D6178002008204D617800C9
:1017D0002008204D6178002008204D696E00200807
:1017E000204D696E002008204D696E004F6666002E
:1017F0004F6E20004175746F74656D700046616EA8
:101800002073706565640046616E20737065656461
:10181000004E6F7A7A6C65004E6F7A7A6C65004381
:101820006F6E74726F6C0053746F726520736574A1
:1018300074696E6773004E6F7A7A6C65004E6F7ACA
:101840007A6C650046616E20737065656400466160
:101850006E2073706565640054656D7065726174A7
:1018600075726500436172642072656D6F766564A0
:10187000004361726420696E736572746564000070
:10188000060900FE070192032120FFFF08FF07FF62
:10189000000000060000010707060200808080802B
:1018A000800080030202060105A0A00507070600CC
:1018B000005050F850F850500507070600002078F7
:1018C000A07028F020050707060000C0C8102040BF
:1018D00098180507070600006090A040A8906802CD
:1018E0000303060104C040800307070601002040EF
:1018F00080808040200307070601008040202020D0
:10190000408005050506000120A870A820050505F2
:101910000600012020F820200203030602FFC04039
:1019200080050101060003F8020202060200C0C0A1
:101930000505050600010810204080050707060080
:10194000007088888888887003070706010040C0F7
:1019500040404040E005070706000070880870809E
:1019600080F8050707060000F81020100808F005A9
:10197000070706000010305090F810100507070602
:101980000000F880F008088870050707060000705E
:101990008080F0888870050707060000F80810208E
:1019A000202020050707060000708888708888704E
:1019B000050707060000708888780808700205058A
:1019C000060200C0C000C0C00206060602FFC0C07A
:1019D00000C040800407070600001020408040201F
:1019E00010050303060002F800F8040707060100CB
:1019F00080402010204080050707060000708808FE
:101A00001020002005070706000070880868A8A8B5
:101A100070050707060000708888F8888888050721
:101A200007060000F08888F08888F00507070600A0
:101A30000070888080808870050707060000F088A5
:101A400088888888F0050707060000F88080F08005
:101A500080F8050707060000F88080F08080800588
:101A60000707060000708880B88888700507070699
:101A70000000888888F888888801070706020080A7
:101A800080808080808005070706000038101010D5
:101A90001090600507070600008890A0C0A09088FD
:101AA000050707060000808080808080F805070712
:101AB00006000088D8A888888888050707060000DF
:101AC0008888C8A898888805070706000070888855
:101AD00088888870050707060000F08888F08080F5
:101AE0008005070706000070888888A890680507A9
:101AF00007060000F08888F0A09088050707060018
:101B000000788080700808F0050707060000F820BC
:101B10002020202020050707060000888888888864
:101B20008870050707060000888888888850200587
:101B300007070600008888888888A85005070706D8
:101B40000000888850205088880507070600008814
:101B5000888850202020050707060000F80810207C
:101B60004080F8030707060100E08080808080E065
:101B7000050505060001804020100803070706013F
:101B800000E02020202020E0050303060004205070
:101B900088050101060000F80202020602058040E5
:101BA0000505050600007008788878050707060017
:101BB000008080B0C88888F00505050600007080A8
:101BC00080887005070706000008086898888878EC
:101BD0000505050600007088F880700507070600F7
:101BE000003048E0404040400506060600FF70888F
:101BF000887808700507070600008080B0C88888CC
:101C0000880107070602008000808080808003082A
:101C1000080601FF200020202020A040040707061E
:101C20000000808090A0C0A090030707060100C0BC
:101C30004040404040E0050505060000D0A8A8A8A7
:101C4000A8050505060000B0C888888805050506B2
:101C5000000070888888700506060600FFF08888F6
:101C6000F080800506060600FF7888887808080559
:101C70000505060000B0C880808005050506000047
:101C800070807008F00407070600004040E0404004
:101C90004030050505060000888888986805050518
:101CA0000600008888885020050505060000888801
:101CB000A8A8500505050600008850205088050694
:101CC000060600FF8888887808700505050600006C
:101CD000F8102040F803070706010020404080402C
:101CE00040200107070602008080808080808003FA
:101CF00007070601008040402040408005020206A0
:101D000000026890000000060000000000060000CD
:101D100000000006000000000006000000000006B1
:101D200000000000000600000000000600000000A7
:101D30000006000000000006000000000006000091
:101D40000000000600000000000600000000000681
:101D50000000000000060000000000060000000077
:101D60000006000000000006000000000006000061
:101D70000000000600000000000600000000000651
:101D80000000000000060000000000060000000047
:101D90000006000000000006000000000006000031
:101DA0000000000600000000000600000000000621
:101DB0000000000000060000000000060000000017
:101DC0000006000000000006000000000006000001
:101DD00001070706020080008080808080050707D9
:101DE0000600002070A8A0A87020050707060000C4
:101DF000304040E04050A8050505060000887050BE
:101E00007088050707060000885020F820F8200198
:101E10000707060200808080008080800508080691
:101E20000000304820505020906003010106010757
:101E3000A0050707060000F888B8B8B888F80507B5
:101E400007060001700878887800F8050505060087
:101E5000012850A05028050303060001F8080802D5
:101E600002020602064080050707060000F888A85F
:101E70008898A8F8050101060006F8040404060085
:101E800003609090600507070600002020F82020DE
:101E900000F804050506000360902040F0030505E6
:101EA000060003E020E020E0020202060206408075
:101EB0000508080600FF8888888898E8808005075C
:101EC000070600007898987818181802020206028F
:101ED00002C0C00202020602FF40800305050600A0
:101EE0000340C04040E0050707060001708888886D
:101EF0007000F8050505060001A0502850A0050750
:101F0000070600008890A858B808080507070600CB
:101F1000008890B848982038050808060000C0409E
:101F2000C048D838080805070706000020002040F0
:101F30008088700508080600004020007088F88836
:101F4000880508080600001020007088F8888805B9
:101F500008080600002050007088F88888050808E6
:101F60000600006890007088F88888050808060058
:101F7000005000708888F88888050808060000204E
:101F800050207088F888880507070600003860A090
:101F9000B8E0A0B80508080600FF70888080887047
:101FA0002060050808060000402000F880F080F856
:101FB000050808060000081000F880F080F8050801
:101FC00008060000205000F880F080F8050707069A
:101FD00000005000F880F080F80308080601008037
:101FE0004000E0404040E0030808060100204000B7
:101FF000E0404040E003080806010040A000E04047
:102000004040E0030707060100A000E0404040E038
:10201000050707060000704848E8484870050808AA
:1020200006000068900088C8A8988805080806007F
:102030000040207088888888700508080600001015
:1020400020708888888870050808060000205000E5
:1020500070888888700508080600006890007088FD
:1020600088887005080806000050007088888888F5
:1020700070050505060001885020508805080806EF
:1020800000FF1070A8A8A8A8704005080806000066
:10209000402088888888887005080806000010207D
:1020A0008888888888700508080600002050008805
:1020B000888888700508080600005000888888888D
:1020C0008870050808060000102088502020202075
:1020D0000509090600FFC040704848704040E00410
:1020E00008080601FF609090A09090E08005080825
:1020F000060000402000700878887805080806006F
:102100000010200070087888780508080600002074
:10211000500070087888780508080600006890006C
:102120007008788878050707060000500070087866
:102130008878050808060000205020700878887804
:10214000050606060000D02878A0A8500506060659
:1021500000FF70808870206005080806000040209D
:10216000007088F8807005080806000010200070D4
:1021700088F880700508080600002050007088F874
:10218000807005070706000050007088F880700313
:10219000080806010080400040C04040E0030808F5
:1021A00006010020400040C04040E003080806014E
:1021B0000040A00040C04040E0030707060100A027
:1021C0000040C04040E0050707060000A040A01006
:1021D000788870050808060000689000B0C88888F4
:1021E000880508080600004020007088888870056F
:1021F000080806000010200070888888700508080C
:1022000006000020500070888888700508080600C5
:1022100000689000708888887005070706000050E5
:102220000070888888700505050600012000F80008
:10223000200507070600FF1070A8A8A87040050831
:10224000080600004020008888889868050808066D
:10225000000010200088888898680508080600009B
:1022600020500088888898680507070600005000FD
:1022700088888898680509090600FF10200088886A
:1022800088F808700407070601FFC04060506040EE
:10229000E00508080600FF50008888887808707CF0
:1022A0003C3E5E2B3D3F2F5B5D3B2C2A225C004574
:1022B00072726F722077726974696E6720746F2012
:1022C000454550524F4D210A00290A002062797479
:1022D00065733B20637263200053657474696E6795
:1022E000732053746F726564202800202863616C2A
:1022F00063756C6174656429210A0020213D20000A
:10230000454550524F4D20435243206D69736D61D6
:10231000746368202D202873746F7265642920000F
:10232000290A002062797465733B20637263200080
:102330002073746F7265642073657474696E67735B
:1023400020726574726965766564202800204D618D
:10235000726C696E3D563431290A00284545505249
:102360004F4D3D00454550524F4D20766572736983
:102370006F6E206D69736D617463682000000021C9
:1023800000240027002A002D003000330001010046
:1023900000040107010A0100002200250028002B8B
:1023A000002E003100340002010000050108010B7D
:1023B00001000020002300260029002C002F0032FD
:1023C00000000100000301060109010505050507DC
:1023D0000508080808020202020A0A0808040404A0
:1023E00004010101010101010103030303030303CC
:1023F00003040707070C0C0C0C0C0C0C0C0202025B
:102400000206060606060606060B0B0B0B0B0B0B4D
:102410000B010210202008081020401020408002EC
:10242000010201080402010102040810204080801A
:10243000402010080402018004020180402010089E
:102440000402010804020101020408102040800176
:102450000204081020408000000A0B02090C0D0E37
:102460000807030401000000000000000000000055
:10247000000000000000000000000000000000005C
:102480000000001211100000000000000000000019
:102490000000000000000000000000000045737410
:1024A0006570732F6D6D004573746570732F6D6D5E
:1024B000005A73746570732F6D6D005A7374657074
:1024C000732F6D6D005973746570732F6D6D0059A6
:1024D00073746570732F6D6D005873746570732F0E
:1024E0006D6D005873746570732F6D6D004D6F7452
:1024F000696F6E0053746570732F6D6D004A65725D
:102500006B00416363656C65726174696F6E005640
:10251000656C6F6369747900436F6E74726F6C00E1
:1025200046696C2E204469612E0046696C2E204459
:1025300069612E004F6666004F6E20004520696E6F
:10254000206D6D3300436F6E74726F6C0043616E6B
:102550006E6F7420656E7465722073756264697243
:102560003A2000022E2E004D61696E0020204E6F31
:102570007A7A6C653A200020004261636B004D69F5
:102580006E696D756D2054656D70206973203137EB
:10259000302E0048656174696E67206661696C65FC
:1025A000640045787472756465206D6F72650052C1
:1025B0006573756D65207072696E74005245535570
:1025C0004D45204F5054494F4E533A004261627975
:1025D00073746570205A004D36303020423000430D
:1025E00068616E67652066696C616D656E74004236
:1025F00061627973746570205A00466C6F7700468B
:102600006C6F770046616E2073706565640046618B
:102610006E207370656564004E6F7A7A6C65004E4B
:102620006F7A7A6C650053706565640053706565F8
:1026300064004D61696E004261636B004E657874A1
:1026400020636F726E6572004D34323800507265CF
:102650006865617420504C4100436F6F6C646F7704
:102660006E00507265686561742041425300436892
:10267000616E67652066696C616D656E74004469A2
:102680007361626C65207374657070657273004D60
:1026900038340053657420686F6D65206F6666730B
:1026A000657473004C6576656C20636F726E65723D
:1026B0007300486F6D65205A00473238205A004831
:1026C0006F6D65205900473238205900486F6D659D
:1026D0002058004732382058004175746F20686FC9
:1026E0006D6500473238004D6F76652061786973FB
:1026F000004D61696E0053442063617264206F6B0A
:102700000A006F70656E526F6F74206661696C6548
:10271000640A00766F6C756D652E696E697420664B
:1027200061696C65640A00534420696E69742066AF
:1027300061696C0A006175746F25692E67004D32FE
:1027400034004D32332025730057726974696E6707
:1027500020746F2066696C653A20006F70656E208A
:102760006661696C65642C2046696C653A20006F6F
:1027700070656E206661696C65642C2046696C65C5
:102780003A200046696C652073656C656374656406
:102790000A002053697A653A200046696C65206F0B
:1027A00070656E65643A20006F70656E20666169C1
:1027B0006C65642C2046696C653A20002066696C63
:1027C000653A20004E6F7720002220706F73002240
:1027D00020706172656E743A2200535542524F5513
:1027E00054494E452043414C4C20746172676574D6
:1027F0003A22004B494C4C45442E200074727969B2
:102800006E6720746F2063616C6C207375622D6736
:10281000636F64652066696C6573207769746820EE
:10282000746F6F206D616E79206C6576656C732EA8
:10283000204D4158206C6576656C2069733A0045DF
:1028400072726F723A0043616E6E6F74206F7065C2
:102850006E207375626469722000544845524D4180
:102860004C2052554E4157415900546865726D6174
:102870006C2052756E6177617900656E7175657552
:1028800065696E672022006563686F3A001FFFFF6D
:10289000FFFFFFFF600000000001FF40000000009C
:1028A00000FF8000000000007F83CF00000C303F5D
:1028B00087FF80000C301F867980000C000F8C3061
:1028C000C7838C30E78C30CFC7CC31F38C30DCEC55
:1028D000EC33B98C30D86C6C33198C30D06C0C3331
:1028E000198C30D86C0C33198C30DC6C0E3B198C85
:1028F00030CF7C079F198C30C77C038F19400000B4
:1029000000000002600000000000061FFFFFFFFF44
:10291000FFF8205A00205900580020204D61783AD5
:102920002000205A00205900580020204D696E3A9E
:1029300020004F6E20004F666600536F667420655E
:102940006E6473746F70733A200020643A002069DB
:102950003A0020703A0043290A0061626C656420E5
:10296000286D696E2074656D702000436F6C642063
:1029700065787472756465732061726520002364E4
:102980006566696E65202044454641554C545F4B51
:1029900064200023646566696E65202044454641D5
:1029A000554C545F4B69200023646566696E652051
:1029B0002044454641554C545F4B702000504944DB
:1029C000204175746F74756E652066696E697368F1
:1029D0006564212050757420746865206C6173747F
:1029E000204B702C204B6920616E64204B64206367
:1029F0006F6E7374616E74732066726F6D206265A2
:102A00006C6F7720696E746F20436F6E66696775AF
:102A1000726174696F6E2E680A00504944204175D6
:102A2000746F74756E65206661696C6564212074CD
:102A3000696D656F75740A00504944204175746F63
:102A400074756E65206661696C6564212054656DDE
:102A5000706572617475726520746F6F2068696744
:102A6000680A00204B643A2000204B693A2000207D
:102A70004B703A20000A20436C61737369632050E5
:102A80004944200A002054753A2000204B753A2012
:102A900000206D61783A2000206D696E3A20002098
:102AA000643A200020626961733A2000000000004F
:102AB0000000000000000000000048420000484202
:102AC00000008040000000005761726E696E673A36
:102AD00020486F6D696E672042756D70204469767D
:102AE00069736F72203C20310A000202040000A0CA
:102AF000400000A0400000004000004643000046A7
:102B00004300005C43FFFFFF4D36303020486F74B8
:102B1000656E6420746F6F20636F6C6420746F2027
:102B20006368616E67652066696C616D656E740AC5
:102B30000000002110422063308440A550C660E7A9
:102B400070088129914AA16BB18CC1ADD1CEE1EF62
:102B5000F13112100273325222B5529442F772D6FA
:102B600062399318837BB35AA3BDD39CC3FFF3DEB2
:102B7000E36224433420040114E664C774A444854A
:102B8000546AA54BB528850995EEE5CFF5ACC58D02
:102B9000D55336722611163006D776F6669556B49A
:102BA000465BB77AA719973887DFF7FEE79DD7BC52
:102BB000C7C448E5588668A77840086118022823EA
:102BC00038CCC9EDD98EE9AFF9488969990AA92BA2
:102BD000B9F55AD44AB77A966A711A500A333A123A
:102BE0002AFDDBDCCBBFFB9EEB799B588B3BBB1AF2
:102BF000ABA66C877CE44CC55C222C033C600C418A
:102C00001CAEED8FFDECCDCDDD2AAD0BBD688D4941
:102C10009D977EB66ED55EF44E133E322E511E70D9
:102C20000E9FFFBEEFDDDFFCCF1BBF3AAF599F7891
:102C30008F8891A981CAB1EBA10CD12DC14EF16F42
:102C4000E18010A100C230E32004502540467067A7
:102C500060B9839893FBA3DAB33DC31CD37FE35ED3
:102C6000F3B1029012F322D23235421452776256F7
:102C700072EAB5CBA5A89589856EF54FE52CD50DE3
:102C8000C5E234C324A01481046674476424540547
:102C900044DBA7FAB79987B8975FE77EF71DC73C73
:102CA000D7D326F2369106B0165766767615463497
:102CB000564CD96DC90EF92FE9C899E9898AB9AB83
:102CC000A94458654806782768C018E1088238A3E7
:102CD000287DCB5CDB3FEB1EFBF98BD89BBBAB9A13
:102CE000BB754A545A376A167AF10AD01AB32A9237
:102CF0003A2EFD0FED6CDD4DCDAABD8BADE89DC923
:102D00008D267C076C645C454CA23C832CE01CC186
:102D10000C1FEF3EFF5DCF7CDF9BAFBABFD98FF8B2
:102D20009F176E367E554E745E932EB23ED10EF0D6
:102D30001E25753A2530327500253032753A25301A
:102D400032750025756420253032753A253032758C
:102D5000005A00590058000920000000000000003F
:102D60000000000000007FFFE00000000000000005
:102D700000000000007000E0000000000000000003
:102D80000000000061F8600000000000000000008A
:102D900000000041F82000000000000000000000DA
:102DA000000040F0200000000000000000000000D3
:102DB0000040602000000000000000000000000053
:102DC0005801A07F80000000000000000000005CAF
:102DD00063A0FFC0000000000000000000005EF7DC
:102DE000A0FFC0000000000000000000005EF7A08F
:102DF000FFC0000000000000000000005C63A07F36
:102E000080000000000000000000005801A07F804A
:102E100000000000000000000000406020FFC00033
:102E200000000000000000000040F020FFC0000093
:102E3000000000000000000041F820FFC00000007A
:102E40000000000000000061F8603F00000000008A
:102E50000000000000007000E01E00000000000004
:102E600000000000007FFFE00C00000000000000F8
:102E70000000000000000000000000000000000052
:102E80000000007FFFE000000000000000000000E4
:102E900000007000E00000000000000000000000E2
:102EA00000630C6000000000000000000000000053
:102EB000470E200000000000000000000000004F4E
:102EC0000F200000000000000000000000005F0F65
:102ED000A00000000000000000000000005E07A04D
:102EE0007F8000000000000000000000406020FF24
:102EF000C00000000000000000000040F020FFC003
:102F00000000000000000000000040F020FFC000B2
:102F10000000000000000000004060207F800000F2
:102F200000000000000000005E07A07F800000009D
:102F3000000000000000005F0FA0FFC000000000C4
:102F40000000000000004F0F20FFC0000000000044
:102F50000000000000470E20FFC00000000000003D
:102F600000000000630C603F000000000000000053
:102F70000000007000E01E000000000000000000E3
:102F800000007FFFE00C00000000000000000000D7
:102F90000000000000060900FE000000000001091A
:102FA0000008FE000005080806000040F0C88888F8
:102FB000987810050808060000C0F8888888888876
:102FC000F80505050600012030F830200508080640
:102FD00000002070F820202020E00509090600FFED
:102FE0002070A8A8B8888870200509090600FFE0AD
:102FF00080C0B0A8283028280509090600FFF8A8D5
:103000008888888888A8F8050A0A0600FE2050509B
:10301000505088A8A8887003030306000340A0400E
:103020005654726176206D696E0056547261762036
:103030006D696E005654726176206D696E00566D32
:10304000696E00566D696E00566D696E00566D6151
:1030500078204500566D6178204500566D617820D6
:103060004500566D6178205A00566D6178205A00EF
:10307000566D6178205A00566D6178205900566D62
:103080006178205900566D6178205900566D61783D
:10309000205800566D6178205800566D6178205890
:1030A000004D6F74696F6E00416D6178204500417D
:1030B0006D6178204500416D6178205A00416D6155
:1030C00078205A00416D6178205900416D61782067
:1030D0005900416D6178205800416D617820580099
:1030E000412D74726176656C00412D747261766554
:1030F0006C00412D7265747261637400412D7265BC
:10310000747261637400416363656C00416363655D
:103110006C004D6F74696F6E0056652D6A65726B39
:103120000056652D6A65726B0056652D6A65726B77
:1031300000567A2D6A65726B00567A2D6A65726B3D
:103140000056792D6A65726B0056792D6A65726B2F
:103150000056792D6A65726B0056782D6A65726B20
:103160000056782D6A65726B0056782D6A65726B11
:10317000004D6F74696F6E0020746F6F206C6F6EFE
:103180006720657874727573696F6E2070726576EA
:10319000656E7465640A0020636F6C6420657874E2
:1031A000727573696F6E2070726576656E74656492
:1031B0000A0070012C0190012701B0012201C00119
:1031C0001D01F00118011002130130020E0160020E
:1031D000090190020401C002FF000003FA0040034D
:1031E000F5008003F000D003EB002004E60070043B
:1031F000E100E004DC004005D700C005D200400635
:10320000CD00D006C8008007C3003008BE00F0081B
:10321000B900C009B400B00AAF00B00BAA00D00CCE
:10322000A500000EA000500F9B00C0109600501289
:10323000910000148C00C0158700B0178200B019EF
:103240007D00D01B7800001E730040206E0090228D
:103250006900F024640040275F0090295A00E02BA9
:103260005500102E500020304B0010324600E03345
:10327000410090353C001037370070383200A039DB
:103280002D00B03A2800A03B2300603C1E00103DFA
:103290001900903D1400103E0F00703E0A00C03E21
:1032A0000500003F0000403FFBFF803FF6FFC03FAE
:1032B000F1FF48656174696E67206661696C6564D9
:1032C0000048656174696E67206661696C656400B9
:1032D0004572723A204D494E54454D50004D494E6D
:1032E00054454D5020747269676765726564004586
:1032F00072723A204D415854454D50004D4158543A
:10330000454D502074726967676572656400526547
:1033100073656E643A20006F6B00627573793A20B2
:1033200070617573656420666F7220696E70757464
:103330000A00627573793A2070617573656420665E
:103340006F7220757365720A00627573793A207026
:10335000726F63657373696E670A004B494C4C4525
:10336000442E20004B494C4C2063617573656420EA
:103370006279204B494C4C20627574746F6E2F70CB
:10338000696E0A004B494C4C45442E20004B494C79
:103390004C2063617573656420627920746F6F20BF
:1033A0006D75636820696E61637469766520746900
:1033B0006D65202D2063757272656E7420636F6D6C
:1033C0006D616E643A2000506C65617365207265B2
:1033D000736574005052494E5445522048414C5434
:1033E0004544005072696E7465722068616C746542
:1033F000642E206B696C6C28292063616C6C656499
:10340000210A004D6F76652058004D6F7665205972
:10341000004D6F7665205A00457874727564657248
:10342000004D6F766520302E316D6D004D6F7665E5
:1034300020316D6D004D6F76652031306D6D004D22
:103440006F7665206178697300457874727564657C
:1034500072004D6F7665205A004D6F7665205900D9
:103460004D6F7665205800457874727564657200FA
:103470004D6F7665205A004D6F76652059004D6F6F
:1034800076652058005072657061726500507269EF
:103490006E7420706175736564004D3132350000C3
:1034A0004D3234005072696E742061626F727465BF
:1034B00064005072696E742066726F6D2053440010
:1034C00053746F70207072696E7400526573756DFD
:1034D00065207072696E74004E6F205344206361E2
:1034E0007264005061757365207072696E74004378
:1034F0006F6E74726F6C005072657061726500540B
:10350000756E6500496E666F2073637265656E0047
:1035100030E4C6E511241FBECFEFD1E2DEBFCDBF40
:1035200000E00CBF13E0A0E0B2E0EEE9F7EE01E04E
:103530000BBF02C007900D92A43DB107D9F724E15B
:10354000A4EDB3E001C01D92AC32B207E1F71AE17D
:10355000C9E8DAE100E006C021970109802FFE01E9
:103560000E9438F3C838D10780E00807A9F70E9405
:10357000C1DD0C94BEF30C9400002F923F924F9249
:103580005F926F927F928F929F92AF92BF92CF92F3
:10359000DF92EF92FF920F931F93CF93DF93CDB7FC
:1035A000DEB7C85BD1090FB6F894DEBF0FBECDBF42
:1035B0000091280620E6029F8001112408551B4F28
:1035C0008091B70B80FF1AC0E7E8F8E284917F0191
:1035D0003FEFE31AF30A811102C0780104C00E9490
:1035E000DC3EF701F3CFD7018D917D01882319F0DF
:1035F0000E94DC3EF8CF8AE00E94DC3E81E090E051
:1036000090932312809322121092FF031092FE03D4
:103610008FE3809302041092010410920004109230
:10362000EE031092EF031092F0031092F103F801F1
:1036300080810F5F1F4F8032D1F38E34B1F48181CE
:1036400090ED980F9A3020F08D3211F08B3269F4A2
:103650003296DF0131962C9120532A30D0F3CD01E0
:10366000FC01019620812032D9F3F093AE13E09350
:10367000AD137F01BFEFEB1AFB0A10816AE270E025
:10368000C7010E9486F3009731F0FC0131978081D9
:103690008032E1F311821D3429F0143519F017340A
:1036A00009F0CEC0F70180812FEFE21AF20A8032D2
:1036B000C9F380538A3008F0C3C0109302042091EC
:1036C0000004309101044AE03196429FC001439FBB
:1036D000900D1124DF0111972C91022E000C330B59
:1036E00020533109280F391F808180538A3060F3BD
:1036F0003093010420930004DF0131968C918032D5
:10370000D9F31D3451F00091AD136091FE03709117
:10371000FF0388248394912C55C02E31310591F0FC
:103720003CF42731310571F02C31310561F70AC0C5
:103730002537310544F32737310524F0203A43E09B
:10374000340709F7B093FF03A093FE0379C0413219
:1037500009F442C0EFEBE40FEA3108F05DC0DC0190
:103760007D015D915032E1F3C701A0EDA50FAA30B4
:1037700008F046C0DC01EE2EF12C670153E0D59431
:10378000C7945A95E1F7A60142515C4F6A014E2F4A
:103790004770F40102C0EE0FFF1F4A95E2F7AF0138
:1037A000F6015081452B40831097A1F1A01BA70182
:1037B0004C525C4FFA01A083DC014C9141544A31D8
:1037C00080F5DC01CD0101964C914111C0CF709381
:1037D000FF036093FE0334C01D3409F0BBCF2032D9
:1037E000310509F0B7CF9093FF038093FE0363E2A6
:1037F00070E00E9486F3009719F1DC011C9220C052
:10380000A3EDA50FA23008F4B5CF5B3211F00C94F4
:103810006137B0CFA0E0CBCF6115710569F6BD016E
:10382000CBCFAD011196FA01908190539A30C8F335
:10383000CA014F5F5F4FFC01A081A032C9F3C1CF25
:10384000809102048D3411F40C94D529843511F43F
:103850000C940937873411F00C944337809100049D
:10386000909101048430910509F497C65CF497FFA8
:1038700002C00C945A3720911902823091050CF045
:103880000DC11CC08A35910511F40C94472954F4DC
:103890008530910509F4C8C64C9711F40C94902812
:1038A0000C945A378B35910511F40C944B298C35B7
:1038B000910511F40C9450290C945A37222311F4D9
:1038C0000C945A370E945C3E84E292E10E9471D4CB
:1038D0000E94D13E8091B70B83FD8FC0C090301203
:1038E000D0903112E0903212F090331220910E14E9
:1038F00030910F144091101450911114C701B6016A
:103900000E941AEC882309F478C08091C90B8111B8
:1039100038C060912E0270912F02072E000C880B88
:10392000990B0E9420EC9B01AC016091C50B70913A
:10393000C60B8091C70B9091C80B0E941AEC87FFB1
:1039400020C0C0920E14D0920F14E0921014F09286
:103950001114E7E8F8E284918F010F5F1F4F88236D
:1039600021F00E94DC3EF801F6CFECE0F2E0849119
:103970008F010F5F1F4F882321F00E94DC3EF8016A
:10398000F6CFC0903012D0903112E0903212F09009
:10399000331220910E1430910F1440911014509155
:1039A0001114C701B6010E9430F020E030E048E475
:1039B00053E40E9457F2181604F5C0920E14D092E8
:1039C0000F14E0921014F0921114E7E8F8E28491D9
:1039D0008F010F5F1F4F882321F00E94DC3EF8010A
:1039E000F6CFEDEEF1E084918F010F5F1F4F88233A
:1039F00021F00E94DC3EF801F6CF20912412309194
:103A00002512409126125091271260910214709154
:103A1000031480910414909105140E941AEC8111F2
:103A20001DC0209128123091291240912A125091E4
:103A30002B126091061470910714809108149091D4
:103A400009140E941AEC811109C060910002709162
:103A5000010280910202909103021AC060912C022F
:103A600070912D02072E000C880B990B0E9420EC00
:103A70002091000230910102409102025091030214
:103A80000E947FEC2AE037ED43E25CE30E947FEC8A
:103A90000E949E3B0E94943B0C945A37222311F4BF
:103AA0000C945A3711E0029709F010E00E945C3E36
:103AB00082E50E94D93D882309F45CC10E94613DE2
:103AC0006B017C0140900214509003146090041428
:103AD0007090051420910614309107144091081439
:103AE0005091091463962CAF3DAF4EAF5FAF639713
:103AF0008091241290912512A0912612B091271244
:103B000067968CAF9DAFAEAFBFAF6797209128127D
:103B10003091291240912A1250912B126F962CAF9E
:103B20003DAF4EAF5FAF6F9720E030E0A901C70116
:103B3000B6010E941AEC882309F415C5A30192016D
:103B400067966CAD7DAD8EAD9FAD67970E941AEC08
:103B5000811111C063962CAD3DAD4EAD5FAD639745
:103B60006F966CAD7DAD8EAD9FAD6F970E941AECD8
:103B7000882309F4F8C420E030E0A901C701B601A8
:103B80000E941AEC881F8827881F18130BC080E03A
:103B900090E0A0E8BFE3AB968CAF9DAFAEAFBFAFF8
:103BA000AB970AC020E030E040E85FEBAB962CAF6B
:103BB0003DAF4EAF5FAFAB97A301920167966CAD7F
:103BC0007DAD8EAD9FAD67970E9430F0A3966CAF30
:103BD0007DAF8EAF9FAFA39763962CAD3DAD4EAD3D
:103BE0005FAD63976F966CAD7DAD8EAD9FAD6F97FA
:103BF0000E9430F0A7966CAF7DAF8EAF9FAFA797B6
:103C0000A3962CAD3DAD4EAD5FADA397CA01B901F2
:103C10000E947FEC4B015C01A7962CAD3DAD4EADF3
:103C20005FADA797CA01B9010E947FEC9B01AC016F
:103C3000C501B4010E9431F00E949CF26B966CAFFA
:103C40007DAF8EAF9FAF6B9720E030E040E05FE349
:103C50000E947FEC4B015C01A7019601C701B601F0
:103C60000E947FEC6B017C01A5019401C501B401A8
:103C70000E947FEC9B01AC01C701B6010E9430F0AD
:103C80000E949CF29B01AC01AB966CAD7DAD8EADFC
:103C90009FADAB970E947FEC4B015C0167962CAD0A
:103CA0003DAD4EAD5FAD6797C301B2010E9431F0EB
:103CB00020E030E040E05FE30E947FEC6B017C019C
:103CC000A7966CAD7DAD8EAD9FADA79790586B96C6
:103CD0002CAD3DAD4EAD5FAD6B970E940DF19B01DC
:103CE000AC01C501B4010E947FEC9B01AC01C7018E
:103CF000B6010E9431F0A30192010E9430F06B01E5
:103D00007C016F962CAD3DAD4EAD5FAD6F97639668
:103D10006CAD7DAD8EAD9FAD63970E9431F020E01C
:103D200030E040E05FE30E947FEC2B013C016B96AA
:103D30002CAD3DAD4EAD5FAD6B97A3966CAD7DAD3B
:103D40008EAD9FADA3970E940DF19B01AC01C50103
:103D5000B4010E947FEC9B01AC01C301B2010E943F
:103D600031F063962CAD3DAD4EAD5FAD63970E94D3
:103D700030F014C089E40E94D93D882329F00E94C4
:103D8000613D6B017C0103C0C12CD12C76018AE41A
:103D90000E94D93D8823F9F00E94613D6F966CAF77
:103DA0007DAF8EAF9FAF6F9720E030E0A901C701D4
:103DB000B6010E941AEC81111EC020E030E0A9017A
:103DC0006F966CAD7DAD8EAD9FAD6F970E941AEC76
:103DD000811111C0C8C320E030E0A901C701B601BC
:103DE0000E941AEC882309F4BEC36F961CAE1DAE68
:103DF0001EAE1FAE6F97D701C601B05863968CAF49
:103E00009DAFAEAFBFAF63976F962CAD3DAD4EADDE
:103E10005FAD6F97505867962CAF3DAF4EAF5FAF19
:103E200067979C01AD01BC01CD010E947FEC4B0165
:103E30005C0167962CAD3DAD4EAD5FAD6797CA0195
:103E4000B9010E947FEC9B01AC01C501B4010E9445
:103E500031F00E949CF2C158DF4F688379838A83D6
:103E60009B83CF57D0408091021490910314A0916E
:103E70000414B09105146B968CAF9DAFAEAFBFAF7D
:103E80006B97A7019601BC01CD010E9431F0AB9662
:103E90006CAF7DAF8EAF9FAFAB97A0900614B09084
:103EA0000714C0900814D0900914A396ACAEBDAE10
:103EB000CEAEDFAEA3976F962CAD3DAD4EAD5FADF0
:103EC0006F97C601B5010E9431F0AF966CAF7DAF20
:103ED0008EAF9FAFAF97C0902412D0902512E09084
:103EE0002612F0902712E396CCAEDDAEEEAEFFAE1A
:103EF000E397AB962CAD3DAD4EAD5FADAB97C70133
:103F0000B6010E9430F06B017C01209128123091A3
:103F1000291240912A1250912B12E7962CAF3DAFF7
:103F20004EAF5FAFE797AF962CAD3DAD4EAD5FADF9
:103F3000AF97E7966CAD7DAD8EAD9FADE7970E94D4
:103F400030F04B015C0180910A1490910B14A09108
:103F50000C14B0910D14EB968CAF9DAFAEAFBFAF0C
:103F6000EB979C01AD0160912C1270912D12809104
:103F70002E1290912F120E9430F0A7966CAF7DAF59
:103F80008EAF9FAFA79720913012309131124091A0
:103F9000321250913312CD57DF4F288339834A8331
:103FA0005B83C358D04080910E1490910F14A09160
:103FB0001014B0911114EF968CAF9DAFAEAFBFAFA0
:103FC000EF97A701960163966CAD7DAD8EAD9FAD69
:103FD00063970E947FEC2B013C01A5019401679639
:103FE0006CAD7DAD8EAD9FAD67970E947FEC9B0160
:103FF000AC01C301B2010E9431F02B013C01A501CB
:10400000940163966CAD7DAD8EAD9FAD63970E94BC
:104010007FEC4B015C01A701960167966CAD7DAD0D
:104020008EAD9FAD67970E947FEC9B01AC01C501EF
:10403000B4010E9430F0A30192010E94A4F06B0130
:104040007C0120E030E0A9010E941AEC87FF0AC041
:104050002BED3FE049EC50E4C701B6010E9431F07E
:104060006B017C01112351F02BED3FE049EC50E452
:10407000C701B6010E9430F06B017C0120E030E006
:10408000A901C701B6010E941AEC811128C0E3966C
:104090002CAD3DAD4EAD5FADE3976B966CAD7DAD98
:1040A0008EAD9FAD6B970E941AEC811118C0E796F8
:1040B0002CAD3DAD4EAD5FADE797A3966CAD7DAD3C
:1040C0008EAD9FADA3970E941AEC811108C04BEDF5
:1040D000C42E4FE0D42E49ECE42E40E4F42EC15817
:1040E000DF4F288139814A815B81CF57D040C7019A
:1040F000B6010E947FEC9B01AC010E947FEC4B015A
:104100005C01A7962CAD3DAD4EAD5FADA797CA0142
:10411000B9010E947FEC9B01AC01C501B4010E9472
:1041200031F00E949CF24B015C012FE632E143E842
:104130005AE30E941AEC87FD12C2C501B4010E9425
:10414000A6F10E947AF1A1967FAF6EAFA197672B7F
:1041500031F421E030E0A1963FAF2EAFA197A196B8
:10416000AEACBFACA197B50180E090E00E941EEC20
:104170004B015C019B01AC01C701B6010E940DF12E
:104180006B966CAF7DAF8EAF9FAF6B97A50194011F
:10419000A7966CAD7DAD8EAD9FADA7970E940DF13A
:1041A000C158DF4F688379838A839B83CF57D04080
:1041B000EF962CAD3DAD4EAD5FADEF97CD57DF4FD8
:1041C000688179818A819B81C358D0400E9430F0F8
:1041D000A50194010E940DF1CD57DF4F68837983CB
:1041E0008A839B83C358D0406B962CAD3DAD4EADBA
:1041F0005FAD6B97CA01B9010E947FEC20E030E00F
:1042000040E05FE30E947FEC9B01AC0160E070E066
:1042100080E89FE30E9430F0A7966CAF7DAF8EAF31
:104220009FAFA797EB96CCACDDACEEACFFACEB97B9
:10423000C986DA86EB86FC86EF96ACACBDACCEAC1C
:10424000DFACEF97AD86BE86CF86D88A60912C0210
:1042500070912D02072E000C880B990B0E9420EC08
:10426000209100023091010240910202509103021C
:104270000E947FEC2AE037ED43E25CE30E947FEC92
:10428000E3966CAF7DAF8EAF9FAFE3970E944585FD
:104290009B01AC0128533F4F4F4F5F4FE7962CAF28
:1042A0003DAF4EAF5FAFE79760964FAC60976196BA
:1042B0005FAC619762966FAC629763967FAC6397D1
:1042C00022242394312C39E1D32EA196AEACBFAC7D
:1042D000A1972A143B0409F42EC10E941AD00E940F
:1042E0004585DC01CB01E7962CAD3DAD4EAD5FAD14
:1042F000E797821B930BA40BB50BB7FD11C00E946F
:1043000045859B01AC0128533F4F4F4F5F4FE796C8
:104310002CAF3DAF4EAF5FAFE79780E00E94C6D1B4
:10432000DA94DD2009F44BC0A7962CAD3DAD4EAD1F
:104330005FADA79767966CAD7DAD8EAD9FAD67976E
:104340000E947FEC4B015C016B962CAD3DAD4EADF8
:104350005FAD6B97B201C3010E947FECA501940190
:104360000E9431F07B018C01A7962CAD3DAD4EAD86
:104370005FADA797B201C3010E947FEC4B015C01C6
:104380006B962CAD3DAD4EAD5FAD6B9767966CAD4A
:104390007DAD8EAD9FAD67970E947FEC9B01AC0118
:1043A000C501B4010E9430F02B013C01C701D801C6
:1043B00067968CAF9DAFAEAFBFAF67975BC0B101E3
:1043C00080E090E00E941EEC6B962CAD3DAD4EADB2
:1043D0005FAD6B970E947FEC4B015C010E940AF17C
:1043E0006B017C01C501B4010E9492F24B015C019A
:1043F000A701960163966CAD7DAD8EAD9FAD6397C1
:104400000E947FEC2B013C01A50194016F966CADDD
:104410007DAD8EAD9FAD6F970E947FEC9B01AC018F
:10442000C301B2010E9431F02B013C01A5019401AE
:1044300063966CAD7DAD8EAD9FAD63970E947FECB2
:104440004B015C01A70196016F966CAD7DAD8EAD01
:104450009FAD6F970E947FEC9B01AC01C501B40139
:104460000E9430F067966CAF7DAF8EAF9FAF6797BD
:1044700099E1D92E9201A301AB966CAD7DAD8EADC5
:104480009FADAB970E9431F069837A838B839C83C5
:1044900067962CAD3DAD4EAD5FAD6797AF966CADF9
:1044A0007DAD8EAD9FADAF970E9431F06D837E8361
:1044B0008F839887C158DF4F288139814A815B817A
:1044C000CF57D04069857A858B859C850E9431F0D5
:1044D00069877A878B879C87CD57DF4F2881398101
:1044E0004A815B81C358D0406D857E858F859889D0
:1044F0000E9431F06D877E878F87988BCE01019661
:104500000E9471D4C090B80BE396ECACFDAC0EAD3C
:104510001FADE3979E01235F3F4FAE01475F5F4FA3
:10452000BE016B5F7F4FCE0101960E94DBBE3FEF65
:10453000231A330ACACEC090B80BE396ECACFDAC9C
:104540000EAD1FADE39720E332E14CE252E168E2A9
:1045500072E184E292E10E94DBBE0E94943B0E94E1
:10456000D13E0C945A37EFE3F8E284918F010F5F4C
:104570001F4F882321F00E94DC3EF801F6CFE7E2CE
:10458000F2E084918F010F5F1F4F882311F40C9488
:104590005A370E94DC3EF801F4CF80E50E94D93DF5
:1045A000882329F00E94213D6B017C0103C0C12CAE
:1045B000D12C760183E50E94D93D882361F00E94C9
:1045C000613D20E030E04AE754E40E947FEC0E9425
:1045D0007AF16B017C010E948F4480915C02811111
:1045E00005C060E08DE392E00E94916C0E94D13E94
:1045F0008091AF139091B013A091B113B091B21309
:10460000C80ED91EEA1EFB1E0E944585DC01CB01A7
:104610008C199D09AE09BF09B7FD02C00C945A3729
:1046200080E00E94C6D1F0CF80911902882311F456
:104630000C945A370E945C3E89E40E94D93D88233D
:1046400029F00E94613D2B013C0103C0412C512CFB
:1046500032018AE40E94D93D882329F00E94613DFD
:104660004B015C0103C0812C912C540180E50E9418
:10467000D93D882329F00E94613D6B017C0103C074
:10468000C12CD12C760181E50E94D93D882349F0C7
:104690000E94613D63966CAF7DAF8EAF9FAF639715
:1046A00006C063961CAE1DAE1EAE1FAE6397209172
:1046B000B80BC055DF4F2883C05BD04060912C02FF
:1046C00070912D02072E000C880B990B0E9420EC94
:1046D00020910002309101024091020250910302A8
:1046E0000E947FEC2AE037ED43E25CE30E947FEC1E
:1046F000CF54DF4F688379838A839B83C15BD0402B
:104700008091021490910314A0910414B0910514A7
:1047100067968CAF9DAFAEAFBFAF6797A301920115
:10472000BC01CD010E9431F0C158DF4F688379830D
:104730008A839B83CF57D040409006145090071433
:104740006090081470900914A5019401C301B2018E
:104750000E9431F0CD57DF4F688379838A839B8332
:10476000C358D04020912412309125124091261236
:1047700050912712C701B6010E9431F0C557DF4F93
:10478000688379838A839B83CB58D04020912812F9
:104790003091291240912A1250912B1263966CADE0
:1047A0007DAD8EAD9FAD63970E9431F0C157DF4F55
:1047B000688379838A839B83CF58D0406796ACAC5B
:1047C000BDACCEACDFAC6797A982BA82CB82DC826B
:1047D0004D825E826F8278860E9445859B01AC0186
:1047E00028533F4F4F4F5F4FC555DF4F28833983C5
:1047F0004A835B83CB5AD0408DEC882E8CEC982E6C
:10480000A92C8DE3B82E60961FAE609764961FAEFC
:1048100064976C961FAE6C9768961FAE68970E945F
:104820001AD00E9445858B019C01C555DF4FC88079
:10483000D980EA80FB80CB5AD0400C191D092E0983
:104840003F0937FD11C09B01AC0128533F4F4F4F2B
:104850005F4FC555DF4F288339834A835B83CB5A2B
:10486000D04080E00E94C6D1A50194016096BFAD02
:1048700060976496AFAD64976C96FFAD6C97689641
:10488000EFAD68976B2F7A2F8F2F9E2F0E9431F0FC
:104890002B011C0120E030E040E85FE30E9457F26A
:1048A000181634F4412C512C10E8212E0FE3302E31
:1048B0008091241290912512A0912612B091271276
:1048C000CD56DF4F88839983AA83BB83C359D040D9
:1048D000A0900214B0900314C0900414D09005145A
:1048E000C956DF4FA882B982CA82DB82C759D0403D
:1048F0003F922F925F924F92CD56DF4FA880B980A2
:10490000CA80DB80C359D040C557DF4FE880F980AB
:104910000A811B81CB58D040C158DF4F2881398193
:104920004A815B81CF57D040C956DF4F688179817A
:104930008A819B81C759D0400E94D64B0F900F901F
:104940000F900F90A0966FAFA097A4967FAFA497FB
:10495000A8968FAFA897AC969FAFAC97C09028123F
:10496000D0902912E0902A12F0902B12C556DF4FFA
:10497000C882D982EA82FB82CB59D04020910614AA
:10498000309107144091081450910914C156DF4F1B
:10499000288339834A835B83CF59D0403F922F923B
:1049A0005F924F92C556DF4FA880B980CA80DB80E6
:1049B000CB59D040C157DF4FE880F9800A811B8175
:1049C000CF58D040CD57DF4F288139814A815B8154
:1049D000C358D040C156DF4F688179818A819B815D
:1049E000CF59D0400E94D64B0F900F900F900F9050
:1049F000E0966FAFE097E4967FAFE497E8968FAFCD
:104A0000E897EC969FAFEC9789819A81AB81BC8146
:104A1000CD55DF4F88839983AA83BB83C35AD04087
:104A2000AD80BE80CF80D884C955DF4FA882B982BF
:104A3000CA82DB82C75AD040C957DF4F1882C75895
:104A4000D04060967FAD609764966FAD64976C962A
:104A50009FAD6C9768968FAD6897272F362F492F9B
:104A6000582F642D752D822D932D0E9430F02FE646
:104A700032E143E05BE30E941AEC87FF08C0C957AC
:104A8000DF4FB880C758D040B11079C257C2242D2B
:104A9000352D422D532D6096BFAD60976496AFAD16
:104AA00064976C96FFAD6C976896EFAD68976B2F27
:104AB0007A2F8F2F9E2F0E9431F020E030E040E0CF
:104AC0005FE30E947FEC3B014C019F928F937F92AA
:104AD0006F93CD56DF4FA880B980CA80DB80C35961
:104AE000D040C557DF4FE880F9800A811B81CB5841
:104AF000D040C158DF4F288139814A815B81CF572F
:104B0000D040C956DF4F688179818A819B81C7591E
:104B1000D0400E94D64B0F900F900F900F90C85727
:104B2000DF4F6883C858D040C757DF4F7883C958D4
:104B3000D040C657DF4F8883CA58D040C155DF4F99
:104B40009883CF5AD0409F928F927F926F92C55692
:104B5000DF4FA880B980CA80DB80CB59D040C157D5
:104B6000DF4FE880F9800A811B81CF58D040CD57B4
:104B7000DF4F288139814A815B81C358D040C156BB
:104B8000DF4F688179818A819B81CF59D0400E9413
:104B9000D64B0F900F900F900F905B018C01A09659
:104BA0002FADA097A4963FADA497A8964FADA89718
:104BB000AC965FADAC97CD55DF4F688179818A8126
:104BC0009B81C35AD0400E9431F020E030E040E0A9
:104BD0005FE30E947FEC9B01AC01C857DF4F688107
:104BE000C858D040C757DF4F7881C958D040C65702
:104BF000DF4F8881CA58D040C155DF4F9881CF5AC6
:104C0000D0400E9430F06B017C01E894F7F8E09608
:104C10002FADE097E4963FADE497E8964FADE89767
:104C2000EC965FADEC97C955DF4F688179818A8139
:104C30009B81C75AD0400E9431F020E030E040E034
:104C40005FE30E947FEC9B01AC01B501C8010E94AB
:104C500030F09B01AC015F77C701B6010E9431F0D3
:104C60002DEC3CEC4CEC5DE30E941AEC18160CF0B9
:104C700006CFE096AFAEE097E496BFAEE497E89635
:104C80000FAFE897EC961FAFEC97C857DF4FC8807F
:104C9000C858D040A096CFAEA097C757DF4FD88056
:104CA000C958D040A496DFAEA497C657DF4FE8801E
:104CB000CA58D040A896EFAEA897C155DF4FF880EC
:104CC000CF5AD040AC96FFAEAC972301140121E03F
:104CD000C957DF4F2883C758D040B3CEA7019601EC
:104CE000C701B6010E9431F09B01AC016096BFADD7
:104CF00060976496AFAD64976C96FFAD6C976896BD
:104D0000EFAD68976B2F7A2F8F2F9E2F0E9431F077
:104D1000962E872E782E692E20E030E040E85FE363
:104D2000D401F3016B2F7A2F8F2F9E2F0E9457F201
:104D300087FF25C16F927F928F929F92CD56DF4F52
:104D4000A880B980CA80DB80C359D040C557DF4FE7
:104D5000E880F9800A811B81CB58D040C158DF4FD1
:104D6000288139814A815B81CF57D040C956DF4FB6
:104D7000688179818A819B81C759D0400E94D64B36
:104D80000F900F900F900F90C957DF4F6883C7584F
:104D9000D040C857DF4F7883C858D040C757DF4F3F
:104DA0008883C958D040C657DF4F9883CA58D0402F
:104DB0006F927F928F929F92C556DF4FA880B980E5
:104DC000CA80DB80CB59D040C157DF4FE880F980E3
:104DD0000A811B81CF58D040CD57DF4F28813981C0
:104DE0004A815B81C358D040C156DF4F68817981C9
:104DF0008A819B81CF59D0400E94D64B0F900F9053
:104E00000F900F905B018C01C957DF4F2881C75865
:104E1000D040C857DF4F3881C858D040C757DF4F00
:104E20004881C958D040C657DF4F5881CA58D04032
:104E3000CD55DF4F688179818A819B81C35AD040EB
:104E40000E9431F020E030E040E05FE30E947FEC20
:104E50009B01AC01A0966FADA097A4967FADA497DF
:104E6000A8968FADA897AC969FADAC970E9430F0F6
:104E70006B017C01E894F7F89501A801C955DF4F53
:104E8000688179818A819B81C75AD0400E9431F024
:104E900020E030E040E05FE30E947FEC9B01AC014A
:104EA000E0966FADE097E4967FADE497E8968FAD1E
:104EB000E897EC969FADEC970E9430F09B01AC0117
:104EC0005F77C701B6010E9431F02DEC3CEC4CEC51
:104ED0005DE30E9457F218160CF451C0E096AFAE95
:104EE000E097E496BFAEE497E8960FAFE897EC96AC
:104EF0001FAFEC97C957DF4F3881C758D040A096F5
:104F00003FAFA097C857DF4F4881C858D040A496FC
:104F10004FAFA497C757DF4F5881C958D040A896C4
:104F20005FAFA897C657DF4F8881CA58D040AC966C
:104F30008FAFAC97492C582C272C362C60967FAD20
:104F4000609764966FAD64976C969FAD6C9768960A
:104F50008FAD6897272F362F492F582F642D752D29
:104F6000822D932D0E9430F06B017C012DEC3CECE6
:104F70004CEC5DE30E9457F218160CF0AFCE609631
:104F80007FAD609764966FAD64976C969FAD6C979C
:104F900068968FAD6897272F362F492F582F642D8D
:104FA000752D822D932D0E9430F04B015C01A0964F
:104FB0008FADA097A4969FADA497A896AFADA897E4
:104FC000AC96BFADAC9789839A83AB83BC83E096E4
:104FD0008FADE097E4969FADE497E896AFADE89784
:104FE000EC96BFADEC978D839E83AF83B887242D5D
:104FF000352D422D532D60E070E080E89FE30E9444
:1050000030F06B017C0120910A1430910B14409117
:105010000C1450910D140E947FEC63966CAF7DAF21
:105020008EAF9FAF639720912C1230912D1240913B
:105030002E1250912F12642D752D822D932D0E94CA
:105040007FEC9B01AC0163966CAD7DAD8EAD9FADE9
:1050500063970E9431F069877A878B879C872091BC
:105060000E1430910F144091101450911114C70177
:10507000B6010E947FEC6B017C01209130123091CF
:1050800031124091321250913312642D752D822DC0
:10509000932D0E947FEC9B01AC01C701B6010E94D9
:1050A00031F06D877E878F87988BCE0101960E94A5
:1050B00071D4C055DF4FC880C05BD040CF54DF4FA4
:1050C000E880F9800A811B81C15BD0409E01235F8B
:1050D0003F4FAE01475F5F4FBE016B5F7F4FCE0119
:1050E00001960E94DBBE20E030E040E85FE3642DE3
:1050F000752D822D932D0E941AEC87FF0DC06096AE
:105100004FAE609764965FAE64976C962FAE6C97C7
:1051100068963FAE689783CB0E94943B0C945A37B5
:105120000E948F448091000290910102A09102029E
:10513000B09103028093FA039093FB03A093FC03C6
:10514000B093FD0380912C0290912D029093F9036E
:105150008093F80384E690E090932D0280932C02D4
:105160000E94D13E81E08093770488E50E94943DBF
:10517000E82E89E50E94943D082F8AE50E94943D1F
:10518000F82EE11005C0011105C011E0182705C077
:10519000011102C010E001C0182F0E948A3B1111BA
:1051A00005C0E11003C0002309F444C020E030E052
:1051B00040EA50E46091C10B7091C20B8091C30B27
:1051C0009091C40B0E9431F060932C1270932D12B9
:1051D00080932E1290932F1220910A1430910B1469
:1051E00040910C1450910D140E9457F218167CF443
:1051F00019821A821B821C829E012F5F3F4F4CE254
:1052000052E166E074E182E094E10E94A93A111152
:1052100005C0E11003C0011107C00CC080E090E0A0
:105220000E94B9B21123B9F381E090E00E94B9B2B3
:10523000111102C0FF2021F082E090E00E94B9B27B
:105240000E94843C8091360B809377048091FA030E
:105250009091FB03A091FC03B091FD0380930002A9
:1052600090930102A0930202B09303028091F8038D
:105270009091F90390932D0280932C020E94D13ECD
:1052800083E080935B020E94E6420C945A371092AE
:10529000F7030C945A3781E08093F7030C945A3744
:1052A00085E40E94D93DB82E811102C00E948F442E
:1052B000F0EA8F2EF2E09F2EA2E0CA2EA4E1DA2EB1
:1052C000B6E1EB2EB2E1FB2E00E010E0A12CD40100
:1052D0008D914D010E94D93D882309F44EC0F601FD
:1052E0002081318142815381CB54DF4F2883C55BBC
:1052F000D040CA54DF4F3883C65BD040C954DF4F1B
:105300004883C75BD040C854DF4F5883C85BD04048
:105310000E94613DD6016D937D938D939C9313976D
:10532000CB54DF4F2881C55BD040CA54DF4F388152
:10533000C65BD040C954DF4F4881C75BD040C854DA
:10534000DF4F5881C85BD04003301105B1F00E9497
:1053500030F09B01AC01F701608171818281938102
:105360000E9431F0D7016D937D938D939C93139799
:10537000C8010E94B73BAA24A3940F5F1F4FB4E05B
:10538000CB0ED11CE4E0EE0EF11C0430110509F047
:105390009ECFAA2019F00E94843C03C0B1100E9445
:1053A00062DA0E94E6420C945A3780910004909190
:1053B00001048237910509F468C70CF0E4C08B340E
:1053C000910509F449C50CF070C08831910509F4C4
:1053D0009EC20CF03EC08231910509F4D1C6FCF4A6
:1053E00097FF02C00C945A37823091050CF4ABC180
:1053F000419711F00C945A3760E087E792E00E94E1
:10540000916C5F988A989FB7F894809108018E7F7D
:10541000809308019FBF479812980C945A378531A2
:10542000910509F45DC23CF4449711F00C945A378D
:10543000EFE8F2E012C28631910509F455C24797B0
:1054400011F00C945A378091FE039091FF03FC01F8
:1054500055C28C31910509F4C3C2A4F48A31910577
:1054600009F474C20CF080C21092770E0E94A0DA88
:1054700080EA92E09093E10D8093E00D0E942B3C36
:105480000C945A378F31910509F401C42CF44E97CE
:1054900009F4B0C20C945A378032910509F4ADC3B7
:1054A0008A9709F49AC40C945A378836910509F4FE
:1054B000DFC40CF040C08235910509F45AC614F5DA
:1054C0008D34910509F4D0C40CF4CAC4813591051A
:1054D00011F00C945A370E94E5CF0E948F440E942D
:1054E0003DD110925A0B1092590B68EE73E080E098
:1054F00090E00E94A66B60E08BEE93E00E94916CBE
:105500000C945A378435910509F43AC60CF434C624
:105510008535910509F437C68C35910511F00C9449
:105520005A3720EAC22E22E0D22E32E1E32E34E1B5
:10553000F32E10E02BC68D36910509F4F9C59CF4C5
:105540008A36910509F40CC60CF4ACC58B3691056E
:1055500009F409C68C36910511F00C945A37109253
:105560009F020C945A378F36910509F4E8C40CF465
:10557000D5C48037910509F452C58137910509F4E6
:1055800055C50C945A378C3D910511F40C94C634D2
:105590000CF054C08139910509F4D9C71CF587373F
:1055A000910509F445C774F48537910509F401C7DD
:1055B0000CF007C78337910511F00C945A37E3EDCF
:1055C000F4E068C68937910509F4BCC70CF4B4C788
:1055D0008D37910509F4CAC58C38910509F44FC57A
:1055E0000C945A378B3C910511F40C946F3384F46E
:1055F000883C910511F40C940533893C910511F414
:105600000C944D338B39910511F00C945A3767C5C2
:105610008D3C910511F40C94F73314F40C948D33F4
:105620008E3C910511F40C946234833D910511F088
:105630000C945A370E943FAC0C945A378A39F1E0E7
:105640009F0709F4F0C49CF58D3231E0930711F403
:105650000C94F534A4F4823E910511F40C94C934F1
:105660008C3251E0950711F40C94CC348D3D9105AA
:1056700011F00C945A370E9418AC0C945A378F32A0
:10568000A1E09A0711F40C94FB3414F40C94F83450
:105690008336E1E09E0711F40C94E23680399140A4
:1056A00011F00C945A370E948F440C945A37873F5C
:1056B00021E0920711F40C94E4355CF5843F41E05D
:1056C000940711F40C94DE35ACF48C3A914011F04F
:1056D0000C945A379BE7C92E94E0D92E22E0E22E93
:1056E00024E1F22E3AEC232E3BE0332E00E010E0D2
:1056F0000C94FE34853FB1E09B0711F40C94E13526
:10570000863F914011F00C945A370E9413550C9427
:105710005A378A39F2E09F0711F40C94A7343CF40D
:105720008835924011F40C94F0350C945A37803A35
:1057300043E0940709F49EC2873E934011F40C9411
:10574000F9360C945A37A090FE03B090FF0380E521
:105750000E94D93D882359F00E94213D6B017C01B4
:1057600011E0672B682B692B31F410E004C010E0C6
:10577000C12CD12C760183E50E94D93D8823F1F01C
:105780000E94613D20E030E04AE754E40E947FEC53
:105790000E947AF16B017C01111112C0672B682BFA
:1057A000692B71F4A114B10459F0D5018C918823AF
:1057B00039F061E0C5010E94B16C07C0112391F37B
:1057C00060E084E692E00E94916C83E090E0909328
:1057D00023128093221281E08093810B0E948F44D8
:1057E0000E94D13EC114D104E104F104F1F0809192
:1057F000AF139091B013A091B113B091B213C80E32
:10580000D91EEA1EFB1E0E944585DC01CB018C19C6
:105810009D09AE09BF09B7FF1CC08091810B882389
:10582000C1F080E00E94C6D1EECF8091810B882329
:1058300021F080E00E94C6D1F8CF8091770E60E021
:10584000882319F085E592E002C086E492E00E9488
:10585000916C1092810B0C945A3784918F010F5FD9
:105860001F4F882321F00E94DC3EF801F6CF1092F2
:10587000FD101092FC1040E050E0BA0188EA9EE072
:105880000E941C728BE1E8EAFEE0DE0115960190B1
:105890000D928A95E1F78091A60E9091A70E9C83B8
:1058A0008B838CEE92E09A83898340E050E0BE01C6
:1058B0006F5F7F4F8BE693E00E943EA1CE01019681
:1058C0000E94E6B3E0E8F2E084918F010F5F1F4F82
:1058D000882311F40C945A370E94DC3EF801F4CF6F
:1058E0000E945D9C0C945A371092770E1092780E9D
:1058F0000C945A37203209F41082319620812111FC
:10590000F9CF40E061E00E943D990C945A3719822A
:105910001A821B821C8218A219A21AA21BA28091B1
:105920003412882341F040E0BE016F5F7F4FCE010B
:1059300080960E9483B18091780E882319F081E0CF
:105940008093770E0E9422DA0C945A378091780E59
:10595000882311F40C945A3783E50E94D93D8111B4
:105960000C946B370C945A378091780E882351F140
:10597000E5EAF2E084918F010F5F1F4F882321F049
:105980000E94DC3EF801F6CF6091F3107091F410A4
:105990008091F5109091F6104AE00E94E33E8FE26C
:1059A0000E94DC3E6091EF107091F0108091F11038
:1059B0009091F2104AE00E94E33E8AE00E94DC3EB1
:1059C0000C945A37E7EBF2E084918F010F5F1F4F81
:1059D000882311F40C945A370E94DC3EF801F4CF6E
:1059E00040E060E08091FE039091FF030E943D99AA
:1059F0000C945A378091780E882311F40C945A37FE
:105A000082E490E10E94EA7182E490E10E9433789E
:105A10001092760E1092750EE090FE03F090FF0348
:105A20008091780E882311F40C945A370E94A09E1E
:105A3000FE0131966F01CF010E94F06F84EA9EE073
:105A40009093C40E8093C30ED7018C918F3209F0CE
:105A500060C06FE270E0C7010E9486F38C010F5FA7
:105A60001F4F09F45CC06FE270E0C8010E9486F32A
:105A70005C01009709F454C00817190708F050C0DA
:105A80004C01801A910AA401B801CE0180960E94AF
:105A9000AFF3E0E2F0E0EC0FFD1FE80DF91D10821E
:105AA0008E01005E1F4FF80181918F01882319F04C
:105AB0000E94DC3EF8CF8AE00E94DC3E6091C30E7B
:105AC0007091C40E6115710511F06C5F7F4F21E07C
:105AD000AE01405E5F4FCE0105960E943B7881117A
:105AE00012C0BE01605E7F4F8EEE92E00E94AE4B10
:105AF0008EE20E94DC3E8AE00E94DC3EC6010E94EB
:105B0000E6B30C945A37D092C40EC092C30E8501EE
:105B1000A6CF85EC9EE09093C40E8093C30E8701C0
:105B20006091C30E7091C40E6115710511F06C5F28
:105B30007F4F18A21BA222E0A801CE0180960E94EE
:105B40003B78811102C0F12C14C0CE0180960E94D6
:105B50000E9E8823C1F361E0CE0180960E9458AD6D
:105B6000009789F325EEDC012C931BA20E94FA6FAB
:105B7000F82ECE0180960E94CB3EFF2009F1E8EC82
:105B8000F2E084917F01BFEFEB1AFB0A882321F03A
:105B90000E94DC3EF701F5CFF80181918F01882347
:105BA00019F00E94DC3EF8CF8AE00E94DC3E1092A1
:105BB000F3101092F4101092F5101092F61018C015
:105BC000E6EDF2E084917F012FEFE21AF20A8823DA
:105BD00021F00E94DC3EF701F5CFD8018D918D01B7
:105BE000882319F00E94DC3EF8CF8EE20E94DC3E52
:105BF000C6010E94E6B30C945A378091770E81114A
:105C00000E948F44E090FE03F090FF0380E50E9425
:105C1000943D182F882319F00E94523D182F80912F
:105C2000780E882311F40C945A37412F61E0C70194
:105C30000E943D9983E50E94D93D882381F00E940E
:105C4000313DAB01BC014093F3105093F4106093CD
:105C5000F5107093F61082E490E10E941C7280911E
:105C6000780E882319F081E08093770E11110C943F
:105C70005A3768CE8091FE039091FF0321E0209374
:105C8000760E40E060E00E943D990C945A370E94E5
:105C900008A1ECE3CE2ED12CE12CF12CA70196012A
:105CA0000E94F5EF762E672ECA01B901A701960171
:105CB0000E94F5EF6B017C01CA01B90128E130E0D7
:105CC00040E050E00E94F5EF4B015C01C9016DE638
:105CD00071E00E94F5F28E010F5F1F4F6115710593
:105CE00099F06F927F92DF92CF929F928F929F93C3
:105CF0008F937F936F938AE293E09F938F931F9389
:105D00000F930E94B3EB12C00097B1F06F927F9295
:105D1000DF92CF929F928F929F938F938AE193E02D
:105D20009F938F931F930F930E94B3EB0FB6F8943A
:105D3000DEBF0FBECDBF36C081149104A104B104F3
:105D400079F06F927F92DF92CF929F928F928EE046
:105D500093E09F938F931F930F930E94B3EBE6CF33
:105D6000C114D104E104F10469F06F927F92DF92D3
:105D7000CF9286E093E09F938F931F930F930E949F
:105D8000B3EBD4CF6F927F9282E093E09F938F9397
:105D90001F930F930E94B3EB0F900F900F900F90F3
:105DA0000F900F9060E0C8010E94B16CE7E8F8E244
:105DB00084917F019FEFE91AF90A882321F00E945C
:105DC000DC3EF701F5CFB8018EE393E00E94AE4BC5
:105DD0008AE00E94DC3E0C945A3783E50E94D93D4C
:105DE000882311F40C945A370E94413DE82E80E537
:105DF0000E94D93D882339F00E94313D8B0177FF05
:105E000004C00C945A370DE010E0902FEBE4F3E05F
:105E10008BE28E0F2491921729F031968E13FACFD0
:105E20000C947B37EFE3F8E284918F010F5F1F4FF3
:105E3000882321F00E94DC3EF801F6CFE6E7F3E08C
:105E400084918F010F5F1F4F882311F40C945A37F0
:105E50000E94DC3EF801F4CF0E9422DA0C945A37FB
:105E60000E94A0DA0C945A370E94AB9E0C945A37C9
:105E700088E690E00E94493F81110C945A37809146
:105E8000B70B83FF02C00C945A3783E50E94D93DBB
:105E9000882309F440C00E94613D0E9475F170930F
:105EA0005C0B60935B0B80E00E949ACF0E94613D87
:105EB00020E030E04AEA52E40E941AEC18163CF066
:105EC0000E94AB9E60E08CE893E00E94916C0E947F
:105ED000613D2091C50B3091C60B4091C70B50918D
:105EE000C80B0E9457F21816B4F48DE293E09F930A
:105EF0008F938091F20390E001969F938F9385E8B2
:105F000093E09F938F931F920E9405DA0FB6F89447
:105F1000DEBF0FBECDBF0E9406E2CCC78EE40E945A
:105F2000D93D882309F4C6C70E94313D6093A4136C
:105F30007093A5138093A6139093A713BBC783E513
:105F40000E94943D882359F083E50E94D93D88231F
:105F500019F00E94413D01C080E08093B70BE7E853
:105F6000F8E284918F010F5F1F4F882321F00E9478
:105F7000DC3EF801F6CFE9EAF3E084918F010F5F90
:105F80001F4F882321F00E94DC3EF801F6CF80915C
:105F9000B70B8823A1F16BE9C62E63E0D62EE12C66
:105FA000F12C20E08091B70B90E00E2C02C095956B
:105FB00087950A94E2F780FF17C0BB24B394B20E12
:105FC000222319F08CE20E94DC3EF60125913491E7
:105FD000F901849189010F5F1F4F882321F00E94EE
:105FE000DC3E9801F5CF2B2DFFEFEF1AFF0A32E0D0
:105FF000C30ED11C45E0E416F104A1F60CC0E5EA9D
:10600000F3E084918F010F5F1F4F882321F00E94DE
:10601000DC3EF801F6CF8AE00E94DC3E4BC780EB05
:1060200093E00E944ED10E94ABA644C783E50E9434
:10603000D93D882359F00E94413D809347028D331A
:1060400008F438C78CE38093470234C7E7E8F8E2E6
:1060500084918F010F5F1F4F882321F00E94DC3E47
:10606000F801F6CF4091470250E060E070E089EB24
:1060700093E00E943E4B8AE00E94DC3E1BC7809169
:10608000B70B83FD17C783E50E94D93D882309F428
:1060900011C70E94613D0E9475F17093D612609302
:1060A000D51208C789E690E00E94493F811111C0CE
:1060B000E0ECF3E084918F010F5F1F4F882321F004
:1060C0000E94DC3EF801F6CF0E9496438AE00E94CF
:1060D000DC3E10922312109222120C94243983E594
:1060E0000E94D93D882309F4E5C60E94413D809372
:1060F000AC138D3318F08CE38093AC130E9445856C
:106100006B017C012091AC1330E0A8EEB3E00E945B
:1061100021F0DC01CB018C0D9D1DAE1DBF1D8093B8
:10612000A8139093A913A093AA13B093AB13C2C65C
:106130008DE690E00E94493F8111BCC68091B70B6B
:1061400083FDB8C683E50E94D93D6C968FAF6C97EE
:106150008111E6C682E50E94D93D8111E1C6AAC639
:106160000E943F3EA7C60E94323EA4C60E94D5AC04
:10617000A1C61092F6039EC681E08093F6039AC6EC
:106180000E94E53D97C60E94C33D94C6D6018D91FD
:106190006D010E94943D882309F46DC0133009F00D
:1061A00063C00E94613D4B015C0120E030E040EAA9
:1061B00051E40E941AEC87FF4EC0A5019401609142
:1061C0001E1470911F1480912014909121140E942C
:1061D0000DF12B013C019B01AC016091BD1270914E
:1061E000BE128091BF129091C0120E947FEC60930A
:1061F000BD127093BE128093BF129093C012A30180
:1062000092016091911270919212809193129091EB
:1062100094120E947FEC609391127093921280937B
:1062200093129093941260913A0670913B0680917C
:106230003C0690913D060E941EECA30192010E9433
:106240007FEC0E947AF160933A0670933B0680934C
:106250003C0690933D0680921E1490921F14A092CB
:106260002014B092211407C00E94613DF7016083A1
:106270007183828393831F5FF4E0EF0EF11C14306F
:1062800009F084CF0E94DA4D15C60E948F440E9407
:10629000E64210C684918F010F5F1F4F882321F0C3
:1062A0000E94DC3EF801F6CFE5ECF4E084918F012A
:1062B0000F5F1F4F882321F00E94DC3EF801F6CFCC
:1062C000EEEAF4E084918F010F5F1F4F882321F0E5
:1062D0000E94DC3EF801F6CFEEE9F4E084918F01F4
:1062E0000F5F1F4F882321F00E94DC3EF801F6CF9C
:1062F000EDE8F4E084918F010F5F1F4F882321F0B8
:106300000E94DC3EF801F6CFECE7F4E084918F01C7
:106310000F5F1F4F882321F00E94DC3EF801F6CF6B
:10632000EDE6F4E084918F010F5F1F4F882321F089
:106330000E94DC3EF801F6CFE8E5F4E084918F019D
:106340000F5F1F4F882321F00E94DC3EF801F6CF3B
:10635000E2E4F4E084918F010F5F1F4F882321F066
:106360000E94DC3EF801F6CFEDE2F4E084918F016B
:106370000F5F1F4F882321F00E94DC3EF801F6CF0B
:10638000E0E1F4E084918F010F5F1F4F882321F03B
:106390000E94DC3EF801F6CFE8EFF3E084918F0134
:1063A0000F5F1F4F882309F485C50E94DC3EF8016A
:1063B000F5CF60E08091FE039091FF030E94B16CE5
:1063C00079C585E40E94943D882381F00E94523D66
:1063D000882361F0E7E8F8E284918F010F5F1F4F97
:1063E000882321F00E94DC3EF801F6CF81E40E9470
:1063F000943D882381F00E94523D882361F0E6E9B4
:10640000F5E084918F010F5F1F4F882321F00E94D8
:10641000DC3EF801F6CF0091FE031091FF03D80196
:106420008D918D01882309F4F6CD0E94DC3EF7CFD3
:10643000EBEBF5E084918F010F5F1F4F882321F074
:106440000E94DC3EF801F6CFE3EBF5E084918F018A
:106450000F5F1F4F882321F00E94DC3EF801F6CF2A
:10646000659903C00EE113E002C003E213E0F801F6
:1064700081918F01882319F00E94DC3EF8CF8AE0D9
:106480000E94DC3EEBEAF5E084918F010F5F1F4F25
:10649000882321F00E94DC3EF801F6CF80910301B1
:1064A00081FD03C00EE113E002C003E213E0D80156
:1064B0008D918D01882319F00E94DC3EF8CF8AE08F
:1064C0000E94DC3EE3EAF5E084918F010F5F1F4FED
:1064D000882321F00E94DC3EF801F6CF4B9903C0DF
:1064E0000EE113E002C003E213E0F80181918F0195
:1064F000882319F00E94DC3EF8CF8AE00E94DC3E3F
:10650000EAE9F5E084918F010F5F1F4F882321F0A6
:106510000E94DC3EF801F6CF4A9903C00EE113E079
:1065200002C003E213E0D8018D918D01882309F4A4
:1065300072CD0E94DC3EF7CF81E080937704809398
:10654000360BB8C4109277041092360BB3C483E5AF
:106550000E94D93D882319F00E94313D02C060E0BD
:1065600070E08B01112702301105CCF0EFE3F8E267
:1065700084918F010F5F1F4F882321F00E94DC3E22
:10658000F801F6CFE5EDF5E084918F010F5F1F4F25
:10659000882309F48FC40E94DC3EF801F5CF88E41B
:1065A0000E94D93D8823A9F00E94313D6A3A7105C5
:1065B0003CF06530B1E07B072CF064E071E002C094
:1065C0006AEA70E0F801EE0FFF1FE35AF44F71839F
:1065D000608386E40E94D93D882309F46BC40E943D
:1065E000313D000F111FF801EF59F44F71836083A3
:1065F0006F3F710519F014F06FEF70E077FF02C084
:1066000060E070E07183608355C488EC90E00E9484
:10661000493F81114FC484E40E94943D8823D1F105
:106620000E94613D11E020E030E0A9010E941AECD7
:10663000811101C010E01093A90B112359F10091B1
:10664000F20310E00E94613D000F111F000F111FA7
:10665000F801EB55F44F608371838283938320E0CC
:1066600030E0A9016091A50B7091A60B8091A70B5A
:106670009091A80B0E941AEC81110CC080E090E070
:10668000A0EEBFE38093A50B9093A60BA093A70B5E
:10669000B093A80B0E94F6D00DC4F5E9EF2EF2E1FD
:1066A000FF2E00EA12E0A4E0DA2ED00EF80181916C
:1066B0008F010E94943D882351F00E94613D0E9409
:1066C0007AF1D7016D937D938D939C931397B4E0EA
:1066D000EB0EF11CD012EACF0E94AD4CEBC375E873
:1066E000E72E72E1F72E00EA12E0E4E0DE2ED00E93
:1066F000F80181918F010E94943D882341F00E940E
:10670000613DD7016D937D938D939C931397B4E076
:10671000EB0EF11CD012ECCFCDC383E50E94943D6B
:106720008823D9F00E94613DAB01BC014093AD12BA
:106730005093AE126093AF127093B0124093A512B3
:106740005093A6126093A7127093A81281E596E069
:106750000E94784B8AE00E94DC3E80E50E94943DD6
:10676000882399F00E94613DAB01BC014093AD12BA
:106770005093AE126093AF127093B01284E396E020
:106780000E94784B8AE00E94DC3E82E50E94943DA4
:10679000882399F00E94613DAB01BC014093A9128E
:1067A0005093AA126093AB127093AC1285E196E0FD
:1067B0000E94784B8AE00E94DC3E84E50E94943D72
:1067C000882309F477C30E94613DAB01BC0140936B
:1067D000A5125093A6126093A7127093A81287EF88
:1067E00095E00E94784B8AE00E94DC3E63C383E51B
:1067F0000E94943D882351F00E94613D6093811274
:1068000070938212809383129093841284E50E9485
:10681000943D882351F00E94613D60937D127093F6
:106820007E1280937F129093801282E40E94943DA6
:10683000882351F00E94213D6093C4127093C512C9
:106840008093C6129093C71288E50E94943D8823D6
:1068500051F00E94613D6093B1127093B212809327
:10686000B3129093B41289E50E94943D882351F0AD
:106870000E94613D6093B5127093B6128093B71277
:106880009093B8128AE50E94943D882351F00E94AB
:10689000613D6093B9127093BA128093BB129093CA
:1068A000BC1285E40E94943D882309F403C30E942E
:1068B000613D6093BD127093BE128093BF1290939E
:1068C000C012F8C240EAA42E42E0B42E52E0C52E17
:1068D00054E1D52E6BE7E62E64E0F62E00E010E0E2
:1068E000F50181915F010E94943D882309F10E9486
:1068F000613D2B013C01D7012D913D914D915C9162
:106900000E9430F09B01AC01F601608171818281AF
:1069100093810E9431F0D6016D937D938D939C936A
:106920001397F7014082518262827382C8011FD798
:106930000F5F1F4FF4E0CF0ED11C24E0E20EF11CDC
:106940000330110569F6E0D70E94E642B3C28AE53A
:106950000E94943D882351F00E94613D60933B0B5F
:1069600070933C0B80933D0B90933E0B40913B0BFF
:1069700050913C0B60913D0B70913E0B89E796E086
:106980000E94784B8AE00E94DC3E94C20E9433ACA5
:1069900091C20E94BCAB8EC283E50E94D93D882380
:1069A00019F00E94313D02C064E071E079A368A350
:1069B00080E50E94D93D882339F00E94313D693835
:1069C00033E1730730F402C068EE73E07A836983C1
:1069D00004C088E893E19A838983BE01605E7F4F9B
:1069E000CE0101960E94A59D65C20E941FAB62C2A6
:1069F0000E94C9AA5FC20E9404A75CC2A1014A5CAE
:106A00005B4061965FAF4EAF6197D1018D911D01E3
:106A1000882309F4A2C0F70140805180628073800E
:106A2000F801E45BFD4F2081318142815381F801FF
:106A3000EF53FC4E60817181828193810E9431F01D
:106A400020E030E040E05FE30E947FEC9B01AC017E
:106A5000C301B2010E9457F2181644F4F801E4553C
:106A6000F54D85909590A590B49003C0812C912C04
:106A70005401F801E754F44F208131814281538160
:106A8000C301B2010E9430F09B01AC01C501B40109
:106A90000E9430F04B015C0120E030E040EA51EC14
:106AA0000E9457F287FD2AC020E030E040EA51E41E
:106AB000C501B4010E941AEC181604F1D6012D91FB
:106AC0003D914D915C91C501B4010E9430F09B0154
:106AD000AC01C301B2010E9431F0F7016083718300
:106AE00082839383D6018D929D92AD92BC9213972F
:106AF00061968EAD9FAD61973AD62FC0EFE3F8E275
:106B000084918F010F5F1F4F882321F00E94DC3E8C
:106B1000F801F6CFE9EBF6E084918F010F5F1F4F8C
:106B2000882321F00E94DC3EF801F6CF61E08BEA79
:106B300096E00E94916C0E94CFB888E290E09A8320
:106B4000898388EC90E099A388A3BE016F5F7F4F93
:106B5000CE0180960E94A59DADC1B4E0CB0ED11CA4
:106B60000C5F1F4FE4E0EE0EF11C0C30110509F034
:106B700045CFCAD60E94E64260E08BE996E00E94CB
:106B8000916C83E992E099A388A304E610E01A834C
:106B90000983BE01605E7F4FCE0101960E94A59DD4
:106BA0008AEB92E099A388A31A830983BE01605EF1
:106BB0007F4FCE0101960E94A59D7CC10E94697EF7
:106BC00079C10E94D37976C183E5AED7882311F0CD
:106BD00069D701C081E091E089270E9460516AC1B4
:106BE00085E4A2D7882311F06CD704C060E070E080
:106BF00080E090EC2F966CAF7DAF8EAF9FAF2F975C
:106C00008AE5D7D7882311F05CD704C060E070E034
:106C100080E291E42B966CAF7DAF8EAF9FAF2B9748
:106C200088E5C7D7882311F04CD704C060E070E036
:106C300080E490E427966CAF7DAF8EAF9FAF27972F
:106C400089E5B7D7882311F03CD704C060E070E035
:106C500080E490E423966CAF7DAF8EAF9FAF239717
:106C600085E562D7882311F02CD704C060E070E07E
:106C700088EC92EC6BAF7CAF8DAF9EAF8CE454D7B9
:106C8000882311F01ED703C060E070E0CB0168A339
:106C900079A38AA39BA382E48CD7882319F0E1D639
:106CA000F62E02C085E0F82EA090670EB090680E18
:106CB0008091341281117FC0CC24C394EF2C8E01BB
:106CC000055C1F4F9E01215C3F4FAE014D5B5F4F46
:106CD000BE01695B7F4FCE01855B9F4F0E941EB056
:106CE000882309F468C083E090E090932312809396
:106CF000221281E08093810B11E08091810B882327
:106D000009F43FC060E08F2DAED38091E20D88235F
:106D1000A1F188E090E00E94B35E8091810B88230E
:106D200021F081E00E94C6D1F8CF1092D1121092CA
:106D3000D2121092D3121092D4121092E20D0E942D
:106D40009ACF39D382E090E00E94B35E0E944585DD
:106D5000DC01CB0188539045AF4FBF4F8093D112D8
:106D60009093D212A093D312B093D4121092E20D4A
:106D70001093810B61E08F2D76D381E00E94C6D104
:106D8000BCCF81E090E0909323128093221280E0A8
:106D900090E0A8E4B2E489839A83AB83BC838091BA
:106DA0003412882341F04F2DBE016F5F7F4FCE011B
:106DB00080960E9483B1AA94AB2809F07BC00E9400
:106DC00022DA78C0EFE3F8E284918F010F5F1F4F62
:106DD000882319F0F1D7F801F7CFE7EDF6E08491B9
:106DE0008F010F5F1F4F882309F464C0E5D7F801B6
:106DF000F6CF81E0809319021092231483E594D694
:106E0000811103C00E9427D555C04CD6811152C0B4
:106E1000F9CFF0900004FF20F9F0E7E8F8E2849160
:106E20008F010F5F1F4F882319F0C6D7F801F7CFE6
:106E300084E5C2D76F2D70E080E090E04AE0C3D7D0
:106E400080E2BAD708E313E0D8018D918D01882341
:106E500009F4E1C8B1D7F8CF1092B80BE7E8F8E22F
:106E600084918F010F5F1F4F882319F0A5D7F80178
:106E7000F7CF6091B80B70E086EE96E00E94954BDC
:106E80008AE09AD717C0E7E8F8E284918F010F5F94
:106E90001F4F882319F090D7F801F7CF6091AD13F9
:106EA0007091AE1388EF96E00E94AE4B82E284D7D9
:106EB0008AE082D710922312109222120E9408D5E3
:106EC000C3C16115710519F4BC0161507109A0E0DD
:106ED000B0E00C94BB1BC5D5AB01BC014093F310D3
:106EE0005093F4106093F5107093F61082E490E1E3
:106EF0000E941C72DFCF61E0802F0E940A846E2DF9
:106F0000802F0E94DB83F12CB701802F0E944684E2
:106F10000930110579F6F0925A0BE092590BCACF5D
:106F2000D0D50E9475F170935C0B60935B0B80E091
:106F30000E949ACFC6D520E030E04AEA52E40E948F
:106F40001AEC181644F00E94AB9E60E08CED93E0C2
:106F50000E94916C02C00E9422DA60915B0B7091DA
:106F60005C0B072E000C880B990B0E9420EC2091E3
:106F7000C50B3091C60B4091C70B5091C80B0E94B6
:106F800057F21816B4F48DE293E09F938F9380919B
:106F9000F20390E001969F938F9385ED93E09F938A
:106FA0008F931F920E9405DA0FB6F894DEBF0FBED2
:106FB000CDBF0E9406E281E080939F0267961CAEDF
:106FC0001DAE1EAE1FAE67976B961CAE1DAE1EAEFD
:106FD0001FAE6B9760961FAE6097A0961FAEA097EE
:106FE0009CE3A4969FAFA497ACE1A896AFAFA897F7
:106FF000B6E4AC96BFAFAC97C12CD12C40E8E42EE0
:107000005FEBF52E812C912C540160915B0B7091FC
:107010005C0B072E000C880B990B0E9420EC162F9E
:10702000072F782E692E262F372F482F592FB6017C
:10703000C7010E941AEC882331F12091C50B3091D1
:10704000C60B4091C70B5091C80B612F702F872D35
:10705000962D0E941AEC881F8827881F60968FAF94
:1070600060976C96CFAC6C97CC2089F0882379F030
:1070700080919F02882309F41DCF60E083EC93E0A8
:107080000E94916C17CF1C2D0D2D7E2C6F2C0E9411
:1070900045856B017C01DC01CB016B962CAD3DADD0
:1070A0004EAD5FAD6B97821B930BA40BB50BB7FD79
:1070B00039C0D701C60188519C4FAF4FBF4F6B9667
:1070C0008CAF9DAFAEAFBFAF6B970E949643E1ED23
:1070D000F3E084912F019FEF491A590A882319F090
:1070E0006BD6F201F6CF81149104A104B104B1F082
:1070F000D501C401805F984DAF4FBF4FBC01CD019A
:107100006C197D098E099F0928EE33E040E050E0BC
:107110000E94F5EFCA01B901F8D602C08FE34CD640
:107120008AE04AD680E00E94C6D13BD62090C50BAB
:107130003090C60B4090C70B5090C80B9101A20134
:10714000612F702F872D962D0E9430F09F7781142C
:107150009104A104B10449F420E030E040E85FE389
:107160000E941AEC87FF0BC008C020E030E040E42A
:1071700050E40E9457F2181614F446015701609625
:10718000AFAD6097AA2309F443C067962CAD3DAD1F
:107190004EAD5FAD6797211531054105510541F0B1
:1071A000D701C601821B930BA40BB50BB7FD30C0F2
:1071B0009101A201A0966FADA097A4967FADA49770
:1071C000A8968FADA897AC969FADAC970E9430F073
:1071D00020E030E040EC5FE30E941AEC87FD48CFEE
:1071E000D701C601805A9541AF4FBF4F67968CAF0C
:1071F0009DAFAEAFBFAF6797A0962FAEA097A496F6
:107200003FAEA497A8964FAEA897AC965FAEAC974A
:1072100080919F02882309F42BCF81149104A1044B
:10722000B10429F4C12ED02EE72CF62CEECE90E13D
:10723000C91A97E2D90AE108F108C818D908EA087A
:10724000FB08F7FE15CFEECFC854DF4F0FB6F8940A
:10725000DEBF0FBECDBFDF91CF911F910F91FF9089
:10726000EF90DF90CF90BF90AF909F908F907F90E6
:107270006F905F904F903F902F90089590912414BD
:10728000E92FF0E0E957FB4F80839F5F943018F4BB
:107290009093241402C010922414809129068F5FC9
:1072A00080932906089582E08093DC1208958FB7B9
:1072B000F8949091A3132091A213291759F0E92F64
:1072C000F0E0EE5DFC4E208130E09F5F9F77909371
:1072D000A31302C02FEF3FEF8FBFC90108950F9393
:1072E0001F93CF93DF93EC010E9445850E811F8190
:1072F00028853985011511052105310559F52C859C
:107300002223A9F13A8521502C8721E0230F2A87D7
:107310004D85241301C01A86FE0124E0329FE00D42
:10732000F11D112406851785208931890A831B8365
:107330002C833D83DC01CB01800F911FA11DB11D6A
:107340008E839F83A887B9878C819D81892B79F053
:10735000409A0DC0DC01CB01801B910BA20BB30B3B
:10736000B7FD05C040981E821F8218861986DF91DE
:10737000CF911F910F910895CF92EF92FF920F93AB
:107380001F93E0900002F090010200910202109120
:107390000302C090B80B2EE034E14AE054E166E00D
:1073A00074E182E094E10E94DBBE1F910F91FF9097
:1073B000EF90CF900895CF92DF92EF92FF92CF930C
:1073C00081E080939F02C1E080919F02882309F4AD
:1073D00044C0CC2309F441C080E00E94C6D1609132
:1073E0005B0B70915C0BC0E06115710569F3072EB2
:1073F000000C880B990B0E9420EC9B01AC01609162
:10740000C50B7091C60B8091C70B9091C80B0E9461
:1074100030F06B017C0120E030E0A9010E9457F2BE
:1074200018165CF020E030E040E450ECC701B601F3
:107430000E941AEC87FFC8CF0BC020E030E040E488
:1074400050E4C701B6010E9457F218160CF0BCCFE9
:1074500089E090E00E94B35EB6CFCF91FF90EF90AD
:10746000DF90CF900895CF92DF92EF92FF920F932B
:107470001F93CF93DF9300D01F92CDB7DEB7182FA5
:10748000662351F01092720410926E0410926F04F1
:1074900010927004109271040E944585C0906E0491
:1074A000D0906F04E0907004F09071049B01AC01E7
:1074B0002C193D094E095F0957FD3EC017FD16C046
:1074C00040917204212F012E000C330B2C5F3F4F93
:1074D000E42F042E000CFF0B2E173F076CF1411711
:1074E0002CF000E911E020E030E004C004EC19E0E9
:1074F00020E030E0DC01CB01800F911FA21FB31F01
:1075000080936E0490936F04A0937004B093710401
:1075100080ED97E09C838B838CE291E09A83898352
:10752000BE016D5F7F4FCE0101960E94A59D8091A7
:1075300072048F5F809372040F900F900F900F90E2
:10754000DF91CF911F910F91FF90EF90DF90CF903F
:1075500008954F925F926F927F928F929F92AF9217
:10756000BF92CF92DF92EF92FF920F931F93CF9330
:10757000DF935C014B01EA018901409000025090C9
:1075800001026090020270900302288139814A81D1
:107590005B8160910A1470910B1480910C1490918E
:1075A0000D140E941AEC87FF29C0F801C080D18019
:1075B000E280F38020E030E0A901C701B6010E941B
:1075C0001AEC811106C0E0ECFAE2C590D590E59086
:1075D000F490C0920002D0920102E0920202F09276
:1075E000030288819981AA81BB8180930A149093B8
:1075F0000B14A0930C14B0930D14BEDEF801C080E0
:10760000D180E280F38020E030E0A901C701B6011B
:107610000E941AEC811107C085E5C82EDC2C85E09C
:10762000E82E83E4F82EC0920002D0920102E0928C
:107630000202F0920302F50180819181A281B3815F
:107640008093021490930314A0930414B093051430
:10765000F40180819181A281B3818093061490937B
:107660000714A0930814B093091486DE2881398189
:107670004A815B8160910A1470910B1480910C1403
:1076800090910D140E9457F218164CF5F801C08025
:10769000D180E280F38020E030E0A901C701B6018B
:1076A0000E941AEC811106C0E0ECFAE2C590D59078
:1076B000E590F490C0920002D0920102E0920202A2
:1076C000F092030288819981AA81BB8180930A1478
:1076D00090930B14A0930C14B0930D144DDE0E94E4
:1076E0008F44409200025092010260920202709216
:1076F0000302DF91CF911F910F91FF90EF90DF90E8
:10770000CF90BF90AF909F908F907F906F905F9041
:107710004F90089580E1E2E0F4E1A4E2B2E101904B
:107720000D928A95E1F7089580E1E4E2F2E1A2E0AA
:10773000B4E101900D928A95E1F70895CF92EF920E
:10774000FF920F931F93C090B80B7B018C0120E335
:1077500032E14CE252E168E272E184E292E10E949D
:10776000DBBE1F910F91FF90EF90CF900895CF92C5
:10777000DF92EF92FF920F931F93CF93DF93EC0171
:10778000CC0FDD1FCC0FDD1FFE01E558FB4F20E0C5
:1077900030E0A90160817181828193810E9431F082
:1077A000FE01EA5EFD4E20813181428153810E94BB
:1077B00031F06B017C01FE01E754F44F608371836B
:1077C00082839383FE01EA57F74F65917591859106
:1077D00094918E010F531C4EA70196010E9431F027
:1077E000F8016083718382839383FE01EE56F74F25
:1077F0006591759185919491C45BDD4FA7019601C8
:107800000E9431F0688379838A839B83DF91CF91D3
:107810001F910F91FF90EF90DF90CF900895CF933D
:10782000FC0180818B33A1F080912906843080F4A3
:10783000C62FBF018091241420E6829FC00111242D
:1078400088559B4F0E949AF38C2F18DD81E001C070
:1078500080E0CF910895DF92EF92FF920F931F93F4
:10786000CF93DF93CDB7DEB76E970FB6F894DEBF38
:107870000FBECDBF6091E00D7091E10D61157105F6
:1078800049F14DE150E0CE0101967C010E948AEB66
:107890001E8EF7018F010E191F09D190DD2019F0FE
:1078A0009AE0D912F7CFF701E00FF11F1082C7015C
:1078B0000E94E59D882371F0DD20A9F00F5F1F4F26
:1078C0008091E00D9091E10D080F191F1093E10DCB
:1078D0000093E00D81E02091E00D3091E10D232B2C
:1078E00029F480E003C000E010E0F0CF6E960FB600
:1078F000F894DEBF0FBECDBFDF91CF911F910F91E6
:10790000FF90EF90DF9008952EE034E14AE054E1DB
:1079100066E074E182E094E10C94174D9F92AF927F
:10792000BF92CF92DF92EF92FF920F931F93CF936C
:10793000DF9300D01F92CDB7DEB7902EA12EB22ECE
:10794000D32E7C01EE0CFF1CEE0CFF1C87010E5F9A
:107950001B4EF801108211821282138249835A83CE
:107960006B837C83D1DF49815A816B817C81F801F3
:107970004083518362837383C090B80B20E030E072
:10798000A901692D7A2D8B2D9D2D0E941AEC811154
:1079900008C0F701E854F54DE590F5900591149174
:1079A00006C0892D9A2DAB2DBD2D7C018D012EE0B9
:1079B00034E14AE054E166E074E182E094E10E943F
:1079C000DBBEADD71092A7040F900F900F900F90D1
:1079D000DF91CF911F910F91FF90EF90DF90CF90AB
:1079E000BF90AF909F9008951F920F920FB60F9285
:1079F00011248F9382E08093DC128F910F900FBE41
:107A00000F901F9018951F920F920FB60F9211248E
:107A10008F9382E08093DC128F910F900FBE0F90B6
:107A20001F9018951F920F920FB60F9211248F93EB
:107A300082E08093DC128F910F900FBE0F901F9009
:107A400018958091030490910404009731F04AE066
:107A500050E060E070E00C9436EA60E070E0CB014A
:107A600008958091030490910404009731F04AE056
:107A700050E060E070E00C940EE960E070E0CB0153
:107A80000895EFDF97FD0AC0ECDF6F3F71058105B8
:107A9000910509F02CF4E5DF862F089580E0089524
:107AA0008FEF08958091030490910404892B31F0A5
:107AB000E8DF91E0811103C090E001C091E0892FDF
:107AC00008950F931F93CF93809103049091040422
:107AD0000097F1F0FC018F01C1912C2F2F7D89F0CF
:107AE000C53411F0C536B9F7F801108260E070E0D6
:107AF0000E94A8E7F801C083562F472F382F292F5F
:107B00000BC060E070E0CF911F910F910C94A8E73B
:107B100050E040E030E020E0652F742F832F922F5B
:107B2000CF911F910F91089581548A3150F5482FBC
:107B300050E0FA0193E0F595E7959A95E1F7E25167
:107B4000FC4F208130E08770B90102C075956795C0
:107B50008A95E2F760FF15C0FA01EC52FC4F2081D4
:107B6000222339F08091AD139091AE13820F911DB5
:107B700002C080E090E0909304048093030481E0CD
:107B8000089580E0089583E5CFDF882389F099DFA9
:107B900020E030E04AE754E40E947FEC0E947AF152
:107BA0006093B3137093B4138093B5139093B6138B
:107BB0000895BADF882341F081E0209103043091D9
:107BC0000404232B09F480E0089583E5F2DF882381
:107BD00091F077DF20E030E04AE754E40E947FEC48
:107BE0000E947AF1609348027093490280934A029E
:107BF00090934B02089588E597DF81110FC089E5C6
:107C000093DF81110BC08AE58FDF811107C085E406
:107C10008BDF811103C083D60C943DD180D688E5DB
:107C200083DF882319F05F9A1092780489E57CDF5E
:107C3000882319F08A9A109279048AE575DF8823DF
:107C400059F09FB7F89480910801816080930801F2
:107C50009FBF479A10927A0485E466DF81110C94E5
:107C60003BD1089580E5A5DF811105C010925A0B24
:107C70001092590B0895F5DE672BC1F30895CF9349
:107C8000DF9383E596DF882331F0EBDEEB016F3F76
:107C9000710519F010F0CFEFD0E080E58ADF811197
:107CA00005C0D0935A0BC093590B03C0EADE88235A
:107CB000C1F3DF91CF910895BF92CF92DF92EF92FF
:107CC000FF920F931F93CF93DF9384E2E82E82E11C
:107CD000F82E02E014E193EFC92E93E0D92EC0EA0A
:107CE000D2E0BC2E84E0B80E89911EDF8823D1F04B
:107CF000E8DEF6012081211104C02091F703222340
:107D000031F0F801208131814281538103C020E0AC
:107D100030E0A9010E9431F0F70160837183828312
:107D200093830AC0F80180819181A281B381F70118
:107D300080839183A283B383F4E0EF0EF11C0C5F88
:107D40001F4F8FEFC81AD80ABC12CECF86E431DF9E
:107D50008823B9F0B6DE20E030E0A9010E9457F296
:107D600018167CF4AEDE20E030E040E752E40E94DA
:107D70000DF16093000270930102809302029093D0
:107D80000302DF91CF911F910F91FF90EF90DF9051
:107D9000CF90BF900895FC01238121110C9433787A
:107DA00008950E9445856093AF137093B01380933C
:107DB000B1139093B21308959091C00095FFFCCF3A
:107DC0008093C60008958F929F92AF92BF92EF92D8
:107DD000FF921F93CF93DF93CDB7DEB7A0970FB677
:107DE000F894DEBF0FBECDBF611571058105910509
:107DF00079F110E0842E912CA12CB12CEE24E39487
:107E0000F12CEC0EFD1EE10EF11C17FDFA94A501FC
:107E100094010E94F5EFF7016083B901CA011F5F69
:107E2000611571058105910549F7115010F1E1E0E7
:107E3000F0E0EC0FFD1FE10FF11D17FDFA958081B9
:107E40008A3010F097E301C090E3890FB5DFEDCFE2
:107E500080E3A0960FB6F894DEBF0FBECDBFDF91D2
:107E6000CF911F91FF90EF90BF90AF909F908F9018
:107E7000A3CFA0960FB6F894DEBF0FBECDBFDF91A3
:107E8000CF911F91FF90EF90BF90AF909F908F90F8
:107E90000895EF92FF920F931F93CF93DF937C018E
:107EA00084E587DED82F882321F1EBDDC82F181653
:107EB000E4F4E7E8F8E284918F010F5F1F4F882315
:107EC00019F07ADFF801F7CF8DE476DFB70180E0B3
:107ED00090E04AE078DF6C2FCC0F770B83E798E0D7
:107EE0000E94954B8AE068DF08C08093F203D0E0DF
:107EF00004C08091B80B8093F2038D2FDF91CF9156
:107F00001F910F91FF90EF900895CF92DF92EF9223
:107F1000FF926B017C0197FF0AC08DE24DDFF09468
:107F2000E094D094C094C11CD11CE11CF11C4AE027
:107F3000C701B601FF90EF90DF90CF9044CFEF9252
:107F4000FF920F931F93CF93DF931F92CDB7DEB7AE
:107F5000082F162FEFE3F8E284917F012FEFE21A4A
:107F6000F20A882329F0998327DFF7019981F4CF5A
:107F7000E02FF92F84917F019FEFE91AF90A8823F6
:107F800019F01ADFF701F6CF6091A4137091A513D1
:107F90008091A6139091A713B8DF8AE00DDF11112D
:107FA0000E9427D510926A04109269040F90DF9105
:107FB000CF911F910F91FF90EF9008952F923F92D4
:107FC0004F925F926F927F928F929F92AF92BF92E9
:107FD000CF92DF92EF92FF920F931F93CF93DF9395
:107FE0001F92CDB7DEB737DC81116BC280912906B5
:107FF000843020F45CD99C0197FF40C18091770EBA
:10800000882309F45EC280912906811102C0109272
:108010006D04EE24E3944091F3105091F4106091BC
:10802000F5107091F6108091EF109091F010A091E2
:10803000F110B091F210481759076A077B0708F44E
:10804000E12C00E010E09924939480E6882E94E4DB
:10805000C92E98E0D92E20E4A22E28E0B22E3DE8C9
:10806000732E80912906843008F02BC2E11029C2BA
:1080700080916D04811125C280914A1090914B101E
:10808000A0914C10B0914D108093F3109093F41088
:10809000A093F510B093F61041E050E0BE016F5F81
:1080A0007F4F82E490E10E944274019719F4898124
:1080B00090E002C08FEF9FEFF82EEE24E394209023
:1080C000F3103090F4104090F5105090F61040915D
:1080D000EF105091F0106091F1107091F210241691
:1080E000350646065706C8F4E12C8F3FEFEF9E0792
:1080F00009F478C0FAE08F1709F491C02DE08217D7
:1081000009F48DC083E2F81619F09AE3F9129CC0C5
:1081100080916C04811198C07DC0EFE5F8E08491F6
:108120002F012FEF421A520A882319F045DEF2017F
:10813000F6CFF5D382E490E10E94337880915D1010
:10814000882359F1815080935D10789EC0011124DD
:1081500041E061E08E599F4E0E943D99E0915D1093
:1081600084E0E89FF0011124E25AFF4E40815181E2
:10817000628173814093F3105093F4106093F51073
:108180007093F61082E490E10E941C728091780E48
:108190008823C1F09092770E15C01092770ED0927E
:1081A000E10DC092E00D57DB0E94AB9E0E9408A13A
:1081B0006D3371058105910528F0B092E10DA09213
:1081C000E00D49DB1092FB108091780E882319F0A6
:1081D0000E94AA9B1FC00E945D9C8091780E811115
:1081E000F7CF18C0EFE3F8E284912F019FEF491A0F
:1081F000590A882319F0E0DDF201F6CFE0E5F8E056
:1082000084912F012FEF421A520A882319F0D4DDEE
:10821000F201F6CF83E2F81202C090926D04109240
:108220006C040115110509F41CCF80912414889E5B
:10823000000D111D1124F801E855FB4F108280E05C
:108240001DD800E010E00DCF0F35110508F009CF63
:108250009BE3F91202C090926C0480916C0481112E
:1082600000CF80912414F801889EE00DF11D1124A7
:10827000E855FB4FF0820F5F1F4FF3CE982F009110
:10828000690410916A048A3019F09D3009F0EBC03E
:1082900010926B040115110509F4A8CEF801E75FEF
:1082A000FB4F108210926A041092690429E034E0B6
:1082B0006901F90180812F5F3F4F8032C9F3860148
:1082C0008E3411F0C12CD12C6AE270E0C8010E94FA
:1082D00086F35C01C114D10409F475C06BE378E046
:1082E000C8010E9499EBFF24F394892B11F4F12C1F
:1082F00009C06EE470E0C80104960E9486F30097FE
:1083000009F06C014AE050E060E070E0C6010196BF
:108310000E940EE96093050470930604809307049D
:10832000909308044090A4135090A5136090A61356
:108330007090A713FFEF4F1A5F0A6F0A7F0A641548
:1083400075058605970531F0F11004C061E088E0FD
:1083500098E026C0A114B10401F180E0F12CF801ED
:10836000E80FF11D90819A3219F08F5FF926F7CF4F
:108370004AE050E060E070E0C50101960E940EE91D
:10838000CF2CD12CE12CF12C6C157D058E059F0591
:1083900049F061E089EE97E003C061E08FEB97E080
:1083A000CEDD2CCE8091050490910604A0910704A7
:1083B000B09108048093A4139093A513A093A613DF
:1083C000B093A71306C0892B21F060E08BE097E003
:1083D000E7CF80911902811122C067E470E0C801E3
:1083E0000E9486F30097D9F04AE050E060E070E028
:1083F00001960E940EE96430710588F4E8E4F7E024
:1084000084917F012FEFE21AF20A882319F0D4DC5D
:10841000F701F6CF60E08EE397E00E94916C69E48B
:1084200073E0C8010E9491F3892B21F410929F02FE
:108430001092810B6EE473E0C8010E9491F3892BC6
:1084400021F485E397E00E944ED163E573E0C80113
:108450000E9491F3892B11F40E94ABA661E089E0A0
:1084600094E0DDD9C3CD0F3511050CF0BFCD9C359F
:10847000A1F40E94573997FDB9CD20916B042111C9
:10848000B5CD98012F5F3F4F30936A042093690464
:10849000F801E75FFB4F8083A9CD9B3319F481E09E
:1084A00080936B0480916B048111A0CDC80101966B
:1084B00090936A0480936904F801E75FFB4F20837F
:1084C00095CD0F90DF91CF911F910F91FF90EF907D
:1084D000DF90CF90BF90AF909F908F907F906F90E4
:1084E0005F904F903F902F9008958F929F92AF9200
:1084F000BF92CF92DF92EF92FF92CF936B017C01FC
:10850000B42E20E030E0A9010E941AEC87FF06C0DB
:108510008DE252DCF7FAF094F7F8F094C0E060E0F6
:1085200070E080E09FE3CB1541F02DEC3CEC4CEC8F
:108530005DE30E947FECCF5FF6CF9B01AC01C701EA
:10854000B6010E9431F06B017C010E947AF14B016F
:108550005C014AE038DCCC2379F1C501B4010E940A
:108560001EEC9B01AC01C701B6010E9430F06B010B
:108570007C018EE221DC20E030E040E251E4C701E2
:10858000B6010E947FEC4B015C010E9475F16B010A
:10859000770FEE08FF08C701B601B7DCC701B601C7
:1085A0000E9420EC9B01AC01C501B4010E9430F097
:1085B0006B017C01C150F9F6CF91FF90EF90DF90F5
:1085C000CF90BF90AF909F908F9008954F925F9201
:1085D0006F927F928F929F92AF92BF92CF92DF92D3
:1085E000EF92FF92CF93DF93E3ECF8E08491EF01F9
:1085F0002196882319F0E0DBFE01F8CF6091021488
:1086000070910314809104149091051442E06DDF81
:10861000EFEBF8E08491EF012196882319F0CCDB91
:10862000FE01F8CF60910614709107148091081430
:108630009091091442E059DFEBEBF8E08491EF01EF
:108640002196882319F0B8DBFE01F8CF60910A1457
:1086500070910B1480910C1490910D1442E045DF41
:10866000E7EBF8E08491EF012196882319F0A4DB71
:10867000FE01F8CF60910E1470910F1480911014C8
:108680009091111442E031DF8FB7F8944090F213CB
:108690005090F3136090F4137090F5138090F613DC
:1086A0009090F713A090F813B090F913C090FA13BC
:1086B000D090FB13E090FC13F090FD138FBFEDEA18
:1086C000F8E08491EF012196882319F075DBFE0113
:1086D000F8CFC301B20119DCE9EAF8E08491EF01B7
:1086E0002196882319F068DBFE01F8CFC501B4019B
:1086F0000CDCE5EAF8E08491EF012196882319F07B
:108700005BDBFE01F8CFC701B601FFDB8AE0DF913A
:10871000CF91FF90EF90DF90CF90BF90AF909F9060
:108720008F907F906F905F904F9046CB8F929F92EB
:10873000AF92BF92CF92DF92EF92FF92CF93DF93EF
:1087400060915B0B70915C0B072E000C880B990BF2
:108750000E9420EC6B017C018090C50B9090C60BB1
:10876000A090C70BB090C80B80E226DB84E524DB29
:108770008AE322DB42E0C501B401B7DEB701A601FE
:108780008EE998E0B5D7E1EAF8E08491EF0121960F
:10879000882319F011DBFE01F8CFE091F203F0E03D
:1087A000E152FD4E608170E080E090E0DF91CF917A
:1087B000FF90EF90DF90CF90BF90AF909F908F9001
:1087C000A4CB1F920F920FB60F9211240BB60F92EB
:1087D0002F938F939F93EF93FF93E091A21381E0E8
:1087E0008E0F8F779091C6002091A313821731F0DE
:1087F000F0E0EE5DFC4E90838093A213FF91EF9129
:108800009F918F912F910F900BBE0F900FBE0F90E5
:108810001F901895CF92DF92FF920F931F93CF93E3
:10882000DF931F921F92CDB7DEB7F82E8A01809199
:108830001902882309F43EC0EFE3F8E284916F0146
:108840009FEFC91AD90A882339F069837A83B4DA89
:10885000F60169817A81F2CFFB0184916F019FEF6C
:10886000C91AD90A882319F0A7DAF601F6CFE3E48A
:10887000F2E184916F019FEFC91AD90A882319F098
:108880009BDAF601F6CFF7FC09C06F2DFF0C770BD2
:10889000880B990B3ADB8AE08FDA0CC0EEE3F2E149
:1088A00084916F019FEFC91AD90A882319F084DADD
:1088B000F601F6CF8091350B811108C01092190294
:1088C00081E08093350BC8010E944ED10F900F902C
:1088D000DF91CF911F910F91FF90DF90CF900C947B
:1088E000E5CFCF93DF932FB7F894EC01CC0FDD1FCA
:1088F000CC0FDD1FFE01EE50FC4E60817181828144
:1089000093812FBF0E9420ECC557DB4F288139810E
:108910004A815B810E947FECDF91CF910895909115
:10892000470E8091480E981721F080E00E94C6D132
:10893000F6CF08958091120B80FF03C089988FEFC6
:1089400002C0899A81E080933F028091120B81FFDF
:1089500003C08F988FEF02C08F9A81E0809340020E
:108960008091120B9FB782FF0AC0F89480910B018F
:10897000826080930B019FBF439A8FEF09C0F894E8
:1089800080910B018D7F80930B019FBF439881E005
:10899000809341028091120B83FF03C0169A8FEFE0
:1089A00002C0169881E08093420208959091470E8C
:1089B0008091480E981731F08091480E8F5F8F702C
:1089C0008093480E08951F920F920FB60F921124B4
:1089D0000BB60F92BF92CF92DF92EF92FF920F935E
:1089E0001F932F933F934F935F936F937F938F9337
:1089F0009F93AF93BF93EF93FF93CF93DF9300D0F9
:108A00001F92CDB7DEB780916E008B7F80936E0092
:108A100080916F008D7F80936F0078948091150B0B
:108A20009091160B0097C9F08C0101501109109319
:108A3000160B0093150B1092140B1092130BB6DF4C
:108A4000012B41F482E392E19093E10D8093E00DDC
:108A50000E942B3C88EC90E0B5C1C090130BD090E5
:108A6000140BC114D10409F0B2C19091470E80914A
:108A7000480E981749F19091480E0DE4909F90018F
:108A80001124225C394F8091750B9091760BA09147
:108A9000770BB091780BF901E75BFF4F4081518173
:108AA00062817381841B950BA60BB70B8093750BAA
:108AB0009093760BA093770BB093780BD9018C91A0
:108AC00088608C9369010BC08FB7F8941092750B76
:108AD0001092760B1092770B1092780B8FBFD0927A
:108AE000140BC092130BC114D10409F469C1F6012F
:108AF00052A18091120B418158130AC0242F30E0FB
:108B000080911802082E000C990B2817390729F0BC
:108B10005093120B409318020DDF1092310B1092FC
:108B2000320B1092330B1092340BD601D7968D91E5
:108B30009C91D8978134BCE99B0728F48132EEE4FC
:108B40009E0748F002C080E49CE99695879596952B
:108B5000879524E007C08131F7E29F0730F09695B2
:108B6000879522E02093300B08C021E02093300B42
:108B70008032910510F480E290E08C0100521109DE
:108B8000011528E01207D8F0E12FFF27EE0FFF1F95
:108B9000EE0FFF1FCF018E5C914FFC013296459185
:108BA0005491AA27059F9001049F210D3A1F069416
:108BB0002A1F3A1F1124FC01859194911CC0980131
:108BC000369527952C7F2E5C354FF9018591949130
:108BD000F901329665917491A80147705527649FF9
:108BE0009001659F300D749F300D112443E0369540
:108BF00027954A95E1F7821B930B8436910580F403
:108C000088E5E82E83E0F82ED7018D917D01882339
:108C100011F0D2D8F9CFC8010E94D99D84E690E026
:108C200090932F0B80932E0B8091300B80932D0B04
:108C3000F60183AD94AD90932C0B80932B0B813474
:108C4000FCE99F0728F481320EE4900748F002C047
:108C500080E49CE9969587959695879524E007C0D2
:108C6000813117E2910730F09695879522E02093A5
:108C7000300B08C021E02093300B8032910510F4B6
:108C800080E290E08C0100521109011528E01207E2
:108C9000D8F0E12FFF27EE0FFF1FEE0FFF1FCF01D0
:108CA0008E5C914FFC01329645915491AA27059F05
:108CB0009001049F210D3A1F06942A1F3A1F112488
:108CC000FC01859194911CC09801369527952C7FC5
:108CD0002E5C354FF90185919491F9013296659199
:108CE0007491A80147705527649F9001659F300DCE
:108CF000749F300D112473E0369527957A95E1F72E
:108D0000821B930B8436910580F458E5E52E53E0E1
:108D1000F52ED7018D917D01882311F04DD8F9CF23
:108D2000C8010E94D99D84E690E0AC0160E070E04B
:108D30004093270B5093280B6093290B70932A0BB9
:108D40009093890080938800F60182899389A48991
:108D5000B589B695A79597958795B095A095909567
:108D600081959F4FAF4FBF4F8093230B9093240B60
:108D7000A093250BB093260B80931F0B9093200B91
:108D8000A093210BB093220B80931B0B90931C0B91
:108D9000A0931D0BB0931E0B8093170B9093180B91
:108DA000A093190BB0931A0B10920E0B10920F0B8D
:108DB0001092100B1092110B82E08093DC1207C00E
:108DC00080ED97E090938900809388000BC4809198
:108DD000DC12882321F080917704811136C4209120
:108DE000300B222309F4EEC1E091130BF091140B28
:108DF0004091170B5091180B6091190B70911A0B41
:108E000082819381A481B581840F951FA61FB71F0E
:108E10008093170B9093180BA093190BB0931A0B18
:108E2000181619061A061B060CF4889AE091130B03
:108E3000F091140B40911B0B50911C0B60911D0B7A
:108E400070911E0B86819781A085B185840F951F37
:108E5000A61FB71F80931B0B90931C0BA0931D0B99
:108E6000B0931E0B181619061A061B060CF48E9AE0
:108E7000E091130BF091140B40911F0B5091200BBC
:108E80006091210B7091220B82859385A485B58515
:108E9000840F951FA61FB71F80931F0B9093200B65
:108EA000A093210BB093220B181619061A061B0665
:108EB0003CF58091DB128823D1F08091D91282FF9A
:108EC00004C08091410287FD05C08091D81288239B
:108ED00009F4C2C38091D91287FF04C08091410276
:108EE00087FD0EC08091D71281110AC008C09FB7BC
:108EF000F89480910B01886080930B019FBF419A89
:108F0000E091130BF091140B4091230B5091240B23
:108F10006091250B7091260B86859785A089B18974
:108F2000840F951FA61FB71F8093230B9093240BCC
:108F3000A093250BB093260B181619061A061B06CC
:108F40000CF4149A8091170B9091180BA091190BA7
:108F5000B0911A0B181619061A061B0684F5E09133
:108F6000130BF091140B4289538964897589841B12
:108F7000950BA60BB70B8093170B9093180BA09330
:108F8000190BB0931A0B80913F024091F21350914C
:108F9000F3136091F4137091F513082E000C990BE4
:108FA000AA0BBB0B840F951FA61FB71F8093F2134C
:108FB0009093F313A093F413B093F51388988091D2
:108FC0001B0B90911C0BA0911D0BB0911E0B181642
:108FD00019061A061B0684F5E091130BF091140B89
:108FE0004289538964897589841B950BA60BB70B3D
:108FF00080931B0B90931C0BA0931D0BB0931E0B27
:10900000809140024091F6135091F7136091F8134C
:109010007091F913082E000C990BAA0BBB0B840F4F
:10902000951FA61FB71F8093F6139093F713A09375
:10903000F813B093F9138E9880911F0B9091200B29
:10904000A091210BB091220B181619061A061B06C7
:109050000CF056C0E091130BF091140B4289538928
:1090600064897589841B950BA60BB70B80931F0B26
:109070009093200BA093210BB093220B809141027F
:109080004091FA135091FB136091FC137091FD1302
:10909000082E000C990BAA0BBB0B840F951FA61F63
:1090A000B71F8093FA139093FB13A093FC13B09314
:1090B000FD138091DB128823D1F08091D91282FFB9
:1090C00004C08091410287FD05C08091D812882399
:1090D00009F4CBC28091D91287FF04C0809141026C
:1090E00087FD0EC08091D71281110AC008C09FB7BA
:1090F000F89480910B01877F80930B019FBF41986B
:109100008091230B9091240BA091250BB091260BFD
:10911000181619061A061B0684F5E091130BF09138
:10912000140B4289538964897589841B950BA60B9E
:10913000B70B8093230B9093240BA093250BB09334
:10914000260B809142024091FE135091FF136091D3
:10915000001470910114082E000C990BAA0BBB0B84
:10916000840F951FA61FB71F8093FE139093FF13C4
:10917000A0930014B0930114149880910E0B909159
:109180000F0BA091100BB091110B0196A11DB11DF9
:1091900080930E0B90930F0BA093100BB093110BB9
:1091A0002150E091130BF091140B4289538964898B
:1091B000758984179507A607B70708F412CEBB2454
:1091C000B39401C0B12C40910E0B50910F0B6091E4
:1091D000100B7091110BE090130BF090140BF70132
:1091E00086899789A08DB18D84179507A607B70743
:1091F00008F4DCC04091270B5091280B6091290B9B
:1092000070912A0B068D178D20A131A1AA27419FAD
:10921000B12D529FC001629F900D619F800D911DE5
:10922000429FB00D811D9A1F519FB00D811D9A1F45
:10923000609FB00D811D9A1F509FB10D8A1F9A1F0C
:10924000B6958A1F9A1F349F800D911D359F900DF2
:10925000112423AD34AD820F931F90932C0B809378
:109260002B0B47A950AD61AD72ADA0E0B0E048173F
:1092700059076A077B0720F450932C0B40932B0B64
:1092800080912B0B90912C0B8134BCE99B0728F427
:109290008132EEE49E0748F002C080E49CE9969596
:1092A00087959695879524E007C08131F7E29F075F
:1092B00030F09695879522E02093300B08C021E08E
:1092C0002093300B8032910510F480E290E08C0105
:1092D00000521109011528E01207D8F0E12FFF27ED
:1092E000EE0FFF1FEE0FFF1FCF018E5C914FFC01B1
:1092F000329645915491AA27059F9001049F210D14
:109300003A1F06942A1F3A1F1124FC01859194915B
:109310001CC09801369527952C7F2E5C354FF9019E
:1093200085919491F901329665917491A8014770E5
:109330005527649F9001659F300D749F300D112457
:10934000B3E036952795BA95E1F7821B930B8436E7
:10935000910588F4F8E5EF2EF3E0FF2ED7018D910B
:109360007D01882319F00E94DC3EF8CFC8010E94DD
:10937000D99D84E690E09093890080938800409185
:10938000270B5091280B6091290B70912A0B8A01B1
:109390009B01080F191F211D311D0093270B1093EE
:1093A000280B2093290B30932A0B00C140910E0B00
:1093B00050910F0B6091100B7091110BF701828D82
:1093C000938DA48DB58D84179507A607B70708F070
:1093D000E1C02091310B3091320B4091330B509111
:1093E000340B29833A834B835C83468D578D60A170
:1093F00071A109811A812B813C81AA27059FB12D7A
:10940000169F6001269FD00C259FC00CD11C069F83
:10941000B00DC11CDA1E159FB00DC11CDA1E249FB1
:10942000B00DC11CDA1E149FB10DCA1EDA1EB6950E
:10943000CA1EDA1E709FC00CD11C719FD00C112463
:1094400080912B0B90912C0BFF96C816D90680F4B7
:109450008C199D0940815181628173816C01E12CDD
:10946000F12CC416D506E606F70620F4CA0102C0A0
:109470008081918181341CE9910728F481322EE4A6
:10948000920748F002C080E49CE9969587959695EE
:10949000879524E007C0813137E2930730F0969535
:1094A000879522E02093300B08C021E02093300BF9
:1094B0008032910510F480E290E08C010052110995
:1094C000011548E01407E8F0E12FFF27EE0FFF1F1A
:1094D000EE0FFF1FCF018E5C914FFC01329645913C
:1094E0005491AA27059F9001049F210D3A1F0694CD
:1094F0002A1F3A1F1124FC0185919491821B930B22
:1095000020C0C801969587958C7F8E5C954FFC0195
:1095100025913491FC01329665917491A8014770B0
:109520005527649FC001659F900D749F900D112475
:1095300043E0969587954A95E1F7D901A81BB90BA9
:10954000CD018436910588F488E5E82E83E0F82E75
:10955000F70181917F01882319F00E94DC3EF8CF4A
:10956000C8010E94D99D84E690E090938900809381
:10957000880029813A814B815C81280F391F411D68
:10958000511D2093310B3093320B4093330B50938A
:10959000340B0CC080912E0B90912F0B909389006F
:1095A0008093880080912D0B8093300B2091880050
:1095B0003091890080918400909185004096281711
:1095C000390748F4809184009091850040969093EB
:1095D000890080938800BB2029F01092140B109210
:1095E000130BE4D9F8948091E012882321F0809144
:1095F0006E008B7F03C080916E00846080936E004C
:1096000080916F00826080936F000F900F900F9099
:109610000F90DF91CF91FF91EF91BF91AF919F910B
:109620008F917F916F915F914F913F912F911F91FA
:109630000F91FF90EF90DF90CF90BF900F900BBEF7
:109640000F900FBE0F901F90189528D58091DC12B7
:1096500081508093DC12C3CB9FB7F89480910B01AB
:10966000886080930B019FBF35CC9FB7F8948091A1
:109670000B01877F80930B019FBF2CCDCF92DF9290
:10968000EF92FF92CF93DF936A017B01FC018491FB
:10969000EF012196882321F00E94DC3EFE01F7CFE6
:1096A0004AE0C701B601DF91CF91FF90EF90DF90C4
:1096B000CF900C94E33ECF92DF92EF92FF92CF9344
:1096C000DF936A017B01FC018491EF0121968823DD
:1096D00021F00E94DC3EFE01F7CF42E0C701B60157
:1096E000DF91CF91FF90EF90DF90CF900C94754277
:1096F000CF92DF92EF92FF92CF93DF936A017B01CB
:10970000FC018491EF012196882321F00E94DC3E28
:10971000FE01F7CF42E0C701B601DF91CF91FF9084
:10972000EF90DF90CF900C9475420F931F93CF93DF
:10973000DF938B01FC018491EF012196882321F0B6
:109740000E94DC3EFE01F7CFB801110F880B990B88
:10975000DF91CF911F910F910C94853F0F931F9331
:10976000CF93DF931F921F92CDB7DEB7FC01849198
:109770008F010F5F1F4F811102C08B0108C06983E9
:109780007A830E94DC3EF80169817A81F0CFF8018A
:1097900081918F01882319F00E94DC3EF8CF0F9051
:1097A0000F90DF91CF911F910F9108954F925F928B
:1097B0006F927F928F929F92AF92BF92CF92DF92E1
:1097C000EF92FF920F931F93CF93DF93CDB7DEB746
:1097D0002C970FB6F894DEBF0FBECDBF2B013C0116
:1097E00029833A834B835C83ED82FE820F83188743
:1097F000A986BA86CB86DC8628A139A14AA15BA1BD
:1098000060E070E080E89FE30E9430F06B017C0133
:1098100029813A814B815C810E947FEC4B015C0184
:109820002D813E814F81588568A179A18AA19BA194
:109830000E947FEC9B01AC01C501B4010E9431F094
:109840004B015C01A3019201C701B6010E947FECAC
:109850002B013C0129813A814B815C8168A179A16E
:109860008AA19BA10E947FEC9B01AC01C301B201C4
:109870000E9431F09B01AC01C701B6010E947FEC50
:109880002B013C01A501940168A179A18AA19BA1AA
:109890000E947FEC9B01AC01C301B2010E9431F038
:1098A0009B01AC01C701B6010E947FEC2B013C017A
:1098B000A5019401C701B6010E947FEC4B015C0138
:1098C0002D813E814F815885C701B6010E947FECF2
:1098D0006B017C0129853A854B855C8568A179A15E
:1098E0008AA19BA10E947FEC9B01AC01C701B6013C
:1098F0000E9431F09B01AC0168A179A18AA19BA1D2
:109900000E947FEC9B01AC01C501B4010E9431F0C3
:109910009B01AC0168A179A18AA19BA10E947FEC67
:109920009B01AC01C301B2010E9431F02C960FB62D
:10993000F894DEBF0FBECDBFDF91CF911F910F9185
:10994000FF90EF90DF90CF90BF90AF909F908F905F
:109950007F906F905F904F9008958F929F92AF92FB
:10996000BF92CF92DF92EF92FF920F931F93CF930C
:10997000DF9300D01F92CDB7DEB785E9882E82E154
:10998000982E92E1A92E94E1B92E0EE216E0C12C98
:10999000D12C7601C394F4016191719181919191DF
:1099A0004F01F50121913191419151915F0129833D
:1099B0003A834B835C830E941EEC29813A814B8160
:1099C0005C810E947FEC0E947AF1F80161937193AF
:1099D000819391938F01C616D706E806F90610F415
:1099E0006B017C01F5EA8F16F2E19F06A1F66FEF9D
:1099F0007FEFCB01A70196010E94F5EF20932A0685
:109A000030932B0640932C0650932D060F900F9009
:109A10000F900F90DF91CF911F910F91FF90EF90DA
:109A2000DF90CF90BF90AF909F908F9008952F922E
:109A30003F924F925F926F927F928F929F92AF92DE
:109A4000BF92CF92DF92EF92FF920F931F93CF932B
:109A5000DF9300D01F92CDB7DEB77B016A011901F9
:109A6000A2E1B4E12D913D914D915C91FC016081A9
:109A70007181828193810E947FEC0E9462F22B01AE
:109A80003C0107E31EE0D8016D937D938D939C9379
:109A90001397209116143091171440911814509177
:109AA0001914F70160817181828193810E947FEC9A
:109AB0000E9462F24B015C01D80114966D937D9374
:109AC0008D939C93179720911A1430911B144091F9
:109AD0001C1450911D14F601608171818281938163
:109AE0000E947FEC0E9462F26B017C01D801189603
:109AF0006D937D938D939C931B9720911E143091B1
:109B00001F144091201450912114F1016081718142
:109B1000828193810E947FEC0E9462F2D8011C96A0
:109B20006D937D938D939C931F9769837A838B8329
:109B30009C830E948F442FB7F894E2EFF3E14082B8
:109B400051826282738284829582A682B782C086A5
:109B5000D186E286F38669817A818B819C816487D4
:109B60007587868797872FBF1092230E1092240E39
:109B70001092250E1092260E80E1E7E2FEE0DF0152
:109B80001D928A95E9F70F900F900F900F90DF913B
:109B9000CF911F910F91FF90EF90DF90CF90BF90EA
:109BA000AF909F908F907F906F905F904F903F907D
:109BB0002F9008950F931F93CF93DF93C2E1D4E1C9
:109BC0000BE814E0299139914991599160E070E0D6
:109BD00080E89FE30E940DF1F801619371938193F6
:109BE00091938F01F4E1C232DF0761F72EE034E197
:109BF0004AE054E166E074E182E094E118DFDF912D
:109C0000CF911F910F91A9CE4F925F926F927F9249
:109C1000AF92BF92CF92DF92EF92FF920F931F937A
:109C2000CF93DF93009709F456C0FC01208121FDFA
:109C300052C0EB018C0147A050A461A472A4AFA054
:109C4000B8A4C9A4DAA49501A601C301B2010E9477
:109C50001AEC87FF40C0A3019201C301B2010E9428
:109C60007FEC2B013C01F80183A994A9A5A9B6A911
:109C7000BC01CD0190589B01AC010E9431F0F8016C
:109C800027A530A941A952A90E947FEC9B01AC01F4
:109C9000C301B2010E9430F00E949CF27B018C0152
:109CA0009B01AC01B501C6010E941AEC87FF02C0FE
:109CB000750186019701A801B501C6010E941AEC41
:109CC000882349F0A701B8014FA358A769A77AA72D
:109CD000888181608883DF91CF911F910F91FF90E0
:109CE000EF90DF90CF90BF90AF907F906F905F909C
:109CF0004F9008952F923F924F925F926F927F9272
:109D00008F929F92AF92BF92CF92DF92EF92FF928B
:109D10000F931F93CF93DF93CDB7DEB768970FB63E
:109D2000F894DEBF0FBECDBF1C015B018A01DC01D0
:109D3000D7966D917D918D919C91DA970E941EEC42
:109D40006B017C01F50120813181428153810E94A8
:109D50007FEC0E94F7F00E947AF169877A878B87FF
:109D60009C87D8012D913D914D915C91C701B60121
:109D70000E947FEC0E94F7F00E947AF16D877E8747
:109D80008F87988B29853A854B855C8528373105E7
:109D90004105510540F488E790E0A0E0B0E08987F4
:109DA0009A87AB87BC872D853E854F855889283794
:109DB00031054105510540F488E790E0A0E0B0E0AE
:109DC0008D879E87AF87B88B91012D5B3F4FD9015F
:109DD0008D919D910D90BC91A02D8D839E83AF831D
:109DE000B887BC01CD010E9420EC69837A838B8304
:109DF0009C8369857A858B859C850E941EEC698B86
:109E00007A8B8B8B9C8B20E030E0A90169817A8171
:109E10008B819C810E941AEC882339F1A70196015D
:109E2000C701B6010E947FEC4B015C0129893A8988
:109E30004B895C89CA01B9010E947FEC9B01AC018E
:109E4000C501B4010E9430F04B015C0129813A81C7
:109E50004B815C81CA01B9010E9431F09B01AC01C8
:109E6000C501B4010E940DF103C060E070E0CB01B8
:109E70000E94F7F00E9475F12B013C016D817E81FB
:109E80008F81988590958095709561957F4F8F4FC4
:109E90009F4F0E9420EC4B015C016D857E858F8574
:109EA00098890E941EEC6D837E838F83988720E0C3
:109EB00030E0A901C501B4010E941AEC882349F1E0
:109EC0002D813E814F815885CA01B9010E947FECE6
:109ED0006D8B7E8B8F8B988FA7019601C701B60182
:109EE0000E947FEC9B01AC016D897E898F89988DE2
:109EF0000E9430F06B017C01A5019401C501B40101
:109F00000E9431F09B01AC01C701B6010E940DF126
:109F100003C060E070E0CB010E94A6F1F1018288ED
:109F20009388A488B58875016401C418D508E6082B
:109F3000F7080E9475F1C61AD70AE80AF90AF7FE6F
:109F40006BC020E030E0A90169817A818B819C811E
:109F50000E941AEC882309F447C029813A814B8179
:109F60005C81CA01B9010E9431F06B017C01C5011D
:109F7000B4010E941EEC9B01AC01C701B6010E9416
:109F80007FEC6B017C0129893A894B895C89CA0184
:109F9000B9010E947FEC9B01AC01C701B6010E9490
:109FA00030F06B017C012D813E814F815885CA01C3
:109FB000B9010E947FEC9B01AC01C701B6010E9470
:109FC00031F06B017C0120E030E040E850E4698131
:109FD0007A818B819C810E947FEC9B01AC01C7013F
:109FE000B6010E940DF103C060E070E0CB010E9459
:109FF000F7F00E9475F12B013C0197FF03C0412C43
:10A00000512C3201481459046A047B0410F02401D5
:10A010003501C12CD12C76018FB7F894D1019C91D8
:10A0200093FD22C0F101468A578A608E718EC40C5E
:10A03000D51CE61CF71C5A96CD92DD92ED92FC924F
:10A040005D9729853A854B855C85DB962D933D93FD
:10A050004D935C93DE97FF962D853E854F855889FD
:10A0600020833183428353838FBF68960FB6F89461
:10A07000DEBF0FBECDBFDF91CF911F910F91FF903B
:10A08000EF90DF90CF90BF90AF909F908F907F9098
:10A090006F905F904F903F902F900895CF92DF92F6
:10A0A000EF92FF920F931F93E091130BF091140B1B
:10A0B000C280D380E480F5801C141D041E041F049C
:10A0C0000CF03FC06091120B60FF3BC01CB160916F
:10A0D0003F0B7091400B15FBAA27A0F9B0E06E7FF3
:10A0E0006A2B7B2B7093400B60933F0BA091D9128E
:10A0F000B091DA12A170BB276A237B23672B09F189
:10A100006091A70461606093A704C090F213D0909F
:10A11000F313E090F413F090F513C0929B04D092E7
:10A120009C04E0929D04F0929E04C288D388E48847
:10A13000F588C0920E0BD0920F0BE092100BF092AC
:10A14000110BC680D780E084F1841C141D041E040A
:10A150001F040CF046C06091120B61FF42C0A09139
:10A16000030160913F0B7091400BA1FB222720F966
:10A1700030E0319521953109262737272270332782
:10A18000262737273093400B20933F0B6091D9123D
:10A190007091DA126270772726233723232B09F177
:10A1A0002091A70422602093A7040091F613109138
:10A1B000F7132091F8133091F91300939F04109333
:10A1C000A0042093A1043093A20402891389248956
:10A1D000358900930E0B10930F0B2093100B3093C7
:10A1E000110B02851385248535851016110612067C
:10A1F00013060CF056C02091120B22FF52C069B119
:10A2000020913F0B3091400B63FB882780F990E051
:10A2100091958195910982279327847099278227A8
:10A2200093279093400B80933F0B29B122FB442747
:10A2300040F950E0519541955109482759274078F8
:10A240005527842795279093400B80933F0B2091AF
:10A25000D9123091DA12822393239C0136952795E7
:10A2600036952795217087FD02C080E001C082E00D
:10A27000282BB9F08091A70484608093A704809173
:10A28000DB12882311F0233061F482899389A48939
:10A29000B58980930E0B90930F0BA093100BB09386
:10A2A000110B80913F0B9091400B9093DA128093A9
:10A2B000D9121F910F91FF90EF90DF90CF900895EA
:10A2C000AF92BF92CF92DF92EF92FF920F931F93C4
:10A2D000CF93C82F882319F0ECEFF4E10CC0E7E826
:10A2E000F8E284918F010F5F1F4F8823A9F30E942A
:10A2F000DC3EF801F6CF84918F010F5F1F4F88235A
:10A3000021F00E94DC3EF801F6CFCC2319F0EFEDEE
:10A31000F4E10CC0E7E8F8E284918F010F5F1F4F72
:10A320008823A9F30E94DC3EF801F6CF84918F01C7
:10A330000F5F1F4F882321F00E94DC3EF801F6CF0B
:10A340008AE00E94DC3EC1112CC0E7E8F8E284916B
:10A350008F010F5F1F4F882321F00E94DC3EF80120
:10A36000F6CFECECF4E184918F010F5F1F4F88234F
:10A3700021F00E94DC3EF801F6CF8091A90B8823E2
:10A3800021F08AE00E94DC3E39C0E1ECF4E18491E6
:10A390008F010F5F1F4F882389F10E94DC3EF80177
:10A3A000F6CF4091A50B5091A60B6091A70B709131
:10A3B000A80B88EB94E19CD98AE00E94DC3E809156
:10A3C000A90B811127C0CC2319F0EDEAF4E10CC0F0
:10A3D000E7E8F8E284918F010F5F1F4F8823A9F30C
:10A3E0000E94DC3EF801F6CF84918F010F5F1F4F72
:10A3F000882381F00E94DC3EF801F6CFE7E8F8E21E
:10A4000084918F010F5F1F4F882359F20E94DC3E19
:10A41000F801F6CFC11124C0E7E8F8E284918F017A
:10A420000F5F1F4F882321F00E94DC3EF801F6CF1A
:10A43000ECE9F4E184918F010F5F1F4F882321F035
:10A440000E94DC3EF801F6CFE7E8F8E284918F0144
:10A450000F5F1F4F882321F00E94DC3EF801F6CFEA
:10A4600040911214509113146091141470911514AA
:10A4700084E994E13DD940911614509117146091EC
:10A4800018147091191481E994E132D940911A1489
:10A4900050911B1460911C1470911D148EE894E16E
:10A4A00027D940911E1450911F146091201470916F
:10A4B00021148BE894E11CD98AE00E94DC3EC11192
:10A4C00024C0E7E8F8E284918F010F5F1F4F8823D3
:10A4D00021F00E94DC3EF801F6CFEDE6F4E1849134
:10A4E0008F010F5F1F4F882321F00E94DC3EF8018F
:10A4F000F6CFE7E8F8E284918F010F5F1F4F8823C2
:10A5000021F00E94DC3EF801F6CF40918512509177
:10A510008612609187127091881284E694E1E8D8DF
:10A520004091891250918A1260918B1270918C1215
:10A5300081E694E1DDD840918D1250918E126091A8
:10A540008F12709190128EE594E1D2D840919112C1
:10A550005091921260919312709194128BE594E154
:10A56000C7D88AE00E94DC3EC11124C0E7E8F8E2C7
:10A5700084918F010F5F1F4F882321F00E94DC3EE2
:10A58000F801F6CFE9E3F4E184918F010F5F1F4FEB
:10A59000882321F00E94DC3EF801F6CFE7E8F8E2DC
:10A5A00084918F010F5F1F4F882321F00E94DC3EB2
:10A5B000F801F6CF40919512509196126091971242
:10A5C0007091981280E394E159D84091991250917A
:10A5D0009A1260919B1270919C128DE294E14ED878
:10A5E00040919D1250919E1260919F127091A01205
:10A5F0008AE294E143D84091A1125091A212609155
:10A60000A3127091A41287E294E138D88AE00E94E4
:10A61000DC3EC11124C0E7E8F8E284918F010F5FAE
:10A620001F4F882321F00E94DC3EF801F6CFEDEDAC
:10A63000F3E184918F010F5F1F4F882321F00E9467
:10A64000DC3EF801F6CFE7E8F8E284918F010F5F76
:10A650001F4F882321F00E94DC3EF801F6CF409185
:10A66000AD125091AE126091AF127091B01284EDA4
:10A6700093E13ED84091A9125091AA126091AB1279
:10A680007091AC1281ED93E133D84091A5125091B5
:10A69000A6126091A7127091A8128EEC93E128D8AF
:10A6A0008AE00E94DC3EC11124C0E7E8F8E2849110
:10A6B0008F010F5F1F4F882321F00E94DC3EF801BD
:10A6C000F6CFEAE5F3E184918F010F5F1F4F8823F6
:10A6D00021F00E94DC3EF801F6CFE7E8F8E2849131
:10A6E0008F010F5F1F4F882321F00E94DC3EF8018D
:10A6F000F6CF409181125091821260918312709135
:10A70000841281E593E10E94784B40917D12509133
:10A710007E1260917F12709180128EE493E10E940C
:10A72000784B4091C4125091C5126091C61270913D
:10A73000C7128BE493E10E943E4B4091B1125091BD
:10A74000B2126091B3127091B41288E493E10E9446
:10A75000784B4091B5125091B6126091B71270913A
:10A76000B81285E493E10E94784B4091B912509160
:10A77000BA126091BB127091BC1282E493E10E9404
:10A78000784B4091BD125091BE126091BF127091F2
:10A79000C0128FE393E10E94784B8AE00E94DC3E76
:10A7A000C11124C0E7E8F8E284918F010F5F1F4FC9
:10A7B000882321F00E94DC3EF801F6CFE1E3F3E1CB
:10A7C00084918F010F5F1F4F882321F00E94DC3E90
:10A7D000F801F6CFE7E8F8E284918F010F5F1F4F91
:10A7E000882321F00E94DC3EF801F6CF40917B04E3
:10A7F00050917C0460917D0470917E0488E293E125
:10A800000E94784B40917F045091800460918104B4
:10A810007091820485E293E10E94784B4091830419
:10A8200050918404609185047091860482E293E1E2
:10A830000E94784B8AE00E94DC3EC11124C0E7E808
:10A84000F8E284918F010F5F1F4F882321F00E944F
:10A85000DC3EF801F6CFEAE0F3E184918F010F5F6F
:10A860001F4F882321F00E94DC3EF801F6CFE7E875
:10A87000F8E284918F010F5F1F4F882321F00E941F
:10A88000DC3EF801F6CF40913B0B50913C0B6091C0
:10A890003D0B70913E0B81E093E10E94784B8AE082
:10A8A0000E94DC3ECC2379F08DE5A82E8BE0B82EFB
:10A8B00097E3C92E9BE0D92E21E6E22E2BE0F22E63
:10A8C00000E010E024C0E7E8F8E284918F010F5F18
:10A8D0001F4F882321F00E94DC3EF801F6CFE4EE02
:10A8E000F2E184918F010F5F1F4F882321F00E94B6
:10A8F000DC3EF801F6CFE7E8F8E284918F010F5FC4
:10A900001F4F882389F20E94DC3EF801F6CFB80180
:10A910008BED92E10E94954BF501619171915F0180
:10A9200088ED92E10E94954BF601619171916F0162
:10A9300085ED92E10E94954BF701619171917F0144
:10A9400082ED92E10E94954B8AE00E94DC3E01304C
:10A95000110519F001E010E0DACFC11124C0E7E8D9
:10A96000F8E284918F010F5F1F4F882321F00E942E
:10A97000DC3EF801F6CFE3ECF2E184918F010F5F4A
:10A980001F4F882321F00E94DC3EF801F6CFE7E854
:10A99000F8E284918F010F5F1F4F882321F00E94FE
:10A9A000DC3EF801F6CF40914C0B50914D0B60917D
:10A9B0004E0B70914F0B8AEB92E10E94784B2CEA80
:10A9C00035EC47E25EE36091540B7091550B80913A
:10A9D000560B9091570B0E940DF1AB01BC0187EB18
:10A9E00092E10E945B4B2CEA35EC47E25EE360911A
:10A9F000500B7091510B8091520B9091530B0E9410
:10AA00007FECAB01BC0184EB92E10E945B4B8AE0DE
:10AA1000CF911F910F91FF90EF90DF90CF90BF905B
:10AA2000AF900C94DC3ECF93DF9322E134E1C5E894
:10AA3000D2E1A5E9B2E180E090E0FC01EC55FD4EE9
:10AA40004591559165917491F901419351936193A9
:10AA500071939F01FC01EC56FD4E45915591659116
:10AA600074914993599369937993FC01EC57FD4E86
:10AA700045915591659174914D935D936D937D933F
:10AA8000049680319105C9F680E090E0A8ECB3E42B
:10AA90008093AD129093AE12A093AF12B093B01208
:10AAA00080E090E0AAE7B4E48093A9129093AA1200
:10AAB000A093AB12B093AC1280E090E0A6E1B4E4B6
:10AAC0008093A5129093A612A093A712B093A812F8
:10AAD000109281121092821210928312109284129C
:10AAE00080E29EE4A0E0B0E08093C4129093C5128F
:10AAF000A093C612B093C71210927D1210927E12CC
:10AB000010927F121092801280E090E0A0EAB0E4F0
:10AB10008093B1129093B212A093B312B093B41277
:10AB20008093B5129093B612A093B712B093B81257
:10AB30008DEC9CECACECBEE38093B9129093BA120E
:10AB4000A093BB12B093BC1280E090E0A0E4B0E40C
:10AB50008093BD129093BE12A093BF12B093C01207
:10AB60008CE0EBE7F4E0DF011D928A95E9F71092A3
:10AB70003B0B10923C0B10923D0B10923E0B8CED58
:10AB800090E090935E0B80935D0B80EF90E090934C
:10AB9000600B80935F0B82E390E09093380B80937F
:10ABA000370B84E690E090933A0B8093390B109228
:10ABB000620B1092610B1092640B1092630B89E28E
:10ABC0009CE5ABEEB1E480934C0B90934D0BA093BE
:10ABD0004E0BB0934F0B84E795EDA7E9BEE380934E
:10ABE000540B9093550BA093560BB093570B80E0EA
:10ABF00091E2A6E3B4E48093500B9093510BA093A1
:10AC0000520BB093530B1092A90B80E090E0A0EE92
:10AC1000BFE38093A50B9093A60BA093A70BB093D3
:10AC2000A80B109277041092360B0E94C86FE7E8C9
:10AC3000F8E28491EF012196882321F00E94DC3E06
:10AC4000FE01F7CFE1E6F2E18491EF01219688233E
:10AC500021F00E94DC3EFE01F7CFDF91CF910895F5
:10AC6000CF92DF92EF92FF920F931F93CF93DF93D8
:10AC700000D01F92CDB7DEB78091D8139091D91331
:10AC8000A091DA13B091DB13B7FF08C01092D8136C
:10AC90001092D9131092DA131092DB138091DC1307
:10ACA0009091DD13A091DE13B091DF134091D81382
:10ACB0005091D9136091DA137091DB1384179507C3
:10ACC000A607B70744F48093D8139093D913A093A1
:10ACD000DA13B093DB1380915B02882379F1409102
:10ACE000D8135091D9136091DA137091DB138091CE
:10ACF000E0139091E113A091E213B091E3136A0184
:10AD00007B01C80ED91EEA1EFB1EC701B6010E94B8
:10AD100020EC20E030E048EC52E40E947FEC6983B4
:10AD20007A838B839C83CE0101960E94DA68BC01F2
:10AD30008091E6139091E7130E9416A68091800BF4
:10AD40001091D513811106C01123D1F180915B02BE
:10AD50008823B1F14091D8135091D9136091DA133F
:10AD60007091DB138091E0139091E113A091E213B5
:10AD7000B091E3136A017B01C80ED91EEA1EFB1EC7
:10AD8000C701B6010E9420EC20E030E048EC52E41C
:10AD90000E947FECE091E413F091E513309721F0ED
:10ADA0006083718382839383112329F0E091D6130A
:10ADB000F091D71319958091800B81110E94D5B81D
:10ADC0000F900F900F900F90DF91CF911F910F91E7
:10ADD000FF90EF90DF90CF900895CF92DF92EF92A7
:10ADE000FF920F931F93CF93DF9300D01F92CDB7A5
:10ADF000DEB78091D8139091D913A091DA13B09156
:10AE0000DB13B7FF08C01092D8131092D913109219
:10AE1000DA131092DB138091DC139091DD13A09173
:10AE2000DE13B091DF134091D8135091D913609184
:10AE3000DA137091DB1384179507A607B70744F45C
:10AE40008093D8139093D913A093DA13B093DB13A4
:10AE500080915B02882379F14091D8135091D913E6
:10AE60006091DA137091DB138091E0139091E113FC
:10AE7000A091E213B091E3136A017B01C80ED91EC1
:10AE8000EA1EFB1EC701B6010E9420EC2FE632E14C
:10AE900043E85AE30E947FEC69837A838B839C8327
:10AEA000CE0101960E94EBDABC018091E6139091ED
:10AEB000E7130E9416A68091800B1091D513811183
:10AEC00006C01123D1F180915B028823B1F140913A
:10AED000D8135091D9136091DA137091DB138091DC
:10AEE000E0139091E113A091E213B091E3136A0192
:10AEF0007B01C80ED91EEA1EFB1EC701B6010E94C7
:10AF000020EC2FE632E143E85AE30E947FECE09127
:10AF1000E413F091E513309721F06083718382830D
:10AF20009383112329F0E091D613F091D71319954B
:10AF30008091800B81110E94D5B88091800B88236D
:10AF400029F0E091D613F091D71319950F900F9037
:10AF50000F900F90DF91CF911F910F91FF90EF9085
:10AF6000DF90CF900895CF92DF92EF92FF920F93F0
:10AF70001F93CF93DF9300D01F92CDB7DEB78091A0
:10AF8000D8139091D913A091DA13B091DB13B7FFC6
:10AF900008C01092D8131092D9131092DA1310929D
:10AFA000DB138091DC139091DD13A091DE13B0913F
:10AFB000DF134091D8135091D9136091DA13709137
:10AFC000DB1384179507A607B70744F48093D813BB
:10AFD0009093D913A093DA13B093DB1380915B02A3
:10AFE000882379F14091D8135091D9136091DA13E5
:10AFF0007091DB138091E0139091E113A091E21323
:10B00000B091E3136A017B01C80ED91EEA1EFB1E34
:10B01000C701B6010E9420EC2AE037ED43E25CE371
:10B020000E947FEC69837A838B839C83CE01019697
:10B030000E948B6ABC018091E6139091E7130E94F5
:10B0400016A68091800B1091D513811106C0112393
:10B05000D1F180915B028823B1F14091D8135091D6
:10B06000D9136091DA137091DB138091E013909102
:10B07000E113A091E213B091E3136A017B01C80EC2
:10B08000D91EEA1EFB1EC701B6010E9420EC2AE071
:10B0900037ED43E25CE30E947FECE091E413F09132
:10B0A000E513309721F060837183828393831123AA
:10B0B00029F0E091D613F091D71319958091800B68
:10B0C00081110E94D5B80F900F900F900F90DF91D3
:10B0D000CF911F910F91FF90EF90DF90CF90089547
:10B0E0000F931F93CF938091D8139091D913A09170
:10B0F000DA13B091DB13B7FF08C01092D813109287
:10B10000D9131092DA131092DB138091DC13909113
:10B11000DD13A091DE13B091DF134091D81350914D
:10B12000D9136091DA137091DB1384179507A60782
:10B13000B70744F48093D8139093D913A093DA13EC
:10B14000B093DB1380915B02882331F14091D813D7
:10B150005091D9136091DA137091DB138091E01351
:10B160009091E113A091E213B091E3138A019B0146
:10B17000080F191F2A1F3B1FC901B8010E9420ECAC
:10B180000E9475F1CB010E94706BBC018091E613A7
:10B190009091E7130E9416A68091800BC091D51361
:10B1A000811106C0CC23C1F180915B028823A1F1FB
:10B1B0004091D8135091D9136091DA137091DB1339
:10B1C0008091E0139091E113A091E213B091E31309
:10B1D0008A019B01080F191F2A1F3B1FC901B801D3
:10B1E0000E9420ECE091E413F091E513309721F0F8
:10B1F0006083718382839383CC2329F0E091D613FB
:10B20000F091D71319958091800B882329F0CF9165
:10B210001F910F910C94D5B8CF911F910F91089564
:10B220008091D8139091D913A091DA13B091DB13C8
:10B23000B7FF08C01092D8131092D9131092DA13E6
:10B240001092DB138091DC139091DD13A091DE133B
:10B25000B091DF134091D8135091D9136091DA1354
:10B260007091DB1384179507A607B70744F4809302
:10B27000D8139093D913A093DA13B093DB13809172
:10B280005B02882399F02091E0133091E1138091C3
:10B29000D8139091D913820F931F0E94706BBC0139
:10B2A0008091E6139091E7130E9416A68091800B7F
:10B2B0002091D513811106C0222311F180915B02E8
:10B2C0008823F1F04091E0135091E1138091D8135D
:10B2D0009091D913840F951FE091E413F091E51339
:10B2E000309711F091838083222329F0E091D613C7
:10B2F000F091D71319958091800B81110E94D5B8D8
:10B300008091800B08958CCF8BDF882329F0E0910A
:10B31000D613F091D713199408951F93CF93DF9309
:10B3200010927E0B8091D8139091D913A091DA13CB
:10B33000B091DB1381309048A105B10540F0109227
:10B34000D8131092D9131092DA131092DB13C09114
:10B35000D8138091440B18160CF5282F082E000CDA
:10B36000330B255031094C2F0C2E000C550B421776
:10B370005307A4F085301CF0CBEFC80F01C0C0E02C
:10B380008C2F0C2E000C990BAA0BBB0B8093D8139F
:10B390009093D913A093DA13B093DB13C093410BAE
:10B3A000D0E012E0C11109C080915B028823D9F17D
:10B3B00021E041E065E475E115C0C13049F48091B8
:10B3C0005B02882381F120E041E066E375E10AC079
:10B3D000C23061F480915B02882329F120E041E0D2
:10B3E00066E275E18D2F0E94E7E51DC0C33049F488
:10B3F00080915B028823B9F020E041E06FE175E1C4
:10B40000F1CFC43081F480915B02882351F021E0B8
:10B4100040E064E175E18D2F0E94E7E58D2F0E94E9
:10B4200077E510935B02DF5FCF5FD53009F0BACFCD
:10B43000D093440BDF91CF911F9108951F93CF9329
:10B44000DF9310927E0B8091D8139091D913A09125
:10B45000DA13B091DB1381309048A105B10540F0BB
:10B460001092D8131092D9131092DA131092DB13A2
:10B47000C091D8138091450B18160CF5282F082E73
:10B48000000C330B255031094C2F0C2E000C550BA2
:10B4900042175307A4F085301CF0CBEFC80F01C052
:10B4A000C0E08C2F0C2E000C990BAA0BBB0B8093C9
:10B4B000D8139093D913A093DA13B093DB13C093EE
:10B4C000410BD0E012E0C11109C080915B028823DA
:10B4D000D9F121E041E068E775E115C0C13049F4D8
:10B4E00080915B02882381F120E041E06FE675E105
:10B4F0000AC0C23061F480915B02882329F120E008
:10B5000041E06FE575E18D2F0E94E7E51DC0C33076
:10B5100049F480915B028823B9F020E041E06DE5B9
:10B5200075E1F1CFC43081F480915B02882351F042
:10B5300021E040E062E575E18D2F0E94E7E58D2F67
:10B540000E9477E510935B02DF5FCF5FD53009F093
:10B55000BACFD093450BDF91CF911F9108951F93E0
:10B56000CF93DF9310927E0B8091D8139091D913D3
:10B57000A091DA13B091DB1381309048A105B10599
:10B5800040F01092D8131092D9131092DA1310923F
:10B59000DB13C091D8138091480B18160CF5282F97
:10B5A000082E000C330B255031094C2F0C2E000CAB
:10B5B000550B42175307A4F085301CF0CBEFC80F92
:10B5C00001C0C0E08C2F0C2E000C990BAA0BBB0BFA
:10B5D0008093D8139093D913A093DA13B093DB130D
:10B5E000C093410BD0E012E0C11109C080915B0211
:10B5F0008823D9F121E041E06FE276E115C0C13046
:10B6000049F480915B02882381F120E041E06FE101
:10B6100076E10AC0C23061F480915B02882329F18F
:10B6200020E041E06EE076E18D2F0E94E7E51DC04D
:10B63000C33049F480915B028823B9F020E041E0F7
:10B640006FEF75E1F1CFC43081F480915B02882304
:10B6500051F021E040E064EF75E18D2F0E94E7E5B5
:10B660008D2F0E9477E510935B02DF5FCF5FD530AF
:10B6700009F0BACFD093480BDF91CF911F91089575
:10B680001F93CF93DF9310927E0B8091D8139091EC
:10B69000D913A091DA13B091DB1381309048A10542
:10B6A000B10540F01092D8131092D9131092DA130A
:10B6B0001092DB13C091D8138091490B18160CF52A
:10B6C000282F082E000C330B255031094C2F0C2E3F
:10B6D000000C550B42175307A4F085301CF0CBEF3C
:10B6E000C80F01C0C0E08C2F0C2E000C990BAA0BC8
:10B6F000BB0B8093D8139093D913A093DA13B09314
:10B70000DB13C093410BD0E012E0C11109C080915E
:10B710005B028823D9F121E041E060E676E115C0C3
:10B72000C13049F480915B02882381F120E041E03F
:10B7300067E576E10AC0C23061F480915B0288233C
:10B7400029F120E041E069E476E18D2F0E94E7E5F0
:10B750001DC0C33049F480915B028823B9F020E01A
:10B7600041E067E476E1F1CFC43081F480915B027F
:10B77000882351F021E040E06CE376E18D2F0E94B8
:10B78000E7E58D2F0E9477E510935B02DF5FCF5FC7
:10B79000D53009F0BACFD093490BDF91CF911F91EB
:10B7A00008951F93CF93DF9310927E0B8091D8134F
:10B7B0009091D913A091DA13B091DB1381309048A6
:10B7C000A105B10540F01092D8131092D913109230
:10B7D000DA131092DB13C091D81380914A0B18161C
:10B7E0000CF5282F082E000C330B255031094C2F57
:10B7F0000C2E000C550B42175307A4F085301CF09B
:10B80000CBEFC80F01C0C0E08C2F0C2E000C990BA1
:10B81000AA0BBB0B8093D8139093D913A093DA1380
:10B82000B093DB13C093410BD0E012E0C11109C00B
:10B8300080915B028823D9F121E041E064E976E15F
:10B8400015C0C13049F480915B02882381F120E06A
:10B8500041E06BE876E10AC0C23061F480915B029E
:10B86000882329F120E041E06AE776E18D2F0E94EC
:10B87000E7E51DC0C33049F480915B028823B9F02D
:10B8800020E041E068E776E1F1CFC43081F48091B7
:10B890005B02882351F021E040E06DE676E18D2FD8
:10B8A0000E94E7E58D2F0E9477E510935B02DF5F32
:10B8B000CF5FD53009F0BACFD0934A0BDF91CF914B
:10B8C0001F9108951F93CF93DF9310927E0B809169
:10B8D000D8139091D913A091DA13B091DB13813072
:10B8E0009048A105B10540F01092D8131092D913D9
:10B8F0001092DA131092DB13C091D8138091470B8A
:10B9000018160CF5282F082E000C330B2550310982
:10B910004C2F0C2E000C550B42175307A4F085300A
:10B920001CF0CBEFC80F01C0C0E08C2F0C2E000C18
:10B93000990BAA0BBB0B8093D8139093D913A093A8
:10B94000DA13B093DB13C093410BD0E012E0C111C6
:10B9500009C080915B028823D9F121E041E067EEC4
:10B9600075E115C0C13049F480915B02882381F1F3
:10B9700020E041E067ED75E10AC0C23061F48091DA
:10B980005B02882329F120E041E06AEC75E18D2F0C
:10B990000E94E7E51DC0C33049F480915B02882313
:10B9A000B9F020E041E068EC75E1F1CFC43081F4FA
:10B9B00080915B02882351F021E040E06DEB75E15E
:10B9C0008D2F0E94E7E58D2F0E9477E510935B0293
:10B9D000DF5FCF5FD53009F0BACFD093470BDF914F
:10B9E000CF911F9108951F93CF93DF9310927E0BF9
:10B9F0008091D8139091D913A091DA13B091DB13F1
:10BA000081309048A105B10540F01092D8131092F2
:10BA1000D9131092DA131092DB13C091D8138091CE
:10BA2000460B18160CF5282F082E000C330B25504A
:10BA300031094C2F0C2E000C550B42175307A4F064
:10BA400085301CF0CBEFC80F01C0C0E08C2F0C2E4E
:10BA5000000C990BAA0BBB0B8093D8139093D913AE
:10BA6000A093DA13B093DB13C093410BD0E012E044
:10BA7000C11109C080915B028823D9F121E041E026
:10BA800060EB75E115C0C13049F480915B028823F9
:10BA900081F120E041E061EA75E10AC0C23061F461
:10BAA00080915B02882329F120E041E062E975E1A1
:10BAB0008D2F0E94E7E51DC0C33049F480915B02E1
:10BAC0008823B9F020E041E060E975E1F1CFC430AE
:10BAD00081F480915B02882351F021E040E065E829
:10BAE00075E18D2F0E94E7E58D2F0E9477E5109379
:10BAF0005B02DF5FCF5FD53009F0BACFD093460B42
:10BB0000DF91CF911F910895CF93DF9310927E0B19
:10BB10008091D8139091D913A091DA13B091DB13CF
:10BB200081309048A105B10540F01092D8131092D1
:10BB3000D9131092DA131092DB13C091D8138091AD
:10BB40004B0B18160CF5282F082E000C330B255024
:10BB500031094C2F0C2E000C550B42175307A4F043
:10BB600085301CF0CBEFC80F01C0C0E08C2F0C2E2D
:10BB7000000C990BAA0BBB0B8093D8139093D9138D
:10BB8000A093DA13B093DB13C093410BD0E0C11143
:10BB900009C080915B028823E9F021E041E06AEB73
:10BBA00076E115C0C13049F480915B02882391F0A1
:10BBB00020E041E06BEA76E10AC0C23059F480919E
:10BBC0005B02882339F020E041E061EA76E18D2FC5
:10BBD0000E94E7E5DF5FCF5FD530C9F683E0809351
:10BBE0004B0BDF91CF910895CF92DF92EF92FF92AE
:10BBF0000F931F93CF93DF9300D01F92CDB7DEB783
:10BC00008091D8139091D913A091DA13B091DB13DE
:10BC1000B7FF08C01092D8131092D9131092DA13FC
:10BC20001092DB138091DC139091DD13A091DE1351
:10BC3000B091DF134091D8135091D9136091DA136A
:10BC40007091DB1384179507A607B70744F4809318
:10BC5000D8139093D913A093DA13B093DB13809188
:10BC60005B02882379F14091D8135091D9136091E8
:10BC7000DA137091DB138091E0139091E113A0919E
:10BC8000E213B091E3136A017B01C80ED91EEA1ECC
:10BC9000FB1EC701B6010E9420EC2AE037ED43E20B
:10BCA0005CE30E947FEC69837A838B839C83CE0163
:10BCB00001960E945968BC018091E6139091E713A8
:10BCC0000E9416A68091800B1091D513811106C099
:10BCD0001123D1F180915B028823B1F14091D813F7
:10BCE0005091D9136091DA137091DB138091E013B6
:10BCF0009091E113A091E213B091E3136A017B01EB
:10BD0000C80ED91EEA1EFB1EC701B6010E9420EC18
:10BD10002AE037ED43E25CE30E947FECE091E4131C
:10BD2000F091E513309721F06083718382839383D0
:10BD3000112329F0E091D613F091D7131995809132
:10BD4000800B81110E94D5B88091800B0F900F90CD
:10BD50000F900F90DF91CF911F910F91FF90EF9077
:10BD6000DF90CF9008958A30910508F05FC0FC0104
:10BD70008827EE58FF4F8F4F0C9438F381E0809363
:10BD8000790B40E050E0BA018DE899E508C081E008
:10BD90008093790B40E050E0BA018EE19AE50C9473
:10BDA0000EB481E08093790B40E050E0BA018FEA55
:10BDB0009AE5F5CF81E08093790B40E050E0BA013D
:10BDC00080E49BE5ECCF81E08093790B40E050E08C
:10BDD000BA0181ED9BE5E3CF81E08093790B40E0F0
:10BDE00050E0BA0182E69CE5DACF81E08093790BDE
:10BDF00040E050E0BA0183EF9CE5D1CF81E0809331
:10BE0000790B1092430B1092420B40E050E0BA01C4
:10BE100085E09AE8C4CF81E08093790B40E050E060
:10BE2000BA0184E89DE5BBCF0C94CFB808952CEA05
:10BE300035EC47E25EE36091670B7091680B80918F
:10BE4000690B90916A0B0E940DF16093500B7093F7
:10BE5000510B8093520B9093530B08952CEA35ECC1
:10BE600047E25EE360916B0B70916C0B80916D0B00
:10BE700090916E0B0E947FEC6093540B7093550B66
:10BE80008093560B9093570B08952F923F924F92A9
:10BE90005F926F927F928F929F92AF92BF92DF924A
:10BEA000EF92FF920F931F93CF93DF9310927E0B2D
:10BEB0008091D8139091D913A091DA13B091DB132C
:10BEC00081309048A105B10540F01092D81310922E
:10BED000D9131092DA131092DB13C091D81380910A
:10BEE0006F0B1816DCF4282F082E000C330B215092
:10BEF00031094C2F0C2E000C550B4217530774F0D0
:10BF0000CFEFC80F8C2F90E0A0E0B0E08093D81363
:10BF10009093D913A093DA13B093DB131092AA0B6A
:10BF20008091410BC81714F4C093410B8091410BD1
:10BF3000082E000C990B04962C2F0C2E000C330BA2
:10BF40008217930724F48CEF8C0F8093410BD090D1
:10BF5000410BD0E05EED252E57E1352E66E9862EA9
:10BF6000912CA12CB12C7EE6472E512C612C712CEA
:10BF7000D1101DC08091800B811106C080915B02A1
:10BF8000882309F4D6C109C0C111F8CF0E94D5B8E1
:10BF90008091AA0B882391F364C381E0C11180E0F2
:10BFA00024E04FE158E16D2F0E94DA6BC2C181E0BD
:10BFB000D8126EC08091800B811106C080915B0207
:10BFC000882309F4B6C155C0C130C1F7C0937E0BB8
:10BFD00010927A0B10927B0B10927C0B10927D0BBF
:10BFE0000E94EEB383E080935B0288E198E1909336
:10BFF000E7138093E6138BE59BE09093E513809322
:10C00000E4131092E0131092E1131092E2131092D5
:10C01000E31384E091E0A0E0B0E08093DC13909320
:10C02000DD13A093DE13B093DF1380915B0B90912F
:10C030005C0B092E000CAA0BBB0B8093D8139093BA
:10C04000D913A093DA13B093DB1384E899E59093A6
:10C050005A028093590285E691E99093D713809311
:10C06000D6131092D5138091AA0B882309F4A6CF7A
:10C07000F8C280915B0B90915C0B0E94706B9C01ED
:10C0800081E0C13009F080E000E041E158E14EC1BB
:10C0900092E0D91235C08091800B811106C0809149
:10C0A0005B02882309F445C11CC0C230C1F781E09E
:10C0B00080937E0B10927A0B10927B0B10927C0B6C
:10C0C00010927D0B2FEF30E040E050E069E57BE01F
:10C0D00087E098E10E94ADE28091AA0B8823F9F2F3
:10C0E000C0C28091590B90915A0B0E94706B9C01B9
:10C0F00081E0C23009F080E000E04DEF57E116C169
:10C10000A3E0DA1229C08091800B811105C08091D3
:10C110005B02811110C00DC1C330C9F79091580B5B
:10C1200081E089278093580BC0935B028091AA0B12
:10C13000882369F396C28091580B811103C02CEEBD
:10C1400037E102C020EF37E181E0C33009F080E041
:10C1500001E044EF57E1EAC0B4E0DB123FC0809158
:10C16000800B811106C080915B02882309F4E1C035
:10C1700014C0C430C1F7E12CF12C02E813E420E034
:10C1800030E0A90164E272E085EE97E10E9436E2B8
:10C190008091AA0B882339F364C281E08F9384E0F5
:10C1A0008F931F921F9284E292E09F938F93A7ED4B
:10C1B000B7E1BF93AF933F922F92DF9381E0C430FA
:10C1C00009F080E08F930E945CE58DB79EB70C96D6
:10C1D0000FB6F8949EBF0FBE8DBFABC095E0D912CD
:10C1E00041C08091800B811106C080915B02882341
:10C1F00009F49FC014C0C530C1F7E12CF12C02E84E
:10C2000013E420E030E0A90160E272E080ED97E104
:10C210000E9436E28091AA0B882339F322C281E082
:10C220008F9384E08F931F921F9280E292E09F93FE
:10C230008F93A2ECB7E1BF93AF93A9ECB7E1BF93A3
:10C24000AF93DF9381E0C53009F080E08F930E94C7
:10C250005CE58DB79EB70C960FB6F8949EBF0FBEE7
:10C260008DBF67C096E0D91264C08091800B8111A8
:10C2700006C080915B02882309F45BC04BC0C630C6
:10C28000C1F70E94EEB383E080935B02AAEBB7E1B3
:10C29000B093E713A093E6138CE192E09093E5133B
:10C2A0008093E4131092E0131092E1131092E213C2
:10C2B0001092E31384E690E0A0E0B0E08093DC13FA
:10C2C0009093DD13A093DE13B093DF1320E030E0F2
:10C2D00048EC52E460911C0270911D0280911E0294
:10C2E00090911F020E947FEC0E947AF16093D81314
:10C2F0007093D9138093DA139093DB13A3EBB7E514
:10C30000B0935A02A09359028091AA0B882309F492
:10C31000B0CFA7C18CE192E00E948B6A9C0181E0C2
:10C32000C63009F080E000E042EB57E16D2F0E943B
:10C33000ECE42CEA35EC47E25EE36091540B70913B
:10C34000550B8091560B9091570B0E940DF1609305
:10C350006B0B70936C0B80936D0B90936E0B2CEAB0
:10C3600035EC47E25EE36091500B7091510B809188
:10C37000520B9091530B0E947FEC6093670B70936C
:10C38000680B8093690B90936A0BB7E0DB1232C0A5
:10C390008091800B811106C080915B02882309F493
:10C3A00058C11CC0C730C1F7E12C18E1F12E0CE1D7
:10C3B00016E420E030E040E85FE36CE47BE08CEAE8
:10C3C00097E10E9418E384E996E690935A028093DD
:10C3D00059028091AA0B8823F9F243C18CE49BE0B7
:10C3E00068D69C0181E0C73009F080E000E046EAB1
:10C3F00057E179C028E0D2123AC08091800B8111B8
:10C4000006C080915B02882309F423C124C0C83090
:10C41000C1F7E12C18E1F12E0CE116E42AE037ED2A
:10C4200043E25CE36BE67BE080EA97E10E9418E37D
:10C430008AE896E690935A02809359028EE29FE52D
:10C440009093D7138093D6131092D5138091AA0B93
:10C450008823B9F206C18BE69BE02BD69C0181E0D4
:10C46000C83009F080E000E04AE957E13CC089E0CB
:10C47000D8123DC08091800B811106C080915B0273
:10C48000882309F4E6C024C0C930C1F7E12C18E1C3
:10C49000F12E0CE116E420E030E040E85FE367E6CF
:10C4A0007BE084E997E10E9418E38AE896E690939E
:10C4B0005A028093590287E19FE59093D7138093A6
:10C4C000D6131092D5138091AA0B8823B9F2C9C054
:10C4D00087E69BE0EED59C0181E0C93009F080E061
:10C4E00000E04EE857E16D2F0E94ECE4B2C09AE004
:10C4F000D9126FC08091800B811106C080915B02C0
:10C50000882309F4A6C056C0CA30C1F781E08093E1
:10C510007E0B10927A0B10927B0B10927C0B109278
:10C520007D0B0E94EEB383E080935B0281E897E18C
:10C530009093E7138093E6138AE192E09093E513DA
:10C540008093E4138092E0139092E113A092E2139F
:10C55000B092E3134092DC135092DD136092DE132D
:10C560007092DF1380911A0290911B02092E000C29
:10C57000AA0BBB0B86599109A109B1098093D81365
:10C580009093D913A093DA13B093DB1384E899E561
:10C5900090935A028093590283E493E69093D713C1
:10C5A0008093D6131092D5138091AA0B882309F497
:10C5B000A5CF57C080911A0290911B020E94706B08
:10C5C0009C0181E0CA3009F080E000E044E757E1D7
:10C5D0008ACFABE0DA121CC08091800B811105C0BC
:10C5E00080915B028823A9F10BC0CB30C9F788ED9D
:10C5F0009EEB0E9403E38091AA0B882389F331C04C
:10C6000081E0CB3009F080E023E043E657E11EC033
:10C61000BCE0DB121EC08091800B811105C08091AF
:10C620005B028823B1F00BC0CC30C9F785ED9EEBDF
:10C630000E9403E38091AA0B882389F312C081E052
:10C64000CC3009F080E023E042E557E16D2F0E94F5
:10C65000DA6BDF5FD394D53009F08ACC8DE080931C
:10C660006F0BDF91CF911F910F91FF90EF90DF90B3
:10C67000BF90AF909F908F907F906F905F904F9002
:10C680003F902F9008950F931F93CF93DF93CDB7D3
:10C69000DEB76E970FB6F894DEBF0FBECDBF8091A8
:10C6A0001B028F9380911A028F931F921F9282E434
:10C6B00097E19F938F938E010F5F1F4F1F930F93EF
:10C6C0000E94B3EBC8010E94E59D0FB6F894DEBF4F
:10C6D0000FBECDBF6E960FB6F894DEBF0FBECDBFB6
:10C6E000DF91CF911F910F9108951F93CF93DF9307
:10C6F00010927E0B8091D8139091D913A091DA13E8
:10C70000B091DB1381309048A105B10540F0109243
:10C71000D8131092D9131092DA131092DB13C09130
:10C72000D8138091660B1816DCF4282F082E000C05
:10C73000330B215031094C2F0C2E000C550B421796
:10C74000530774F0CFEFC80F8C2F90E0A0E0B0E05B
:10C750008093D8139093D913A093DA13B093DB137B
:10C760001092AA0B8091410BC81714F4C093410B8F
:10C770008091410B082E000C990B04962C2F0C2E47
:10C78000000C330B8217930724F48CEF8C0F8093EB
:10C79000410B1091410BD0E011111AC08091800B18
:10C7A000811106C080915B02882309F4F0C009C0A2
:10C7B000C111F8CF0E94D5B88091AA0B882391F3BC
:10C7C000EEC081E0C11180E024E04DE357E1DDC01F
:10C7D0001130E9F48091800B811106C080915B02D9
:10C7E000882309F4D4C00BC0C130C1F785E49FE5AC
:10C7F0000E9403E38091AA0B882381F3D0C081E0DB
:10C80000C13009F080E023E041E357E1BEC01230BF
:10C81000E9F48091800B811106C080915B0288232E
:10C8200009F4B5C00BC0C230C1F783E29FE80E9493
:10C8300003E38091AA0B882381F3B1C081E0C23069
:10C8400009F080E023E04AE257E19FC01330E9F4A9
:10C850008091800B811106C080915B02882309F4CE
:10C8600096C00BC0C330C1F78FEB9DE80E9403E375
:10C870008091AA0B882381F392C081E0C33009F034
:10C8800080E023E041E257E180C01430D9F4809188
:10C89000800B811106C080915B02882309F477C068
:10C8A00009C0C430C1F70E9424E48091AA0B8823F8
:10C8B00091F375C081E0C43009F080E020E242E1EC
:10C8C00057E163C0153039F58091800B811106C0A6
:10C8D00080915B02882309F45AC015C0C530C1F7A6
:10C8E0000E94D379882311F055D708C048EB51E056
:10C8F00064E170E080E090E00E94A9DD8091AA0BE5
:10C90000882331F34CC081E0C53009F080E020E29B
:10C9100042EF56E13AC01630D9F48091800B811174
:10C9200005C080915B02882391F10AC0C630C9F727
:10C930000E9413552FD78091AA0B882391F32FC003
:10C9400081E0C63009F080E020E241EE56E11DC0F2
:10C950001730E9F48091800B811105C080915B0252
:10C960008823A9F00BC0C730C9F783ED94E60E9475
:10C9700003E38091AA0B882389F311C081E0C730BB
:10C9800009F080E023E040E057E16D2F13D7DF5F2F
:10C990001F5FD53009F000CF88E08093660BDF91F0
:10C9A000CF911F9108951F93CF93DF9310927E0B29
:10C9B0008091D8139091D913A091DA13B091DB1321
:10C9C00081309048A105B10540F01092D813109223
:10C9D000D9131092DA131092DB13C091D8138091FF
:10C9E000650B1816DCF4282F082E000C330B215091
:10C9F00031094C2F0C2E000C550B4217530774F0C5
:10CA0000CFEFC80F8C2F90E0A0E0B0E08093D81358
:10CA10009093D913A093DA13B093DB131092AA0B5F
:10CA20008091410BC81714F4C093410B8091410BC6
:10CA3000082E000C990B04962C2F0C2E000C330B97
:10CA40008217930724F48CEF8C0F8093410B109185
:10CA5000410BD0E08D2F810FC9F48091800B8111A3
:10CA600005C080915B02882399F109C0C111F9CFFB
:10CA70000E94D5B88091AA0B882399F330C081E039
:10CA8000C11180E024E049ED56E120C0813001F57C
:10CA90008091800B811105C080915B028823C1F0D9
:10CAA0000EC0C130C9F70E94135574D60E94697E2A
:10CAB0000E94D5B88091AA0B882371F310C081E041
:10CAC000C13009F080E020E247EC56E16D2F72D6CC
:10CAD000DF5FD53009F0BECF82E08093650BDF9138
:10CAE000CF911F910895CF92DF92EF92FF920F9313
:10CAF0001F93CF93DF9310927E0B4091D8135091E8
:10CB0000D9136091DA137091DB13413050486105FD
:10CB1000710540F01092D8131092D9131092DA13C5
:10CB20001092DB13C091D8139091700B1916DCF49E
:10CB3000292F092E000C330B215031094C2F0C2EBC
:10CB4000000C550B4217530774F0CFEFC90F4C2F51
:10CB500050E060E070E04093D8135093D913609395
:10CB6000DA137093DB131092AA0B9091410BC91743
:10CB700014F4C093410B2091410B022E000C330B97
:10CB80002C5F3F4F4C2F0C2E000C550B24173507F4
:10CB900024F49CEF9C0F9093410B1091410BD0E03B
:10CBA000E82EF12CC701880F991FFC01E35AF44FBE
:10CBB0006F019C012F59344F790111111AC08091D6
:10CBC000800B811106C080915B02882309F483C029
:10CBD00009C0C111F8CF0E94D5B88091AA0B882353
:10CBE00091F381C081E0C11180E024E048E558E183
:10CBF00070C0113039F58091800B811106C0809191
:10CC00005B02882309F467C010C0C130C1F72FEF61
:10CC100030E040E050E0B7018EE498E10E94ADE2E0
:10CC20008091AA0B882359F35EC0F701808191811E
:10CC300057D59C0181E0C13009F080E000E044E478
:10CC400058E128C0123051F58091800B811106C047
:10CC500080915B02882309F43EC010C0C230C1F746
:10CC600024E031E045E050E0B6018DE398E10E9418
:10CC7000ADE28091AA0B882359F335C0F60180817B
:10CC800091812ED59C0181E0C23009F080E000E066
:10CC900046E358E16D2F0E94ECE41DC01330D9F437
:10CCA0008091800B811105C080915B02882399F0EF
:10CCB00009C0C330C9F70E9424E48091AA0B8823DD
:10CCC00099F311C081E0C33009F080E020E247E22F
:10CCD00058E16D2F6FD5DF5F1F5FD53009F06DCF45
:10CCE00084E08093700BDF91CF911F910F91FF90A3
:10CCF000EF90DF90CF900895FC01E60FF11D849135
:10CD000090E0982F88273196E4918E0F911D089519
:10CD100081E008950E94F45D882329F0E091D61304
:10CD2000F091D713199408950C94F45D0B96FC01BF
:10CD3000849108950A96FC018491089568E0DCCFFF
:10CD400066E0DACFFC0184910895FCDF882321F0AE
:10CD5000823011F083E0089586E0089588E290E043
:10CD60000197F1F708952EE93FE0009729F0F901C6
:10CD70003197F1F70197F9CF08950F93FC01015016
:10CD8000040F84A996A9941718F0081728F402C074
:10CD9000081750F0041740F42150260F83A995A9D5
:10CDA000961720F4281720F480E007C0281720F4F5
:10CDB00081E0261710F0F8CF81E00F9108958F924F
:10CDC0009F92AF92BF92CF92DF92EF92FF92CF935A
:10CDD000FC01C080D180E280F38020E030E0A90136
:10CDE000C701B6010E941AEC87FF08C0C701B6014F
:10CDF000905820E030E048EC52E406C020E030E0FB
:10CE000048EC52E4C701B6010E947FEC0E9475F124
:10CE10006B017C01603AF6E87F07F1E08F0791052E
:10CE200084F020EA36E841E050E00E941CF3CA0199
:10CE3000B9012AE030E040E050E00E941CF3605D60
:10CE400001C060E26093EA1380E1C81687E2D80669
:10CE5000E104F10494F0C701B60120E137E240E0BB
:10CE600050E00E941CF3CA01B9012AE030E040E022
:10CE700050E00E941CF3605D01C060E26093EB1320
:10CE8000E8EECE16E3E0DE06E104F10494F0C7011B
:10CE9000B60128EE33E040E050E00E941CF3CA01E6
:10CEA000B9012AE030E040E050E00E941CF3605DF0
:10CEB00001C060E26093EC13C701B60124E630E0E4
:10CEC00040E050E00E941CF38AE0882E912CA12CB7
:10CED000B12CCA01B901A50194010E941CF3605D47
:10CEE0006093ED138EE28093EE13C701B601A501A6
:10CEF00094010E941CF3C62FCA01B901A501940137
:10CF00000E941CF3605D6093EF13C05DC093F0134B
:10CF10008AEE93E1CF91FF90EF90DF90CF90BF909A
:10CF2000AF909F908F900895CF92DF92EF92FF92F3
:10CF30000F931F93CF93DF9300D01F92CDB7DEB72F
:10CF40008091D8139091D913A091DA13B091DB138B
:10CF5000B7FF08C01092D8131092D9131092DA13A9
:10CF60001092DB138091DC139091DD13A091DE13FE
:10CF7000B091DF134091D8135091D9136091DA1317
:10CF80007091DB1384179507A607B70744F48093C5
:10CF9000D8139093D913A093DA13B093DB13809135
:10CFA0005B02882371F14091D8135091D91360919D
:10CFB000DA137091DB138091E0139091E113A0914B
:10CFC000E213B091E3136A017B01C80ED91EEA1E79
:10CFD000FB1EC701B6010E9420EC2AE037ED43E2B8
:10CFE0005CE30E947FEC69837A838B839C83CE0110
:10CFF0000196E5DEBC018091E6139091E7130E9453
:10D0000016A68091800B1091D513811106C01123B3
:10D01000D1F180915B028823B1F14091D8135091F6
:10D02000D9136091DA137091DB138091E013909122
:10D03000E113A091E213B091E3136A017B01C80EE2
:10D04000D91EEA1EFB1EC701B6010E9420EC2AE091
:10D0500037ED43E25CE30E947FECE091E413F09152
:10D06000E513309721F060837183828393831123CA
:10D0700029F0E091D613F091D71319958091800B88
:10D0800081110E94D5B88091800B882329F0E0910E
:10D09000D613F091D71319950F900F900F900F9012
:10D0A000DF91CF911F910F91FF90EF90DF90CF9084
:10D0B00008958F929F92AF92BF92CF92DF92EF929C
:10D0C000FF92CF9320E030E048EC52E4FC01608115
:10D0D0007181828193810E947FEC0E9475F16B01C6
:10D0E0007C0197FF0AC0F094E094D094C094C11CD6
:10D0F000D11CE11CF11C8DE201C08BE28093EA138C
:10D10000C701B60120E137E240E050E00E941CF385
:10D110008AE0882E912CA12CB12CCA01B901A5015D
:10D1200094010E941CF3605D6093EB13C701B6018C
:10D1300028EE33E040E050E00E941CF3CA01B90140
:10D14000A50194010E941CF3605D6093EC13C7017C
:10D15000B60124E630E040E050E00E941CF3CA0132
:10D16000B901A50194010E941CF3605D6093ED1369
:10D170008EE28093EE13C701B601A50194010E94CF
:10D180001CF3C62FCA01B901A50194010E941CF32A
:10D19000605D6093EF13C05DC093F0138AEE93E17E
:10D1A000CF91FF90EF90DF90CF90BF90AF909F9086
:10D1B0008F9008958F929F92AF92BF92CF92DF92FD
:10D1C000EF92FF92FC01C080D180E280F38020E0EA
:10D1D00030E0A901C701B6010E941AEC87FF04C024
:10D1E000C701B601905802C0C701B6010E9475F18F
:10D1F0006B017C016031F7E27F078105910584F0C6
:10D2000020E137E240E050E00E941CF3CA01B9017E
:10D210002AE030E040E050E00E941CF3605D01C075
:10D2200060E26093EC1388EEC81683E0D806E10450
:10D23000F10494F0C701B60128EE33E040E050E07D
:10D240000E941CF3CA01B9012AE030E040E050E03E
:10D250000E941CF3605D01C060E26093ED13E4E6A0
:10D26000CE16D104E104F10494F0C701B60124E61E
:10D2700030E040E050E00E941CF3CA01B9012AE00E
:10D2800030E040E050E00E941CF3605D01C060E2CD
:10D290006093EE13FAE0CF16D104E104F1049CF0A0
:10D2A0008AE0882E912CA12CB12CC701B601A501D2
:10D2B00094010E941CF3CA01B901A50194010E94C6
:10D2C0001CF3605D01C060E26093EF13C701B6011B
:10D2D0002AE030E040E050E00E941CF3605D609383
:10D2E000F0138CEE93E1FF90EF90DF90CF90BF9022
:10D2F000AF909F908F900895CF92DF92EF92FF9220
:10D300000F931F93CF93DF9300D01F92CDB7DEB75B
:10D310008091D8139091D913A091DA13B091DB13B7
:10D32000B7FF08C01092D8131092D9131092DA13D5
:10D330001092DB138091DC139091DD13A091DE132A
:10D34000B091DF134091D8135091D9136091DA1343
:10D350007091DB1384179507A607B70744F48093F1
:10D36000D8139093D913A093DA13B093DB13809161
:10D370005B02882371F14091D8135091D9136091C9
:10D38000DA137091DB138091E0139091E113A09177
:10D39000E213B091E3136A017B01C80ED91EEA1EA5
:10D3A000FB1EC701B6010E941EEC20E030E048ECF5
:10D3B00052E40E947FEC69837A838B839C83CE0145
:10D3C0000196F8DEBC018091E6139091E7130E946C
:10D3D00016A68091800B1091D513811106C01123E0
:10D3E000E1F180915B028823C1F14091D813509103
:10D3F000D9136091DA137091DB138091E01390914F
:10D40000E113A091E213B091E3136A017B01C80E0E
:10D41000D91EEA1EFB1EC701B6010E941EEC20E0C9
:10D4200030E048EC52E40E947FEC0E947AF1E091F7
:10D43000E413F091E513309721F0608371838283C8
:10D440009383112329F0E091D613F091D713199506
:10D450008091800B81110E94D5B88091800B882328
:10D4600029F0E091D613F091D71319950F900F90F2
:10D470000F900F90DF91CF911F910F91FF90EF9040
:10D48000DF90CF90089520E030E040E251E4FC01CD
:10D4900060817181828193810E947FEC0E9475F18D
:10D4A0009B0177FF06C022273327261B370B8DE20F
:10D4B00001C08BE28093EB13C90168EE73E00E9418
:10D4C00009F3CB01EAE0F0E0BF010E9409F3805DBF
:10D4D0008093EC13C90164E670E00E9409F3CB016C
:10D4E000BF010E9409F3805D8093ED13C901BF0164
:10D4F0000E9409F3282FCB01BF010E9409F3805D30
:10D500008093EE138EE28093EF13205D2093F0134F
:10D510008BEE93E108958F929F92AF92BF92CF923C
:10D52000DF92EF92FF92CF9320E030E048EC52E49C
:10D53000FC0160817181828193810E947FEC0E9455
:10D5400075F16B017C0197FD10C020E137E240E0EE
:10D5500050E00E941CF3CA01B9012AE030E040E02B
:10D5600050E00E941CF3605D09C0F094E094D094F8
:10D57000C094C11CD11CE11CF11C6DE26093EB1343
:10D58000C701B60128EE33E040E050E00E941CF3F2
:10D590008AE0882E912CA12CB12CCA01B901A501D9
:10D5A00094010E941CF3605D6093EC13C701B60107
:10D5B00024E630E040E050E00E941CF3CA01B901CB
:10D5C000A50194010E941CF3605D6093ED138EE24F
:10D5D0008093EE13C701B601A50194010E941CF3CC
:10D5E000C62FCA01B901A50194010E941CF3605D18
:10D5F0006093EF13C05DC093F0138BEE93E1CF9176
:10D60000FF90EF90DF90CF90BF90AF909F908F9062
:10D610000895AC01952F991F9927991F29F022276A
:10D620003327241B350B01C09A01483E5340ACF010
:10D63000C90168EE73E00E9409F3CB01EAE0F0E073
:10D64000BF010E9409F3805D8093ED13C90164E678
:10D6500070E00E9409F3CB0112C024363105B4F00A
:10D66000911102C080E201C08DE28093ED13C901E7
:10D6700064E670E00E9409F3CB01EAE0F0E0BF014C
:10D680000E9409F3805D8093EE130EC080E28093C8
:10D69000ED138093EE132A30310584F091118DE261
:10D6A0008093EE13EAE0F0E0C901BF010E9409F3A4
:10D6B000CB01BF010E9409F3805D05C0911102C03A
:10D6C00080E201C08DE28093EF13C9016AE070E04F
:10D6D0000E9409F3805D8093F0138DEE93E108952D
:10D6E0009C0197FD0EC08436910584F064E670E0DD
:10D6F0000E9409F3CB016AE070E00E9409F3805DAB
:10D7000006C03195219531098DE201C080E28093F8
:10D71000EE132A30310564F0EAE0F0E0C901BF0100
:10D720000E9409F3CB01BF010E9409F3805D01C093
:10D7300080E28093EF13C9016AE070E00E9409F370
:10D74000805D8093F0138EEE93E10895CF92DF9287
:10D75000EF92FF926B017C0183E3C816D104E104D0
:10D76000F10470F082E3C81AD108E108F10862E31D
:10D7700070E080E090E00E940D850E941AD0ECCF0E
:10D78000C701B6010E940D85FF90EF90DF90CF900A
:10D790000C941AD043E952E064E670E080E090E037
:10D7A0000E94A9DD4AEB52E064E670E080E090E080
:10D7B0000C94A9DD0F931F93CF93DF93982F862F9F
:10D7C0008A01D22F692F0E941EA590911D0E809173
:10D7D000E913891748F190911F0E8091E81398176B
:10D7E00018F1C4E1F8018491882331F00E94D9A591
:10D7F000C81B0F5F1F4FF6CFCC2329F080E20E9499
:10D80000FE9EC150F9CF8091E9139AE79093200EC4
:10D810008093210E8D2F0E94EDA580E2DF91CF91A4
:10D820001F910F910C94FE9EDF91CF911F910F914C
:10D8300008958FE798E10E94099F81E08093820B11
:10D8400008950F931F930E9445850091970B1091A7
:10D85000980B2091990B30919A0BDC01CB01801B26
:10D86000910BA20BB30BB7FD0CC086B186FB9927B9
:10D8700090F981E08927349B8260329B8460809399
:10D88000960B8091960B81709091960B91FD826022
:10D890009091950B891731F18130A9F028F08230F1
:10D8A00041F0833059F01CC0913089F0923099F0EA
:10D8B00017C0992361F0933071F012C0913059F084
:10D8C000923071F404C0992331F0933049F490916F
:10D8D000940B915003C09091940B9F5F9093940B85
:10D8E0008093950B1F910F910895ECE5F2E080E095
:10D8F0009191992329F0863111F08F5FF9CF089526
:10D90000982F863169F080E2E92F9F5F973129F0E7
:10D91000F0E0E45AFD4F8083F7CF10927202089531
:10D920000895FC0167FF03C01092231460E020916A
:10D93000231430E0462F062E000C550B42175307D8
:10D940007CF06093231442E450E0BF018CE592E048
:10D950000E948AEBCADF83E080935B02109222145C
:10D9600008952091231421110DC0BC0142E450E020
:10D970008CE592E00E94AFF3B8DF83E080935B0216
:10D980001092221408954F925F926F927F928F921D
:10D990009F92AF92BF92CF92DF92EF92FF920F933E
:10D9A0001F93CF93C0912802CF3FF9F00E94458585
:10D9B000C090710BD090720BE090730BF090740BD1
:10D9C000DC01CB018C199D09AE09BF09B7FD0DC063
:10D9D0002091480E8091470E30E090E001968F70C4
:10D9E00099272817390709F00FC22BDF8091960B72
:10D9F00082FF39C08091930B811137C081E0809301
:10DA0000930B9091810B89278093800B1092810B4F
:10DA100083E080935B021092960B0E944585DC01A7
:10DA2000CB018C509E4FAF4FBF4F8093970B90937D
:10DA3000980BA093990BB0939A0B48E853E162E0DE
:10DA400070E080E090E00E94A9DDC6E0C15069F07E
:10DA500089E49EE00E946F3962E070E080E090E02F
:10DA60000E940D85F3CF1092930BC0910901C095D0
:10DA7000C1708091920BC817A1F0CC2309F4E5C1C5
:10DA80000E945D9C8091920B823021F060E081E7E2
:10DA900098E147DFC093920B83E080935B020E9482
:10DAA00079A50E9445856B017C0180918E0B909138
:10DAB0008F0BA091900BB091910BA7019601281BA1
:10DAC000390B4A0B5B0B57FF05C080917F0B8823F6
:10DAD00009F4F6C1D701C6018C599F4FAF4FBF4F14
:10DAE00080938E0B90938F0BA093900BB093910B20
:10DAF0008091940B18162CF48091940B843074F45C
:10DB000008C08091940B992781950CF49095049707
:10DB10002CF48091800B81119FC0AFC080917E0B4F
:10DB2000882309F472C08091940B181664F48091D4
:10DB3000940B082E000C990B97FD039695958795ED
:10DB4000959587950EC08091940B082E000C990B2B
:10DB500097FD0396959587959595879591958195D0
:10DB6000910980907A0B90907B0BA0907C0BB090E9
:10DB70007D0B81149104A104B104D1F1BC01990F72
:10DB8000880B990B0E9420EC2B013C01C701B601C8
:10DB9000681979098A099B090E941EEC9B01AC0156
:10DBA000C301B2010E940DF120E030E04AE754E4E5
:10DBB0000E947FEC4B015C0120E030E040E253E446
:10DBC0000E9457F287FF0FC020E030E046E952E4A0
:10DBD000C501B4010E9457F287FD0AC02AE030E077
:10DBE00040E050E009C024E630E040E050E004C0EE
:10DBF00021E030E040E050E0C0927A0BD0927B0B05
:10DC0000E0927C0BF0927D0B04C021E030E040E01C
:10DC100050E0A091940B0A2E000CBB0B0E9440F325
:10DC200024E030E040E050E00E941CF38091D813E3
:10DC30009091D913A091DA13B091DB13820F931F47
:10DC4000A41FB51F8093D8139093D913A093DA1310
:10DC5000B093DB131092940BD701C6018856954CF4
:10DC6000AF4FBF4F80938A0B90938B0BA0938C0B7D
:10DC7000B0938D0B81E080935B028091590290916B
:10DC80005A028153944B41F480912902882309F46C
:10DC9000E7C08150809329022FB7F8948091750BCB
:10DCA0009091760BA091770BB091780B2FBF3AE053
:10DCB000B695A795979587953A95D1F7009741E046
:10DCC000A407B10520F08FEF9FEFA0E0B0E096959C
:10DCD000879520915B02211105C030917F0B311196
:10DCE000EBC055C0009741F04091880B5091890BD3
:10DCF0004817590708F04BC080917F0B811111C064
:10DD0000223050F0243028F0243031F410925B029D
:10DD100003C081E080935B020E947D9F81E080933D
:10DD20007F0B84E00E9460A581E08093090EE09162
:10DD30005902F0915A0219951092800B80917F0B35
:10DD4000882351F00E94C49E91E0811101C090E0AF
:10DD500090937F0B911194C08090880B9090890BC9
:10DD6000A12CB12C0E944585DC01CB018C199D09A9
:10DD7000AE09BF0988169906AA06BB0640F40E94A0
:10DD800045856C197D097093890B6093880B809190
:10DD9000590290915A028153944B21F08091790B52
:10DDA000882379F088E9C80E8AE3D81EE11CF11CAB
:10DDB000C0928A0BD0928B0BE0928C0BF0928D0B61
:10DDC0000FC080918A0B90918B0BA0918C0BB0911E
:10DDD0008D0BC81AD90AEA0AFB0AF7FE0E94CFB8CF
:10DDE00080917F0B81116CC080915B02813049F082
:10DDF00008F466C0843008F063C081E080935B0261
:10DE00005FC010925B025CC024E0C202F0011124EA
:10DE1000EC55FD4F20E030E040E752E46081718135
:10DE2000828193810E940DF1C12C7B018C012EE037
:10DE300034E14AE054E166E074E182E094E10E945A
:10DE4000DBBE8FEF80932802D0CD1092770E109218
:10DE5000780E823009F41ECE60E084E698E119CE97
:10DE60008CE0809329028091880B9091890B019717
:10DE70009093890B8093880B81E080935B020CCF99
:10DE80008090880B9090890BA12CB12C0E94458525
:10DE9000DC01CB018C199D09AE09BF0988169906D2
:10DEA000AA06BB0668F40E9445856C197D0970932B
:10DEB000890B6093880B04C0009709F432CF14CF0C
:10DEC000CF911F910F91FF90EF90DF90CF90BF9077
:10DED000AF909F908F907F906F905F904F9008953C
:10DEE000CF92DF92EF92FF920F931F930E9445858E
:10DEF0000091840B1091850B2091860B3091870B3C
:10DF00006B017C01C01AD10AE20AF30AF7FC13C0C4
:10DF10002091830B20952093830BDC01CB018A5445
:10DF20009C4FAF4FBF4F8093840B9093850BA09372
:10DF3000860BB093870B81E09091830B911101C008
:10DF400080E01F910F91FF90EF90DF90CF900895A8
:10DF50000E9479A53E98469A3C98449A3A98429AEB
:10DF6000EAE0F1E080818E7F80839FB7F894EBE058
:10DF7000F1E08081816080839FBF82E08093920B7B
:10DF800060DC1092940B0895089580E090E008956D
:10DF90000E94AD4C0E94DA4D0E94F6D080E090E0E5
:10DFA0000E94B73B81E090E00E94B73B82E090E0A6
:10DFB0000C94B73BFC0120E03EE2DB014C91403287
:10DFC00041F0283011F430833196DB014C914083CD
:10DFD00031962F5F6F5F7F4F2B3079F71082089556
:10DFE000FC0114821782138212828CEE92E09183DC
:10DFF00080830895CF938091DD0D8823B9F14091FE
:10E00000D50D5091D60D6091D70D7091D80D25ED9D
:10E010003BE08091DE0D9091DF0D0E9413AFC82F81
:10E02000811102C0C0E023C04091D90D5091DA0D9A
:10E030006091DB0D7091DC0D411551056105710595
:10E0400091F025ED3BE08091DE0D9091DF0D0E9477
:10E0500013AF882339F31092D90D1092DA0D109274
:10E06000DB0D1092DC0D1092DD0D01C0C1E08C2F94
:10E07000CF910895CF92DF92EF92FF92CF936B01F1
:10E080007C01C42F8091D50D9091D60DA091D70D14
:10E09000B091D80D8C159D05AE05BF05C9F0AADF5E
:10E0A000811102C080E018C025ED3BE0B701A60158
:10E0B0008091DE0D9091DF0D0E9475AF882391F362
:10E0C000C092D50DD092D60DE092D70DF092D80D1A
:10E0D00081E0C1118093DD0DCF91FF90EF90DF9033
:10E0E000CF9008954F925F926F927F928F929F92FE
:10E0F000AF92BF92CF92DF92EF92FF920F931F9356
:10E10000CF93DF93EC016A017B0128013901423092
:10E1100051056105710510F480E064C089859A8518
:10E12000AB85BC850196A11DB11D84179507A60777
:10E13000B70790F38F89803149F48D2C9E2CAF2C3A
:10E14000BB248B899C89AD89BE890FC0803221F7A1
:10E150008B889C88AD88BE88DB01CA0157E0B695E4
:10E16000A795979587955A95D1F7880E991EAA1E5F
:10E17000BB1E41E0C501B4017DDF882369F29F89A0
:10E18000903161F4DD24EE24FF249601220F331F29
:10E19000F901EB52F44F5182408211C0E894C7F864
:10E1A000DD24EE24FF249601220F331F220F331F9C
:10E1B000F901EB52F44F40825182628273829A8954
:10E1C000923080F04D815E816F817885840E951E3E
:10E1D000A61EB71E8092D90D9092DA0DA092DB0D8B
:10E1E000B092DC0DDF91CF911F910F91FF90EF90D6
:10E1F000DF90CF90BF90AF909F908F907F906F9067
:10E200005F904F900895CF92DF92EF92FF920F931D
:10E210001F93CF93DF93FC0181859285A385B485FD
:10E220000196A11DB11D84179507A607B70710F425
:10E2300080E061C08789803149F4BB27A72F962FE2
:10E24000852FC388D488E588F6880FC0803281F78F
:10E2500083899489A589B6896A017B01C7E0F69410
:10E26000E794D794C794CA95D1F78C0D9D1DAE1D28
:10E27000BF1DE9016A017B018F014091D50D5091CD
:10E28000D60D6091D70D7091D80D84179507A6070C
:10E29000B70799F4F80187898031B1F4B701A60175
:10E2A000552766277727440F551FFA01EB52F44F85
:10E2B00080819181A0E0B0E019C040E0BC01CD01B7
:10E2C000D9DE8111E7CFB4CFB701A6014F7755272B
:10E2D00066277727440F551F440F551FFA01EB524D
:10E2E000F44F80819181A281B381BF70888399832B
:10E2F000AA83BB8381E0DF91CF911F910F91FF90A3
:10E30000EF90DF90CF9008954F925F926F927F923F
:10E31000AF92BF92CF92DF92EF92FF920F931F9333
:10E32000CF93DF9300D01F92CDB7DEB78C01498326
:10E330005A836B837C835901C12CD12C7601412CEB
:10E3400082E0582E612C712C49815A816B817C812D
:10E350009E012F5F3F4FC80156DF882341F1D30153
:10E36000C201F801058404C0880F991FAA1FBB1FB2
:10E370000A94D2F7C80ED91EEA1EFB1E49815A81A3
:10E380006B817C818789803139F481E0483F5F4F20
:10E390006105710538F4D8CF81E0483F5F4F6F4F7A
:10E3A0007F4090F2F501C082D182E282F3820F9029
:10E3B0000F900F900F90DF91CF911F910F91FF90D1
:10E3C000EF90DF90CF90BF90AF907F906F905F9075
:10E3D0004F900895CF93DF93EC018B81882331F127
:10E3E000898187FF20C061E0CE010E9458ADFC0109
:10E3F000892BE1F08081853EC9F08B81823040F429
:10E4000089899A89AB89BC89848F958FA68FB78FAC
:10E410008D899E89AF89B88D938F828FB58BA48BA0
:10E4200089818F778983DF91CF91E4CD81E08883E3
:10E4300080E0DF91CF9108958F929F92AF92BF922B
:10E44000CF92DF92EF92FF920F931F93CF93DF93C0
:10E45000EC018B81811102C080E076C009891A89A4
:10E460002B893C890417150726073707A8F36A018B
:10E470007B01823029F4C886D986EA86FB860DC0E6
:10E48000C114D104E104F10451F41C821D821E82E6
:10E490001F82188619861A861B8681E055C08884DB
:10E4A0009984AA84BB84E98DFA8D258530E0275FA5
:10E4B0003F4FB501A4014150510961097109022E74
:10E4C00004C076956795579547950A94D2F7D7017A
:10E4D000C6010197A109B10904C0B695A795979502
:10E4E00087952A95D2F784179507A607B70720F0D6
:10E4F00089288A288B2849F44D895E896F89788D0F
:10E500004C835D836E837F8304C0841B950BA60BB5
:10E51000B70B4C015D018E010C5F1F4F81149104FC
:10E52000A104B10409F4A7CF4C815D816E817F8184
:10E530009801898D9A8D67DE91E0891A9108A1086A
:10E54000B1088111EBCF88CFDF91CF911F910F914F
:10E55000FF90EF90DF90CF90BF90AF909F908F9003
:10E5600008952F923F924F925F926F927F928F9277
:10E570009F92AF92BF92CF92DF92EF92FF920F9352
:10E580001F93CF93DF9300D01F92CDB7DEB78C01DE
:10E590004B011A01DC0113968C9113978130C1F461
:10E5A00011968C9181FF14C082FF18C0F801418937
:10E5B00052896389748980859185A285B385841782
:10E5C0009507A607B70751F0C80136DF811106C0CD
:10E5D00081E0F80180838FEF9FEF2CC1610185C03E
:10E5E000D80159968D919C915A97FC012481215014
:10E5F0002A013B0139E076946794579447943A9501
:10E60000D1F7722E74207A01F1E0FF22772009F40D
:10E6100078C080E092E08E199F0956018C159D0507
:10E6200008F45C01D80159962D913C915A971496A3
:10E630008D919D910D90BC91A02D0297A109B109DA
:10E64000F901058404C0880F991FAA1FBB1F0A94F3
:10E65000D2F74685578560897189840F951FA61F5B
:10E66000B71F9C01AD01270D311D411D511D290111
:10E670003A01A11432E0B30609F089C08091D50DAA
:10E680009091D60DA091D70DB091D80D8415950518
:10E69000A605B70569F41092DD0D8FEF9FEFDC0141
:10E6A0008093D50D9093D60DA093D70DB093D80D30
:10E6B0009401B301A2018091DE0D9091DF0D0E94C3
:10E6C00013AF882309F484CFF80180859185A28552
:10E6D000B3858A0D9B1DA11DB11D80879187A287DF
:10E6E000B3878A0C9B1CCA18DB08D80118964D9179
:10E6F0005D916D917C911B97C114D10409F070CF8D
:10E700007AC0E114F10409F084CF14964D915D9123
:10E710006D917C911797411551056105710559F46B
:10E7200055968D919D910D90BC91A02D0097A105BE
:10E73000B10539F520C09E012F5F3F4F64DD88236E
:10E7400009F446CF89819A81AB81BC81F801218D82
:10E75000328DF9012789203139F4883FFFEF9F0777
:10E76000A105B10540F40DC0883F2FEF9207A20725
:10E770002FE0B20730F0C8010E9474AD811149CF7B
:10E7800027CFF80184839583A683B78342CFE11412
:10E79000F10411F5D80118964D915D916D917C9120
:10E7A0001B9751968D919D910D90BC91A02D48176E
:10E7B00059076A077B0780F01DDC882309F408CF1E
:10E7C00081E08093DD0D4092D50D5092D60D609280
:10E7D000D70D7092D80D07C041E0C301B2014ADCE9
:10E7E000882309F4F5CEA501B401C7018B52944FDB
:10E7F0000E945FF369CF51968D919D910D90BC91D0
:10E80000A02D84179507A607B70740F4F801418BA0
:10E81000528B638B748B818180688183D8011196C0
:10E820008C9183FD02C0C10105C0C801D3DD8111F7
:10E83000FACFCECE0F900F900F900F90DF91CF9127
:10E840001F910F91FF90EF90DF90CF90BF90AF900E
:10E850009F908F907F906F905F904F903F902F9000
:10E860000895CF93DF931F92CDB7DEB7698341E060
:10E8700050E0BE016F5F7F4F049673DE0F90DF9113
:10E88000CF9108952F923F924F925F926F927F9215
:10E890008F929F92AF92BF92CF92DF92EF92FF92B0
:10E8A0000F931F93CF93DF9300D01F92CDB7DEB7A6
:10E8B0009C838B834B015A01DC0113968C9181114F
:10E8C00003C08FEF9FEFE9C0EB81FC81818180FF66
:10E8D000F8CFAB81BC8151960D911D912D913C914A
:10E8E000549718964D915D916D917C911B97C50140
:10E8F000A0E0B0E068017901C41AD50AE60AF70A77
:10E90000C816D906EA06FB0618F45801A41AB50A77
:10E9100075018B819C8104969A838983612C92E096
:10E92000792EE114F10409F48AC0AB81BC811896F8
:10E930004D915D916D917C911B976A01B1E0DB2255
:10E94000EB81FC8123811A012B0189E056944794C5
:10E95000379427948A95D1F7818D928D223061F476
:10E96000FC01828D938DA48DB58DBC01CD01620D0E
:10E97000731D841D951D49C0DC0114961C91115016
:10E980001221C114D104F9F411111DC0452B462BDD
:10E99000472B59F4EB81FC8185899689A789B08D35
:10E9A00084839583A683B7830EC0AB81BC81149604
:10E9B0004D915D916D917C91179729813A8123DC6E
:10E9C000882309F47ECFEB81FC81218D328D8481F7
:10E9D0009581A681B7810297A109B109F901058442
:10E9E00004C0880F991FAA1FBB1F0A94D2F746853F
:10E9F000578560897189840F951FA61FB71FBC01B9
:10EA0000CD01610F711D811D911D93012C193D09CF
:10EA100087012E153F0508F489010115F2E01F0753
:10EA200079F52091D50D3091D60D4091D70D5091AB
:10EA3000D80D621773078407950719F421C0C50123
:10EA40002CC09401AB01BC018091DE0D9091DF0DD3
:10EA50000E9475AF882309F434CF800E911EEB819C
:10EA6000FC8180859185A285B385800F911FA11DB2
:10EA7000B11D80879187A287B387E01AF10A51CF31
:10EA800040E0F8DA882309F41CCFB6016B52744FCA
:10EA9000A801C4010E945FF3E0CF0F900F900F9088
:10EAA0000F90DF91CF911F910F91FF90EF90DF902A
:10EAB000CF90BF90AF909F908F907F906F905F901E
:10EAC0004F903F902F900895DF92EF92FF920F9317
:10EAD0001F93CF93DF937C01EB018A018DE0D82E49
:10EAE00040E250E0BE01C701CDDE8032910539F031
:10EAF00021E0892B09F420E0822F81953EC02881F6
:10EB0000222399F1253E61F32E3251F301151105AF
:10EB100041F13B853F733F3021F54A8D5B8D452B9D
:10EB200001F52F713FEF320F3230D8F430E0215031
:10EB30003109D29EC001D39E900D1124D801A80F97
:10EB4000B91FFE0120E0AD01253088F431813D93ED
:10EB50002F5F32962D30C1F7288126FF02C0FA01BF
:10EB600015862B8523FDBCCF08C080E006C02B3066
:10EB700010F43481ECCF3681EACFDF91CF911F9131
:10EB80000F91FF90EF90DF9008954F925F926F92F8
:10EB90007F92AF92BF92CF92DF92EF92FF920F934C
:10EBA0001F93CF93DF931F92CDB7DEB78C017B010C
:10EBB0005A01D22EDB0159968D919C915A97F801FA
:10EBC000928F818F40E050E0BA01C70135DCC12C43
:10EBD000F70180859185A285B38541895289638932
:10EBE000748984179507A607B70708F062C025E067
:10EBF000B695A795979587952A95D1F7F82FFF7029
:10EC00007F2ED70113968C91823008F463C041E0C7
:10EC100050E0BE016F5F7F4FC70134DE019719F4EA
:10EC2000898190E002C08FEF9FEF019609F452C0F6
:10EC3000F70180859185A285B3854F96A11DB11DF1
:10EC400080879187A287B387F0E27F9EC00111245D
:10EC5000BC016B52744F61157105E1F1DB012C9120
:10EC6000222319F0253ED1F465C1C1100EC0409198
:10EC7000D50D5091D60D6091D70D7091D80DF8013A
:10EC80004487558766877787708AFC01EB52F44F7B
:10EC90008081882361F0CC24C3949ACF4BE050E06C
:10ECA000C5010E9452F3892B09F092CF15C0CC24E4
:10ECB000C3948D2D8274823469F4CC2009F489C008
:10ECC000D80150967C9061E0C8010E9458AD009731
:10ECD00009F005C180E031C1D7FCFCCFF0E27F9E96
:10ECE000A00111249A012B52344FD9011B968C910B
:10ECF000817121F08D2D827109F067C08091D50D51
:10ED00009091D60DA091D70DB091D80DF8018487C0
:10ED10009587A687B787708AFA01EB52F44F44892A
:10ED2000558960E070E0BA0155274427D80155960F
:10ED30004D935D936D937C935897828D938DA0E056
:10ED4000B0E0482B592B6A2B7B2BD80155964D935D
:10ED50005D936D937C935897D9011B968C91887124
:10ED600059F4848D958DA68DB78DF801818B928B8A
:10ED7000A38BB48B81E00FC0803139F598012F5EF1
:10ED80003F4FD80159968D919C915A97BDDA8823AF
:10ED9000E1F084E0F80183838D2D8F70D801119606
:10EDA0008C931197F8011482158216821782189697
:10EDB0001D921D921D921C921B97D4FEAFC0C801DC
:10EDC0000E940E9E8111AAC085CFD80113961C9275
:10EDD00081CFF7018381823009F47CCF81899289C8
:10EDE000A389B489803E9F4FAF41B10508F072CF2F
:10EDF000C7010E9474AD882309F46CCFFBD8882327
:10EE000009F468CFD70159962D913C915A971496E1
:10EE10008D919D910D90BC91A02D0297A109B109F2
:10EE2000F901058404C0880F991FAA1FBB1F0A940B
:10EE3000D2F74684578460887188480E591E6A1E2E
:10EE40007B1E81E08093DD0D4092D50D5092D60D52
:10EE50006092D70D7092D80D80E092E0E5EDFBE076
:10EE6000DF019C011D9221503040E1F7CC24C39476
:10EE7000D7015996ED91FC915A978481C81698F460
:10EE800025ED3BE0B301A2014C0D511D611D711D2B
:10EE90008091DE0D9091DF0D0E9413AF882309F45D
:10EEA00019CFC394E5CF80E092E0A0E0B0E0058404
:10EEB00004C0880F991FAA1FBB1F0A94D2F7F7013D
:10EEC0004189528963897489840F951FA61FB71FD2
:10EED000818B928BA38BB48B85ED9BE0712C20E210
:10EEE000DC011D922A95E9F72BE0F501DC01019088
:10EEF0000D922A95E1F721E238E2FC01318B208B5B
:10EF000040E058E057874687338B228B318F208F24
:10EF1000578B468B6FD88111E1CEDCCED5FE08C071
:10EF2000F8014189528963897489C80185DA05C06D
:10EF300081E003C0C110AFCE9ACE0F90DF91CF9188
:10EF40001F910F91FF90EF90DF90CF90BF90AF9007
:10EF50007F906F905F904F9008950F931F93CF9382
:10EF6000DF93FC012381222311F080E043C08B0159
:10EF7000EC01FB018789803131F18032B1F783E008
:10EF80008B83F801428D538D648D758D4D8B5E8B17
:10EF90006F8B788F9E012F5E3F4FC801B5D98823B4
:10EFA00021F31A8F098F81E089831C821D821E82C2
:10EFB0001F82188619861A861B861C861D861E8649
:10EFC0001F86188A17C082E08B831D8A1E8A1F8ABB
:10EFD000188EFB01808D918DA0E0B0E025E0880FB8
:10EFE000991FAA1FBB1F2A95D1F7898B9A8BAB8BD0
:10EFF000BC8BD7CFDF91CF911F910F910895CF9305
:10F00000DF93EB01FC012381211102C080E028C0C5
:10F010002250223020F48FE28883198220C060E0E1
:10F020000E9458AD009791F3FC0190E080E02EE241
:10F030003081303269F0883029F4DE01A90FB11D2A
:10F040002C939F5FDE01A90FB11D30813C939F5F20
:10F050008F5F31968B3061F7C90FD11D188281E027
:10F06000DF91CF910895CF93DF93EC01B3D91B8249
:10F07000DF91CF9108952F923F924F925F926F92BE
:10F080007F928F929F92AF92BF92CF92DF92EF9238
:10F09000FF920F931F93CF93DF93CDB7DEB7C55485
:10F0A000D1090FB6F894DEBF0FBECDBF3C015B01A6
:10F0B0008A01322E1C8E1F8E19821C82672B11F43E
:10F0C00010E0A7C0FC0183818111FACFFA01808191
:10F0D0008F3261F4CA018C010196F80120812F3230
:10F0E000D1F3F50183818250823010F475010AC09A
:10F0F000618D728DCE01019630DF882309F3CE0138
:10F1000001967C016E019CE1C90ED11C26014E01C5
:10F11000E7E38E0E911CFBE0F80D2596FFAF2597D7
:10F12000CE01019624969FAF8EAF24972696CFAE40
:10F1300026972D2C35C080E2819325969FAD25978B
:10F140009E13F9CFD80190E027E04A2F3B2F8D91F5
:10F15000811128C08FA9803209F4B2CF842F932F58
:10F160008C01FC01208101962F32D1F3222309F476
:10F170004AC021E0A401B701C60107DD882309F4D4
:10F180009FCFEA14FB0411F0C7016DDFC414D5044E
:10F1900099F126969FAD2697822D7601C92ED82EFD
:10F1A000F401C9CF8F32B1F28E3219F0EFE9F2E2F9
:10F1B0000AC02A3009F484CF98E02AE0C6CF3196FD
:10F1C000381709F47DCF34913111F9CF291708F49C
:10F1D00077CF813208F474CF8F3709F471CF31E0E3
:10F1E000390FF401E90FF11D9FE9980F9A3108F4E6
:10F1F00080528083932FA9CF23969FAD2397249687
:10F200008FAD2497CACF232DA401B701C301BDDC64
:10F21000182FCE0101960E94CB3ECE014C960E9443
:10F22000CB3E812FCB5BDF4F0FB6F894DEBF0FBE16
:10F23000CDBFDF91CF911F910F91FF90EF90DF90A5
:10F24000CF90BF90AF909F908F907F906F905F9086
:10F250004F903F902F900895AF92BF92CF92DF9240
:10F26000EF92FF920F931F93CF93DF931F92CDB72F
:10F27000DEB77C016B018A01590180919B0B8111E2
:10F2800019C0F701808191810E94D0EF8983F60136
:10F2900081936F01BE016F5F7F4FC5010E94BADA93
:10F2A000F701408151814F5F5F4F5183408301508F
:10F2B000110939F70F90DF91CF911F910F91FF90B6
:10F2C000EF90DF90CF90BF90AF9008958F929F9274
:10F2D000AF92BF92CF92DF92EF92FF920F931F9364
:10F2E000CF93DF931F921F92CDB7DEB7E0919B0BB8
:10F2F000E1114AC059016C018B017B01E40EF51E3E
:10F300000E151F0509F440C0F60180809180F801B8
:10F3100061918F016983C4016A830E94D0EF6A8181
:10F32000681729F1C4010E94D8EFC4010E94D0EFF0
:10F3300099818917E1F0E7E8F8E284918F010F5F86
:10F340001F4F882321F00E94DC3EF801F6CFEFEA40
:10F35000F2E284918F010F5F1F4F882321F00E94FA
:10F36000DC3EF801F6CF81E080939B0B0DC0BE011F
:10F370006F5F7F4FC5010E94BADAF60180819181EB
:10F38000019691838083BCCF0F900F90DF91CF9136
:10F390001F910F91FF90EF90DF90CF90BF90AF90B3
:10F3A0009F908F9008952F923F924F925F926F920D
:10F3B0007F928F929F92AF92BF92CF92DF92EF9205
:10F3C000FF920F931F93CF93DF93CDB7DEB7CA554C
:10F3D000D1090FB6F894DEBF0FBECDBF2DB73EB733
:10F3E00069963FAF2EAF69972F961FAE1EAE2F972F
:10F3F00084E690E02D969FAF8EAF2D979E01235B04
:10F400003F4F44E050E0BE016F5B7F4FCE01855B14
:10F410009F4F22DF9E01235B3F4F42E050E0BE0141
:10F42000675B7F4FCE01855B9F4F16DF43E050E067
:10F43000BE016F5B7F4F84EE92E00E94A1F3892BA7
:10F4400009F43AC022968FAD2297863539F08FE3C2
:10F4500022968FAF229723961FAE2397E7E8F8E214
:10F4600084918F010F5F1F4F882321F00E94DC3EA3
:10F47000F801F6CFE4E6F3E284918F010F5F1F4FAE
:10F48000882321F00E94DC3EF801F6CFBE016F5BBD
:10F490007F4F8BE593E20E94AE4BEDE4F3E2849163
:10F4A0008F010F5F1F4F882321F00E94DC3EF8017F
:10F4B000F6CF0E941355E3C36DB67EB621961CAEFF
:10F4C0001DAE1EAE1FAE21972F961FAE1EAE2F97FC
:10F4D0009E01235B3F4F41E050E0BE016B5A7F4FDE
:10F4E000CE01855B9F4FB8DE80E1E4EBF2E0DE0108
:10F4F000919601900D928A95E1F780E1E4ECF2E0BB
:10F50000DE01519601900D928A95E1F780E1E4EDDC
:10F51000F2E08E010F5F1F4FD80101900D928A9586
:10F52000E1F76696CFAC6697D12C33E0C30ED11CC1
:10F53000CC0CDD1CCC0CDD1C8DB79EB78C199D0945
:10F540000FB6F8949EBF0FBE8DBFEDB7FEB73196D4
:10F550004F012DB73EB72C193D090FB6F8943EBFA9
:10F560000FBE2DBF8DB79EB701965C01EDB7FEB7FC
:10F57000EC19FD090FB6F894FEBF0FBEEDBF2DB715
:10F580003EB72F5F3F4F79019E01235B3F4FA6019E
:10F59000B401CE01855B9F4F5FDE9E01235B3F4F31
:10F5A000A601B501CE01855B9F4F56DE9E01235B10
:10F5B0003F4FA601B701CE01855B9F4F4DDE66969A
:10F5C0002FAD669730E02E5F3F4F85E992E16B9655
:10F5D0009FAF8EAF6B97A5E8B2E162E174E180E086
:10F5E00090E040E050E02417350714F0640105C0B6
:10F5F000F1E2CF2ED12CCC0EDD1EC80ED91EF601A5
:10F600002080318042805380FB01219231924192CF
:10F610005192BF012417350714F0650105C0E1E1DF
:10F62000CE2ED12CCC0EDD1EC80ED91EF6012080A8
:10F630003180428053802D923D924D925D922417ED
:10F64000350714F0670101C06801C80ED91EF60124
:10F6500020803180428053806B96EEADFFAD6B977A
:10F6600021923192419251926B96FFAFEEAF6B9720
:10F670004F5F5F4F04964430510509F0B4CF9E01AF
:10F68000235B3F4F44E050E06DEA72E1CE01855BC1
:10F690009F4FE2DD9E01235B3F4F44E050E069EA6B
:10F6A00072E1CE01855B9F4FD7DD9E01235B3F4F0B
:10F6B00044E050E065EA72E1CE01855B9F4FCCDD0E
:10F6C0009E01235B3F4F44E050E061E872E1CE01D0
:10F6D000855B9F4FC1DD9E01235B3F4F44E050E0BF
:10F6E0006DE772E1CE01855B9F4FB6DD9E01235B26
:10F6F0003F4F44E050E064EC72E1CE01855B9F4FE8
:10F70000ABDD9E01235B3F4F40E150E061EB72E1D6
:10F71000CE01855B9F4FA0DD9E01235B3F4F4CE0F8
:10F7200050E06BE774E0CE01855B9F4F95DD9E0155
:10F73000235B3F4F44E050E0BE01635C7F4FCE014E
:10F74000855B9F4F89DD9E01235B3F4F41E050E089
:10F75000BE016C5A7F4FCE01855B9F4F7DDD9E01C0
:10F76000235B3F4F44E050E0BE01635C7F4FCE011E
:10F77000855B9F4F71DD9E01235B3F4F41E050E071
:10F78000BE016D5A7F4FCE01855B9F4F65DD9E01A7
:10F79000235B3F4F41E050E0BE016E5A7F4FCE01E8
:10F7A000855B9F4F59DD64968FAD649763960FAD6F
:10F7B0006397809F80011124E12CF12C9E01235B33
:10F7C0003F4F44E050E0BE01E016F10651F0635CAB
:10F7D0007F4FCE01855B9F4F3FDDFFEFEF1AFF0AA2
:10F7E000EDCF675C7F4FCE01855B9F4F35DD1AE023
:10F7F00011509E01235B3F4F112351F044E050E034
:10F80000BE01635C7F4FCE01855B9F4F25DDF0CF4E
:10F8100041E050E0BE016F5A7F4FCE01855B9F4FA4
:10F820001BDD9E01235B3F4F41E050E0BE01605B6A
:10F830007F4FCE01855B9F4F0FDD9E01235B3F4FC6
:10F8400044E050E0BE016B5C7F4FCE01855B9F4F73
:10F8500003DD9E01235B3F4F44E050E0BE016F5C3F
:10F860007F4FCE01855B9F4FF7DC62968FAD62972D
:10F8700061960FAD6197809F80011124E12CF12CDE
:10F880009E01235B3F4FE016F10669F044E050E033
:10F89000BE01635C7F4FCE01855B9F4FDDDC2FEFA8
:10F8A000E21AF20AEDCF41E050E0BE016A5A7F4F02
:10F8B000CE01855B9F4FD0DC9E01235B3F4F44E030
:10F8C00050E0BE01635C7F4FCE01855B9F4FC4DC7F
:10F8D0009E01235B3F4F41E050E0BE01615B7F4FE3
:10F8E000CE01855B9F4FB8DC9E01235B3F4F44E018
:10F8F00050E06BE37BE0CE01855B9F4FADDC219652
:10F900001CAE1DAE1EAE1FAE21971CE011509E0115
:10F91000235B3F4F44E050E0112341F0BE01635CA4
:10F920007F4FCE01855B9F4F97DCF0CF6DE57BE08D
:10F93000CE01855B9F4F90DC9E01235B3F4F44E0EF
:10F9400050E067E37BE0CE01855B9F4F85DC9E0145
:10F95000235B3F4F44E050E061E67BE0CE01855BF6
:10F960009F4F7ADC9E01235B3F4F44E050E0BE0195
:10F97000635C7F4FCE01855B9F4F6EDC11113BC0F6
:10F980002196CCACDDACEEACFFAC219720E030E8AA
:10F990004BE355E4C701B6010E941AEC882359F1E4
:10F9A000C0924C0BD0924D0BE0924E0BF0924F0B4D
:10F9B0009E01235B3F4F44E050E064E57BE0CE01D5
:10F9C000855B9F4F49DC9E01235B3F4F44E050E045
:10F9D00060E57BE0CE01855B9F4F3EDC9E01235BB3
:10F9E0003F4F44E050E0BE01635C7F4FCE01855B3A
:10F9F0009F4F32DC10C004E0015069F09E01235B90
:10FA00003F4F44E050E0BE01635C7F4FCE01855B19
:10FA10009F4F22DCF1CF1F5F153009F0A3CF9E016D
:10FA2000235B3F4F42E050E0BE01695B7F4FCE0158
:10FA3000855B9F4F11DC14E011509E01235B3F4F0B
:10FA4000112351F044E050E0BE01635C7F4FCE01D2
:10FA5000855B9F4F01DCF0CF42E050E0BE016B5B65
:10FA60007F4FCE01855B9F4FF7DB9E01235B3F4FAE
:10FA700041E050E0BE016A5A7F4FCE01855B9F4F47
:10FA8000EBDB19E011509E01235B3F4F112351F036
:10FA900044E050E0BE01635C7F4FCE01855B9F4F29
:10FAA000DBDBF0CF41E050E069EA7BE0CE01855B33
:10FAB0009F4FD2DB9E01235B3F4F44E050E0BE01ED
:10FAC000635C7F4FCE01855B9F4FC6DB11110EC07B
:10FAD00021968CAD9DADAEADBFAD21978093A50BAA
:10FAE0009093A60BA093A70BB093A80B1F5F1530A4
:10FAF00009F71BE09E01235B3F4F42E050E0BE014F
:10FB00006B5C7F4FCE01855B9F4FA6DB115091F759
:10FB10009E01235B3F4F44E050E0BE01635C7F4F9A
:10FB2000CE01855B9F4F98DB9E01235B3F4F44E0F6
:10FB300050E0BE01635C7F4FCE01855B9F4F8CDB45
:10FB400014E0115069F09E01235B3F4F44E050E008
:10FB5000BE016F5C7F4FCE01855B9F4F7DDBF1CF98
:10FB60002F962EAD3FAD2F972B968EAD9FAD2B9739
:10FB70002817390709F03AC00E94C86FE7E8F8E291
:10FB800084918F010F5F1F4F811103C004EE12E0BB
:10FB900004C00E94DC3EF801F3CFF80181918F018F
:10FBA000882319F00E94DC3EF8CF2D966EAD7FAD14
:10FBB0002D976456710980E393E20E94954B2F962E
:10FBC0004EAD5FAD2F9760E070E083E293E20E945C
:10FBD0003E4BE0E2F3E284918F010F5F1F4F8823D9
:10FBE00009F448C00E94DC3EF801F5CFEFE3F8E2EB
:10FBF00084918F010F5F1F4F882321F00E94DC3E0C
:10FC0000F801F6CFE0E0F3E284918F010F5F1F4F20
:10FC1000882321F00E94DC3EF801F6CF2B966EADD2
:10FC20007FAD2B9780E090E04AE00E94E33EEBEF4F
:10FC3000F2E284918F010F5F1F4F882321F00E9411
:10FC4000DC3EF801F6CF2F966EAD7FAD2F9780E0AA
:10FC500090E04AE00E94E33EEBEEF2E284918F01F5
:10FC60000F5F1F4F882321F00E94DC3EF801F6CF82
:10FC70000E9413550FB6F8947EBE0FBE6DBE80E095
:10FC80000E94605190919B0B81E0892769962EAD6F
:10FC90003FAD69970FB6F8943EBF0FBE2DBFC65A51
:10FCA000DF4F0FB6F894DEBF0FBECDBFDF91CF910F
:10FCB0001F910F91FF90EF90DF90CF90BF90AF908A
:10FCC0009F908F907F906F905F904F903F902F907C
:10FCD00008958F929F92AF92BF92CF92DF92EF9250
:10FCE000FF920F931F93CF93DF93CDB7DEB7C1552C
:10FCF000D1090FB6F894DEBF0FBECDBF19AE1AAE54
:10FD00001BAE1CAE80E390E3A0E3B0E08DAB9EABF6
:10FD1000AFABB8AF29961FAE1EAE299784E690E030
:10FD200027969FAF8EAF279710929B0B9E01295B62
:10FD30003F4F44E050E0BE016B5C7F4FCE018B5BD8
:10FD40009F4FC4DA27968EAD9FAD279702962796D0
:10FD50009FAF8EAF279729961FAE1EAE299781E0E1
:10FD600062968FAF62979E01295B3F4F41E050E062
:10FD7000BE016F5A7F4FCE018B5B9F4FA7DA9E016A
:10FD8000295B3F4F40E150E062E174E1CE018B5BC3
:10FD90009F4F9CDA9E01295B3F4F40E150E065E8B0
:10FDA00072E1CE018B5B9F4F91DA9E01295B3F4F41
:10FDB00040E150E065E972E1CE018B5B9F4F86DA4E
:10FDC0009E01295B3F4F44E050E06DEA72E1CE01B5
:10FDD0008B5B9F4F7BDA9E01295B3F4F44E050E0F5
:10FDE00069EA72E1CE018B5B9F4F70DA9E01295B5D
:10FDF0003F4F44E050E065EA72E1CE018B5B9F4FDC
:10FE000065DA9E01295B3F4F44E050E061E872E112
:10FE1000CE018B5B9F4F5ADA9E01295B3F4F44E036
:10FE200050E06DE772E1CE018B5B9F4F4FDA9E0190
:10FE3000295B3F4F44E050E064EC72E1CE018B5B04
:10FE40009F4F44DA9E01295B3F4F40E150E061EB58
:10FE500072E1CE018B5B9F4F39DA9E01295B3F4FE8
:10FE60004CE050E06BE774E0CE018B5B9F4F2EDAE5
:10FE700080E090E0A0E2B1E489AB9AABABABBCAB65
:10FE80009E01295B3F4F44E050E0BE016F5C7F4F15
:10FE9000CE018B5B9F4F1ADA61961FAE619719AE48
:10FEA0001AAE1BAE1CAE83E060968FAF60972F96A4
:10FEB0008FAF2F979E01295B3F4F41E050E0BE017D
:10FEC000605B7F4FCE018B5B9F4F00DA9E01295B09
:10FED0003F4F44E050E0BE01675C7F4FCE018B5B3B
:10FEE0009F4FF4D99E01295B3F4F41E050E0BE0196
:10FEF000615B7F4FCE018B5B9F4FE8D99E01295BF1
:10FF00003F4F41E050E0BE01625B7F4FCE018B5B13
:10FF10009F4FDCD91AE0115069F09E01295B3F4FD9
:10FF200044E050E0BE01675C7F4FCE018B5B9F4F8A
:10FF3000CDD9F1CF1DA61EA61FA618AA9E01295B2A
:10FF40003F4F44E050E0BE01635D7F4FCE018B5BCD
:10FF50009F4FBCD919AE1AAE1BAE1CAE1AE01150A1
:10FF600069F09E01295B3F4F44E050E0BE01675CB1
:10FF70007F4FCE018B5B9F4FA9D9F1CF83E02E96A7
:10FF80008FAF2E972D968FAF2D9719A61AA61BA669
:10FF90001CA61DA21EA21FA218A619AE1AAE1BAE49
:10FFA0001CAE9E01295B3F4F41E050E0BE01635B08
:10FFB0007F4FCE018B5B9F4F89D99E01295B3F4FBD
:10FFC00041E050E0BE01645B7F4FCE018B5B9F4FF1
:10FFD0007DD99E01295B3F4F44E050E0BE016B5D3F
:10FFE0007F4FCE018B5B9F4F71D99E01295B3F4FA5
:10FFF00044E050E0BE01675D7F4FCE018B5B9F4FB9
:020000021000EC
:1000000065D90AE010E00150110969F09E01295BF1
:100010003F4F44E050E0BE01675C7F4FCE018B5BF9
:100020009F4F54D9F0CF2C961FAE2C9719AE1AAE15
:100030001BAE1CAE8FEF2B968FAF2B979E01295BCB
:100040003F4F41E050E0BE01655B7F4FCE018B5BCF
:100050009F4F3CD99E01295B3F4F44E050E0BE01D9
:10006000675C7F4FCE018B5B9F4F30D99E01295B30
:100070003F4F41E050E0BE01665B7F4FCE018B5B9E
:100080009F4F24D99E01295B3F4F44E050E06BE332
:100090007BE0CE018B5B9F4F19D919AE1AAE1BAE18
:1000A0001CAE1CE011509E01295B3F4F44E050E024
:1000B000112341F0BE01675C7F4FCE018B5B9F4FE8
:1000C00005D9F0CF6DE57BE0CE018B5B9F4FFED86D
:1000D0009E01295B3F4F44E050E067E37BE0CE01A7
:1000E0008B5B9F4FF3D89E01295B3F4F44E050E06C
:1000F00061E67BE0CE018B5B9F4FE8D8C12C80E8A6
:10010000D82E8BE3E82E85E4F82E812C912C90E8F4
:10011000A92E9FE3B92E111132C09E01295B3F4FDA
:1001200044E050E06CE47BE0CE018B5B9F4FCED887
:100130009E01295B3F4F44E050E064E57BE0CE0147
:100140008B5B9F4FC3D89E01295B3F4F44E050E03B
:1001500060E57BE0CE018B5B9F4FB8D889AE9AAE4D
:10016000ABAEBCAE9E01295B3F4F44E050E0BE0108
:10017000675C7F4FCE018B5B9F4FA8D824C0C9AE70
:10018000DAAEEBAEFCAE9E01295B3F4F44E050E09F
:10019000BE01675C7F4FCE018B5B9F4F97D819AE36
:1001A0001AAE1BAE1CAE04E0015069F09E01295B43
:1001B0003F4F44E050E0BE01675C7F4FCE018B5B58
:1001C0009F4F84D8F1CF1F5F153009F0A4CF84E191
:1001D00090E025969FAF8EAF25979E01295B3F4FFC
:1001E00042E050E0BE016D5B7F4FCE018B5B9F4FC5
:1001F0006DD880E090E8ABE3B5E489AF9AAFABAFE0
:10020000BCAF14E0115069F09E01295B3F4F44E000
:1002100050E0BE01675C7F4FCE018B5B9F4F56D88D
:10022000F1CF80E290E023969FAF8EAF23979E019F
:10023000295B3F4F42E050E0BE016F5B7F4FCE0134
:100240008B5B9F4F43D82A961FAE2A9780E090E0A1
:10025000A0E4B0E489A39AA3ABA3BCA380E090E0A0
:10026000A4E3B2E48D8F9E8FAF8FB8A3198E1A8E40
:100270001B8E1C8E1D8A1E8A1F8A188E198A1A8A46
:100280001B8A1C8A80E090E0A0E5B1E48D879E8700
:10029000AF87B88B19861A861B861C8680E090E093
:1002A000A0E0B1E48D839E83AF83B8879E01295B74
:1002B0003F4F41E050E0BE01675B7F4FCE018B5B5B
:1002C0009F4F04D89E01295B3F4F44E050E0BE01A0
:1002D0006F5D7F4FCE018B5B9F4F0E9466799E01C1
:1002E000295B3F4F44E050E0BE01635E7F4FCE018B
:1002F0008B5B9F4F0E9466799E01295B3F4F44E0D4
:1003000050E0BE01675E7F4FCE018B5B9F4F0E9426
:1003100066799E01295B3F4F44E050E0BE016B5E71
:100320007F4FCE018B5B9F4F0E9466799E01295BB8
:100330003F4F44E050E0BE016F5E7F4FCE018B5BCC
:100340009F4F0E9466799E01295B3F4F44E050E039
:10035000BE01635F7F4FCE018B5B9F4F0E9466792A
:100360009E01295B3F4F44E050E0BE01675F7F4F35
:10037000CE018B5B9F4F0E9466799E01295B3F4FA8
:1003800044E050E0BE016B5F7F4FCE018B5B9F4F1F
:100390000E9466799E01295B3F4F41E050E069EA87
:1003A0007BE0CE018B5B9F4F0E94667911110CC0E0
:1003B0008091A50B9091A60BA091A70BB091A80BD3
:1003C00089AF9AAFABAFBCAF9E01295B3F4F44E012
:1003D00050E0BE01675C7F4FCE018B5B9F4F0E9458
:1003E00066791F5F153011F721961FAE1EAE21975B
:1003F0001CE0115071F09E01295B3F4F42E050E03C
:10040000BE01615C7F4FCE018B5B9F4F0E9466797E
:10041000F0CF19AE1AAE1BAE1CAE9E01295B3F4F4A
:1004200044E050E0BE01675C7F4FCE018B5B9F4F85
:100430000E9466799E01295B3F4F44E050E0BE0177
:10044000675C7F4FCE018B5B9F4F0E94667919825C
:100450001A821B821C8214E0115071F09E01295BEC
:100460003F4F44E050E0BE016F5F7F4FCE018B5B9A
:100470009F4F0E946679F0CF80919B0B811150C0F5
:100480002796EEACFFAC279729968EAD9FAD2997A6
:100490009EAF8DAF84E690E027969FAF8EAF2797F3
:1004A0009E01295B3F4F44E050E064EE72E0CE01D4
:1004B0008B5B9F4F0E9466799E01295B3F4F42E014
:1004C00050E0BE01635C7F4FCE018B5B9F4F0E946B
:1004D0006679E7E8F8E284918F010F5F1F4F882368
:1004E00021F00E94DC3EF801F6CFB7016456710995
:1004F00089ED92E20E94954B4DAD5EAD60E070E0FB
:100500008CEC92E20E943E4BE9ECF2E284918F0186
:100510000F5F1F4F882321F00E94DC3EF801F6CFC9
:1005200090919B0B81E08927CF5ADF4F0FB6F8944B
:10053000DEBF0FBECDBFDF91CF911F910F91FF9016
:10054000EF90DF90CF90BF90AF909F908F900895E5
:10055000CF92DF92EF92FF920F931F93CF93DF938F
:100560006C017A018B01C0E0D0E0CE15DF0589F087
:10057000D8016D918D01D601ED91FC910190F08132
:10058000E02DC6011995892B11F47E0102C0219638
:10059000ECCFC701DF91CF911F910F91FF90EF90AA
:1005A000DF90CF90089590E0FC013197E231F105A2
:1005B00008F04EC08827E458FF4F8F4F0C9438F353
:1005C000809180008F7703C0809180008F7D809321
:1005D0008000089580918000877FF9CF84B58F7760
:1005E00002C084B58F7D84BD08958091B0008F775F
:1005F00003C08091B0008F7D8093B00008958091FA
:1006000090008F7707C0809190008F7D03C080910C
:100610009000877F8093900008958091A0008F774D
:1006200007C08091A0008F7D03C08091A000877FCC
:100630008093A0000895809120018F7707C080915A
:1006400020018F7D03C080912001877F809320014E
:1006500008953FB7F8948091A10B9091A20BA091BF
:10066000A30BB091A40B26B5A89B05C02F3F19F092
:100670000196A11DB11D3FBFBA2FA92F982F882722
:10068000820F911DA11DB11DBC01CD0142E0660F7D
:10069000771F881F991F4A95D1F7089508950895E7
:1006A000FC01A681B7818281481B8581483018F002
:1006B000A80FB11D4770382F369536953695562FB1
:1006C000577080E890E002C0959587955A95E2F7BB
:1006D000439F402D1124669566956695E62FF0E0C0
:1006E000E40FF11DEA0FFB1F3081222311F0832B51
:1006F00002C08095832380830895FB014181DC0142
:1007000012962C911297421760F013962C91139722
:10071000241738F0608115962C91621710F424810B
:10072000BFCF0895FC0180819281980F928321812F
:10073000921760F494819F5F94839381890F82174D
:1007400010F08FEF820F838381E0089580E0089599
:10075000FC0112828081815083831482089580E09D
:1007600008950E9446F3CF93DF93282F30E0F901DC
:10077000E95AFB4D8491F901EF5EFB4DD491F901EB
:10078000E553FC4DC491CC2389F081110CDFEC2F93
:10079000F0E0EE0FFF1FEF54FC4DA591B491EC91EA
:1007A000ED2381E090E021F480E002C080E090E061
:1007B000DF91CF9108951F93CF93DF93282F30E0DF
:1007C000F901E95AFB4D8491F901EF5EFB4DD4919B
:1007D000F901E553FC4DC491CC23C1F0162F8111D2
:1007E000E2DEEC2FF0E0EE0FFF1FE956FC4DA59185
:1007F000B4918FB7F894111105C09C91ED2FE0953D
:10080000E92302C0EC91ED2BEC938FBFDF91CF91E8
:100810001F910895CF93DF9390E0FC01EF5EFB4DB5
:100820002491FC01E553FC4D8491882361F190E013
:10083000880F991FFC01E358FC4DC591D491FC0130
:10084000E956FC4DA591B491611109C09FB7F89488
:100850008881209582238883EC912E230BC06230FF
:1008600061F49FB7F8943881822F80958323888321
:10087000EC912E2B2C939FBF06C08FB7F894E88184
:100880002E2B28838FBFDF91CF9108951F93CF9395
:10089000DF93182FEB0161E0BDDF209711F460E0DA
:1008A00004C0CF3FD10531F461E0812FDF91CF91BA
:1008B0001F9181CFE12FF0E0E95AFB4DE4914E2FDB
:1008C00050E0FA013197E231F10508F09DC0882728
:1008D000E257FF4F8F4F0C9438F384B5806884BD86
:1008E000C7BD97C084B5806284BDC8BD92C08091E9
:1008F0008000806880938000D0938900C093880036
:1009000088C080918000806280938000D0938B00AB
:10091000C0938A007EC080918000886080938000B0
:10092000D0938D00C0938C0074C08091B00080681B
:100930008093B000C093B3006CC08091B00080621F
:100940008093B000C093B40064C080919000806830
:1009500080939000D0939900C09398005AC08091E2
:100960009000806280939000D0939B00C0939A0087
:1009700050C080919000886080939000D0939D003B
:10098000C0939C0046C08091A00080688093A00026
:100990008091A0008F7B8093A000D093A900C0938A
:1009A000A80037C08091A00080628093A000D093FF
:1009B000AB00C093AA002DC08091A00088608093F6
:1009C000A000D093AD00C093AC0023C08091200163
:1009D000806880932001D0932901C093280119C019
:1009E00080912001806280932001D0932B01C093DD
:1009F0002A010FC080912001886080932001D0934C
:100A00002D01C0932C0105C0C038D1050CF04CCF8E
:100A100046CFDF91CF911F9108958F929F92AF9211
:100A2000BF92CF92DF92EF92FF926B017C0111DEB9
:100A30004B015C01C114D104E104F104E9F009DEC9
:100A4000DC01CB0188199909AA09BB09883E9340AA
:100A5000A105B10578F321E0C21AD108E108F10837
:100A600088EE880E83E0981EA11CB11CC114D1042D
:100A7000E104F10421F7DECFFF90EF90DF90CF90FB
:100A8000BF90AF909F908F9008952FB7F89460918A
:100A90009D0B70919E0B80919F0B9091A00B2FBF8F
:100AA00008951F920F920FB60F9211242F933F9328
:100AB0008F939F93AF93BF9380919D0B90919E0BCB
:100AC000A0919F0BB091A00B30919C0B23E0230FC2
:100AD0002D3720F40196A11DB11D05C026E8230F76
:100AE0000296A11DB11D20939C0B80939D0B9093AA
:100AF0009E0BA0939F0BB093A00B8091A10B9091A4
:100B0000A20BA091A30BB091A40B0196A11DB11D46
:100B10008093A10B9093A20BA093A30BB093A40B73
:100B2000BF91AF919F918F913F912F910F900FBEE9
:100B30000F901F9018951F920F920FB60F921124CD
:100B40000BB60F922F933F934F935F936F937F93C7
:100B50008F939F93AF93BF93EF93FF93E091160210
:100B6000F09117021995FF91EF91BF91AF919F916D
:100B70008F917F916F915F914F913F912F910F9046
:100B80000BBE0F900FBE0F901F9018951F920F92E3
:100B90000FB60F9211240BB60F922F933F934F93E2
:100BA0005F936F937F938F939F93AF93BF93EF93D5
:100BB000FF93E0911402F09115021995FF91EF91C6
:100BC000BF91AF919F918F917F916F915F914F9165
:100BD0003F912F910F900BBE0F900FBE0F901F9063
:100BE00018951F920F920FB60F9211240BB60F9209
:100BF0002F933F934F935F936F937F938F939F9325
:100C0000AF93BF93EF93FF93E0910A02F0910B0231
:100C10001995FF91EF91BF91AF919F918F917F9126
:100C20006F915F914F913F912F910F900BBE0F905D
:100C30000FBE0F901F9018951F920F920FB60F9234
:100C400011240BB60F922F933F934F935F936F93A3
:100C50007F938F939F93AF93BF93EF93FF93E09115
:100C60000802F09109021995FF91EF91BF91AF91A0
:100C70009F918F917F916F915F914F913F912F91B4
:100C80000F900BBE0F900FBE0F901F9018951F92E4
:100C90000F920FB60F9211240BB60F922F933F9322
:100CA0004F935F936F937F938F939F93AF93BF9374
:100CB000EF93FF93E0911202F09113021995FF91C7
:100CC000EF91BF91AF919F918F917F916F915F91C4
:100CD0004F913F912F910F900BBE0F900FBE0F9031
:100CE0001F9018951F920F920FB60F9211240BB6FA
:100CF0000F922F933F934F935F936F937F938F93B5
:100D00009F93AF93BF93EF93FF93E0911002F09105
:100D100011021995FF91EF91BF91AF919F918F9122
:100D20007F916F915F914F913F912F910F900BBEEB
:100D30000F900FBE0F901F9018951F920F920FB635
:100D40000F9211240BB60F922F933F934F935F9303
:100D50006F937F938F939F93AF93BF93EF93FF9383
:100D6000E0910E02F0910F021995FF91EF91BF9162
:100D7000AF919F918F917F916F915F914F913F9133
:100D80002F910F900BBE0F900FBE0F901F901895D4
:100D90001F920F920FB60F9211240BB60F922F9342
:100DA0003F934F935F936F937F938F939F93AF93F3
:100DB000BF93EF93FF93E0910C02F0910D02199510
:100DC000FF91EF91BF91AF919F918F917F916F9123
:100DD0005F914F913F912F910F900BBE0F900FBEDF
:100DE0000F901F901895CF92DF92FF920F931F9351
:100DF000CF93DF931F921F92CDB7DEB76901DB015E
:100E000012960D911C911397423309F470C0B8F4F7
:100E1000453109F477C0473109F487C0443109F0FE
:100E20009DC0D80115962C9115971696ED91FC91C1
:100E30001797CF01820F911D820F911D5CC0463420
:100E400009F483C0473409F484C04B3309F086C0E9
:100E5000F90181819381913029F0933031F4482F49
:100E6000885004C048E0480F01C0482F21E0D80155
:100E700013963C91381708F420E031E0F8015281D4
:100E8000451708F430E051E0481708F050E0822F91
:100E9000852B382319F4252309F460C0D601129656
:100EA000FC90913051F030F0923049F0933051F491
:100EB0002FEF09C020E031E007C021E004C020E0AE
:100EC0003FEF02C020E030E0F7FE07C0B601C801E6
:100ED0002A83398312DC39812A81F6018081830FCC
:100EE00080838181820F8183FF0C71F737C0B90144
:100EF000C80103DC33C01192E817F907E1F7C80114
:100F000027DC2CC0C8010EDC882349F1F8012581BB
:100F10000680F781E02DCF01820F911D820F911D78
:100F20001192E817F907E1F719C0D9011C92F801ED
:100F3000828111968C9311978581815012968C93A2
:100F40001297838113968C9309C0D80115968C91C2
:100F500003C0D80111968C91F601808381E00F9037
:100F60000F90DF91CF911F910F91FF90DF90CF9065
:100F70000895DB01ED91FC9119948F929F92BF929D
:100F8000CF92DF92EF92FF920F931F93CF93DF9355
:100F90001F92CDB7DEB74C01062FF42E122F522F21
:100FA000E62EE20EBB24BA946C018CE1C80ED11C73
:100FB0008E2D851B583078F0F40162817381848F07
:100FC000F58E178EB68E96014BE3C4015983D1DF9F
:100FD00059815850EDCF812F887F080F212F27701E
:100FE00019F187E02827F40162817381048FF58E5F
:100FF000178E2F5F27708FEF90E001C0880F2A9522
:10100000EAF7868F9401245E3F4F4BE3C4010F90B3
:10101000DF91CF911F910F91FF90EF90DF90CF90D4
:10102000BF909F908F90A5CF0F90DF91CF911F9190
:101030000F91FF90EF90DF90CF90BF909F908F9097
:101040000895EF92FF920F931F93CF93DF937C014C
:10105000D62F122FC42F040F212F4C2F6D2FC70115
:101060008CDFCF5F0C13F8CFDF91CF911F910F91E1
:10107000FF90EF900895DF92EF92FF920F931F93EE
:10108000CF93DF93EC01162FF42EE22E0E94BD6663
:10109000882329F02E2D4F2D612FCE01D2DFDF9135
:1010A000CF911F910F91FF90EF90DF900895EF92F5
:1010B000FF920F931F93CF93DF931F92CDB7DEB7AD
:1010C0008C01DC011296ED90FC901397D196ED9176
:1010D000FC91D29782E0199520E030E04AE0B70118
:1010E000C80147DFF82ED801D196ED91FC91D29737
:1010F00083E01995D801D196ED91FC91D29780E0CB
:101100001995FF2081F1F801628173819E012F5FA3
:101110003F4F46E4C8012DDF8981D8018C93129698
:101120006D917C9113979E012F5F3F4F47E4C8015B
:1011300020DF8981F80181836281738120E030E0C2
:1011400048E4C80116DFD8011B968C931B979801C1
:101150002D5C3F4F12966D917C91139747E1C8012A
:1011600008DF81E001C080E00F90DF91CF911F91F7
:101170000F91FF90EF9008952F923F925F926F92A0
:101180007F928F929F92AF92BF92CF92DF92EF9217
:10119000FF920F931F93CF93DF931F92CDB7DEB7CC
:1011A0001C01C62E142FD22EDC011496ED90FC905B
:1011B0001597C7010E94A266082FF10184819581CD
:1011C0000E94A566982E013019F48FE0A82E02C067
:1011D000AA24AA94D10114968D919C9115970E94EE
:1011E0009A66082FF101848195810E949666B82E37
:1011F000D10114968D919C9115970E949E66B0E640
:10120000BD1530F4009721F0E80EF91E01E611C07B
:10121000F101848195810E94A066F0E4FD1530F40F
:10122000009721F0E80EF91E01E403C021E1E20E6F
:10123000F11CBD1480F4D10150961C925097539626
:101240001C92539754961C92549751961C92519706
:1012500052961C92C6C0B01670F3892D90E0F7012B
:1012600024912F3F21F4FFEFEF1AFF0A5AC00D110E
:101270004FC0D10114968D919C9115970E94A26642
:1012800097012F5F3F4FF701882311F08230E1F47F
:101290008491D10153968C935397F90124915496DC
:1012A0002C935497F7013396E4915096EC93509712
:1012B000F7013496E4915196EC935197F7013596E6
:1012C000E4915296EC9320C08491982F9F70925095
:1012D000D10152969C93529782958F7051968C9320
:1012E0005197F9012491822F8F7054968C935497C3
:1012F00022952F7053962C935397F7013296E491D1
:10130000E295EF705096EC93E114F10479F469C022
:10131000F7013296E491EA219C012E0F311DE20E75
:10132000F31E0B1509F487CF0F5F99CFF10184816C
:1013300095810E94A566B82ED10153969C90539733
:101340005496DC90549751968C915197C80E5296B2
:101350009C919D0D512E591A0D2D292D452D6C2D29
:10136000C1010E94BD668823C9F1C7018B0D911D83
:101370005C0187E0890DF82EF694F694F694D50C6E
:1013800041019CE1890E911C6F2C712C5D1431F18F
:101390005C2D8501802F8A198F15E0F4F801849166
:1013A000D10112966D917C9113975C965C935C973A
:1013B0005D965C925D975F961C925F975E968C93AC
:1013C00094014BE3C1015983D4DD0F5F1F4F598155
:1013D000585FE0CFA60CB71C5394D8CFF101808999
:1013E00001C080E00F90DF91CF911F910F91FF908E
:1013F000EF90DF90CF90BF90AF909F908F907F90B5
:101400006F905F903F902F900895CF92DF92EF9270
:10141000FF921F93CF93DF9310927E0B8091D8138E
:101420009091D913A091DA13B091DB1381309048D9
:10143000A105B10540F01092D8131092D913109263
:10144000DA131092DB13C091D8138091B00B1816E9
:10145000DCF4282F082E000C330B215031094C2FBF
:101460000C2E000C550B4217530774F0CFEFC80F2A
:101470008C2F90E0A0E0B0E08093D8139093D91324
:10148000A093DA13B093DB131092AA0B8091410B57
:10149000C81714F4C093410B8091410B082E000C27
:1014A000990B04962C2F0C2E000C330B82179307EC
:1014B00024F48CEF8C0F8093410B1091410BD0E002
:1014C00081E0EE24E394F12C22E0C22ED12C111104
:1014D00025C08823B1F01C16A4F08091D8139091F8
:1014E000D913A091DA13B091DB130196A11DB11DA0
:1014F0008093D8139093D913A093DA13B093DB138E
:10150000CF5F80915B02882309F446C020E041E070
:101510006CEB75E28D2F0E94E7E53EC01130E1F4DF
:101520008091800B811105C080915B028823A1F11D
:101530000BC0C130C9F7D092430BC092420B8091CF
:10154000AA0B882389F331C081E0C13009F080E023
:1015500020E24FEA55E21DC01230F1F48091800B79
:10156000811105C080915B028823B1F00BC0C230AD
:10157000C9F7F092430BE092420B8091AA0B8823AB
:1015800089F313C081E0C23009F080E020E242EA32
:1015900055E26D2F0E94DA6BDF5F1F5F80E0D53070
:1015A00009F095CF83E08093B00BDF91CF911F912D
:1015B000FF90EF90DF90CF9008950F931F93CF93FC
:1015C000DF9310927E0B8091D8139091D913A09144
:1015D000DA13B091DB1381309048A105B10540F0DA
:1015E0001092D8131092D9131092DA131092DB13C1
:1015F000C091D8138091AF0B1816DCF4282F082E59
:10160000000C330B215031094C2F0C2E000C550BC4
:101610004217530774F0CFEFC80F8C2F90E0A0E073
:10162000B0E08093D8139093D913A093DA13B093BA
:10163000DB131092AA0B8091410BC81714F4C093CE
:10164000410B8091410B082E000C990B04962C2F16
:101650000C2E000C330B8217930724F48CEF8C0FA5
:101660008093410B1091410BD0E081E002E0111119
:1016700022C08823B1F01C16A4F08091D813909159
:10168000D913A091DA13B091DB130196A11DB11DFE
:101690008093D8139093D913A093DA13B093DB13EC
:1016A000CF5F80915B02882309F468C021E041E0AC
:1016B00063E975E24DC0113011F58823B1F0C230F5
:1016C000A4F48091D8139091D913A091DA13B0911A
:1016D000DB130196A11DB11D8093D8139093D913EC
:1016E000A093DA13B093DB13CF5F80915B02882362
:1016F00009F444C020E040E06EE775E229C01230F2
:10170000E9F48091800B811105C080915B028823F0
:10171000A9F109C0C230C9F70E94D5B88091AA0BBF
:10172000882399F333C081E0C23009F080E024E0DF
:1017300049E755E26D2F0E94DA6B20C0133061F447
:1017400080915B028823D1F020E041E067E775E2F9
:101750008D2F0E94E7E512C0143081F480915B0266
:10176000882351F021E040E06CE675E28D2F0E9465
:10177000E7E58D2F0E9477E500935B02DF5F1F5F37
:1017800080E0D53009F073CFD093AF0BDF91CF91CC
:101790001F910F910895AF92BF92CF92DF92EF9277
:1017A000FF920F931F93CF93DF93CDB7DEB76F9761
:1017B0000FB6F894DEBF0FBECDBF80915B028111E2
:1017C00005C08091800B882309F4C8C185EC9EE098
:1017D0009093C40E8093C30E81E090E09093FD102F
:1017E0008093FC101092FF101092FE1040E050E029
:1017F000BA0189EC9EE00E941C728091C30E909108
:10180000C40E2BE1FC013496DE01159601900D9279
:101810002A95E1F7FC01828193819C838B838CEE76
:1018200092E09A83898340E050E0BE016F5F7F4F72
:101830008BE693E00E943EA1CE0101960E94E6B3A2
:10184000A090FE10B090FF1010927E0B8091D813E4
:101850009091D913A091DA13B091DB1381309048A5
:10186000A105B10540F01092D8131092D91310922F
:10187000DA131092DB131091D8138091AE0B181667
:10188000DCF4282F082E000C330B21503109412F96
:10189000012E000C550B4217530774F01FEF180F61
:1018A000812F90E0A0E0B0E08093D8139093D913FB
:1018B000A093DA13B093DB131092AA0B8091410B23
:1018C000181714F41093410B8091410B082E000C53
:1018D000990B0496212F012E000C330B82179307CE
:1018E00024F48CEF810F8093410B0091410BF12C7C
:1018F00021E0A21AB10801111BC08091800B811157
:1019000005C080915B02882399F009C01111F9CFBD
:101910000E94D5B88091AA0B882399F31FC181E05A
:10192000111180E024E047E655E26F2D0E94DA6B4A
:101930006AE77EE089EC9EE00E94FF7780917A0E54
:101940008F32C1F10130C1F58091800B882319F1EC
:10195000113009F580911A108823D1F081508093BD
:101960001A10EFE18E9FC0011124FC01E851F14FE4
:101970002BE1A9ECBEE001900D922A95E1F7FC0164
:10198000EC51F14F828193819093C80E8093C70EE2
:101990001092410B26C080915B02882369F081E0A0
:1019A000113009F080E020E243E655E26F2D0E94FD
:1019B000DA6B02C091E001C092E06501EE24E3948D
:1019C000E00E2EC08AE00E94DC3ECE0101960E940D
:1019D000E6B31092D8131092D9131092DA13109222
:1019E000DB1381E08093AA0B83E080935B02B6C097
:1019F0000913ABC060E070E0C6010E94E8989091C6
:101A0000790E8091800B992309F482C081110DC059
:101A100080915B02811177C09E2DF1E0CF1AD10831
:101A20002FEFC216D20621F792C01013F1CFCE01CC
:101A300001960E94F06F8091CC0E882319F005EC7E
:101A40001EE002C004EA1EE07801F4E0EF0EF11C93
:101A500021E04AE75EE0B701CE0105960E943B789F
:101A6000811124C0E7E8F8E284918F010F5F1F4FD6
:101A7000882321F00E94DC3EF801F6CFEDE4F5E288
:101A800084918F010F5F1F4F811103C00AE71EE091
:101A900004C00E94DC3EF801F3CFF80181918F0170
:101AA000882309F48FCF0E94DC3EF7CF80911A1073
:101AB0008A30C8F491E0980F90931A10FFE18F9F3D
:101AC000C0011124DC01A851B14F2BE1F7010190B5
:101AD0000D922A95E1F7F80122813381FC01EC5146
:101AE000F14F338322838BE1FE013596A9ECBEE0F2
:101AF00001900D928A95E1F78B819C819093C80E9D
:101B00008093C70E62CF81E0101380E041E019C0DE
:101B1000811106C080915B02882309F47DCF0DC03E
:101B20001013F8CF8AE79EE00E944F9B0E94CFB827
:101B30008091AA0B882371F311C081E0101380E01B
:101B400040E06F2D0E9460DB67CF9F5F66CFF3940C
:101B50000F5F85E0F812CFCE9093AE0B6F960FB665
:101B6000F894DEBF0FBECDBFDF91CF911F910F91D3
:101B7000FF90EF90DF90CF90BF90AF9008952F929D
:101B80003F924F925F926F927F928F929F92AF920D
:101B9000BF92CF92DF92EF92FF920F931F93CF935A
:101BA000DF9310927E0B8091D8139091D913A0915E
:101BB000DA13B091DB1381309048A105B10540F0F4
:101BC0001092D8131092D9131092DA131092DB13DB
:101BD000C091D8138091AD0B1816DCF4282F082E75
:101BE000000C330B215031094C2F0C2E000C550BDF
:101BF0004217530774F0CFEFC80F8C2F90E0A0E08E
:101C0000B0E08093D8139093D913A093DA13B093D4
